:0A0000000C94BF000C9400000C9457
:10000A0000000C9400000C9400000C9400000C9466
:10001A0000000C9400000C9400000C9400000C9456
:10002A0000000C94EE000C9400000C9400000C9458
:10003A0000000C9400000C9400000C9400000C9436
:10004A0055010C9400000C9422010C9400000C94AD
:10005A0000000C9400000C9400000C9400000C9416
:10006A00EC610C9400000C9400000C9400000C94B9
:10007A0000001027E80364000A00010000100001D4
:10008A0010000100000000000A0009000100010040
:10009A000A0A0A0A0A0A0A0A0A0A0A0A0A0A0A0AB6
:1000AA000100080008000A00D60001000100010052
:1000BA0001000100FBFFFBFFFBFFFBFF2800E80339
:1000CA000000000000000000000000000000000026
:1000DA000000000000000000000000000000000016
:1000EA000000000000000000000000000000000006
:1000FA0000000000000000000000000000000000F6
:10010A00000000000700020002008E000200040046
:10011A009000010008059200010005079400010003
:10012A002B07960001002C07980010002E079A0052
:10013A0001006F07AA0001007F07AC0001008007D9
:10014A00AE0001009F07B0000100F307B2000700EC
:10015A001B08B40001004708BC000800AC08BE0038
:10016A0001007C09C60002007D09C8000100A1093E
:10017A000E010000F894EE27EFBBF1E0F5BFE5BFF2
:10018A008DE0A2E0BB27ED938A95E9F780E090E144
:10019A00A0E0B1E0ED930197E9F7E0E1F1E08591A4
:1001AA009591009761F0A591B59105901590BF01C1
:1001BA00F00105900D920197E1F7FB01F0CFE4E021
:1001CA00EEBBEFEFEDBFE0E1EEBFC0E0D5E00C948F
:1001DA00A2018A93AA93BA93EA93FA93EFB7EA939E
:1001EA00E0E0E0937A00E09171070E946F63AE0F3E
:1001FA00BF1FE0917800F0917900ED93FC93E091B4
:10020A007107EF5FE0937107A0917107A83018F0AA
:10021A00E0E0E0937107E0917107E0937C0088E0E9
:10022A008A95F1F7E7ECE0937A00E991EFBFF9914B
:10023A00E991B991A99189911895AA93EA93FA93A8
:10024A00EFB7EA931A930A931091C0000091C6007F
:10025A00E12FEC71E9F4E0919C09EF5FE0939C09CE
:10026A00E150F0E0E557F64F0083A0919C09A131D7
:10027A0019F4E0E0E0939C09A0919E09AF5FA09376
:10028A009E09A13129F4E0E0E0939E09689433F8CD
:10029A0009911991E991EFBFF991E991A9911895FD
:1002AA000A92AA93BA93EA93FA93EFB7EA93E09180
:1002BA008707F09188073196E0938707F0938807BC
:1002CA00A0918707B0918807A83BE0E0BE0719F420
:1002DA00E1E0E0933205A0918707B0918807A03743
:1002EA00E1E0BE0741F4E2E0E0933205E0E0E093AA
:1002FA008707E09388070E9475630E947A630E94C9
:10030A007563E8EDF9E50E94AD7DE02149F0E091E1
:10031A00D107F091D2073196E093D107F093D20733
:10032A00E0912207EF5FE0932207E991EFBFF9918D
:10033A00E991B991A99109901895EF97249783E4C7
:10034A00A0E0B0E0EAECF0E00E94F67EFF2450E084
:10035A00E0E8E0936100E0E0E0936100E1B9E2B92E
:10036A00EAEFE4B9E5E0E5B9ECE3E7B9E3ECE8B9CB
:10037A00E0EFEAB9ECE0EBB9E1EAE4BDE3E0E5BDC0
:10038A00E0E0E6BD0E948063E1EAE0938000E3E0FA
:10039A00E0938100E0E0E0938500E0938400E0933D
:1003AA008700E0938600E0938900E0938800E09359
:1003BA008B00E0938A00E093B600E1EAE093B00094
:1003CA00E2E0E093B100E0E0E093B200E093B30032
:1003DA00E093B400E1E0E0936E00E0E0E0936F00A8
:1003EA00E1E0E0937000E0E0E0936900EDBBE093A8
:1003FA006800E093C000E8E9E093C100E6E0E0931A
:10040A00C200E0E0E093C500EDE4E093C400E0E060
:10041A00E093C900E0E8E0BFE0E0E0937F00E0930A
:10042A007E00E0937C00E7EAE0937A00E0E0E09364
:10043A007B00ECBDA4E6B0E00E945061E0E01A99AE
:10044A00E1E0E0931A057894299AA4E60E9484636D
:10045A000E948963A1E00E947F61A0915F05A03894
:10046A0061F40E949863E0E0E0936105E0E4E093C0
:10047A0062050E949E630E94A5630E94AE63A0E08B
:10048A000E947F61A0E03799A1E00E94C063A0E0CA
:10049A003699A1E00E94C563A0915F05EFEF0E9423
:1004AA00727DE02909F465C10E949863E1E0E09356
:1004BA006105E2E3E0936205E0E5E0936305EEE1BE
:1004CA00E0936405E3E2E0936505E2E3E093660501
:1004DA00E4E60E94CA63E2E3E09369050E94D063FE
:1004EA00E3E0E0936C05E8EEE0936D05E2E3E09368
:1004FA006E05E8ECE0936F05E2E3E0937005EAE04D
:10050A00E0937105E0937205E0937305E1E0E093EF
:10051A007405E2E20E94D663EAE00E94DC63E6E93F
:10052A00E0937A05E9E0E0937B05E4ECE0937C054F
:10053A00E3E0E0937D05E4E80E94E463E6E9E09302
:10054A008005E2E0E0938105EEE70E94EA63E2E4D7
:10055A000E94F063E4EBE0938705EAE0E093880504
:10056A00E1E0E0938905E2E00E94F8630E940064FA
:10057A00E1E0E0939305E0E0E0939405E1E00E9476
:10058A000E64E4E20E941C64E4E0E0939E05E1E06C
:10059A000E9424640E942D64E0935F05E6E4E093E0
:1005AA006005E4EA0E943864E2E30E944264EFEFE5
:1005BA00E0936705E0936805EFE00E9448640E94B3
:1005CA004C64E3E8E0936E05E7E4E0936F05E0E549
:1005DA000E945264E4E60E945C64E0E00E94DC63EC
:1005EA00E0E0E0937A05E3E0E0937B05E8EEE09350
:1005FA007C05E0E0E0937D050E94E463E0E0E0939F
:10060A008005E09381050E94EA63E0E00E94F063BE
:10061A000E946064EEE1E0938D05E0E0E0938E05D0
:10062A00E0938F05E0939005E0939105E09392059E
:10063A00E0939305E6E9E0939405E0E0E0939505FD
:10064A00E6E9E0939605E0E0E0939705E0939805E4
:10065A00E4E6E0939905ECEFE0939A050E9468645A
:10066A00ECE30E946F640E948463E0935F05E0E814
:10067A00E0936005E0E0E0936105E1E0E093620564
:10068A00EFE9E0936305E1E0E09364050E944264C8
:10069A00E0E00E94CA63E0E00E9448640E944C6461
:1006AA00E2E3E0936E05E0936F05E0E00E94526496
:1006BA00E0E00E945C64E1E0E0937705E2E0E09329
:1006CA007805E0E0E0937905E0937A05E0937B050D
:1006DA00EAE0E0937C05E0937D05E0E00E94E463B4
:1006EA00E0E0E0938005EAE0E0938105E0E00E9423
:1006FA00EA63E0E00E94F0630E9460640E94006482
:10070A00E0E0E0939305E09394050E940E64E0E034
:10071A000E941C64E0E0E0939E050E942464E3E4E6
:10072A000E946F640E947964E0935F05E0E0E093C1
:10073A006005E1E0E0936105E0936205E0936305FB
:10074A00E4E1E0936405E0936505E0936605E093D0
:10075A006705E8E0E0936805E0936905E2E0E09365
:10076A006A050E946864ECE00E946F64B0E00E942F
:10077A00287B369950C0E0E0E0935F05EAE50E94E5
:10078A007E64E0E00E944264E0E00E94CA63E3E023
:10079A00E0936905E8EE0E94D0630E944C640E94CF
:1007AA0082640E945264E0E00E945C640E94686471
:1007BA00E8E10E946F640E948463E0935F05E2EAC5
:1007CA000E947E64E0E00E944264E0E00E94CA6304
:1007DA00E0E00E9448640E944C640E948264E093B4
:1007EA007005E0E0E09371050E946864E3E10E940D
:1007FA006F640E948463E0935F05E9EB0E947E6464
:10080A00E0E00E9442640E946864E8E00E946F642B
:10081A00B0E00E94287B189905C0689425F8E1E0A9
:10082A00E0935B05689427F846E20E948864E8EC46
:10083A00F0E00E948F64E0EDF7E00E949464E8EC37
:10084A00F0E0E0938208F09383080E94AE63AFE37E
:10085A000E949964EEA7E0916005EC83E09161053E
:10086A00ECA7E0916205EAA7E0916305E0936607C9
:10087A00E0916405E0936707E0916505E0936807F6
:10088A00E0916605E9A7E0916705E8A7E0916805A8
:10089A00EBA3E0916905EF8FE0916A05F0E00E9411
:1008AA009E64F0919107E0E00E949E64E0916B05DE
:1008BA00F0E00E94A364EA0FFB1F0E949E64E0918D
:1008CA006C05F0E00E94A864E0916D05F0E00E94DA
:1008DA00AD64E0916E05F0E00E94B264E0916F05AC
:1008EA00E0936B07E0917005E0936C07E091710566
:1008FA00E0936D07E0917205F0E00E94B764F09111
:10090A00F907E0E00E94B764E0917305F0E00E9405
:10091A00BC64EA0FFB1F0E94B764E0917405E09380
:10092A002105E0917505E0932305E0917605E093B2
:10093A002205A5E0B8E0E0917705F0E0ED93FC939D
:10094A00F0910508E0E0E0930508F0930608A0910D
:10095A000508B0910608E0917805F0E0EA0FFB1F60
:10096A00E0930508F0930608E0917905F0E00E940B
:10097A00C164F091F507E0E00E94C164E0917A0554
:10098A00F0E00E94C664EA0FFB1F0E94C164E09176
:10099A007B05F0E00E94CB64F0910108E0E00E9440
:1009AA00CB64E0917C05F0E00E94D064EA0FFB1F63
:1009BA000E94CB64A7E0B8E0E0917D05F0E0ED93FA
:1009CA00FC93F0910708E0E0E0930708F093080829
:1009DA00A0910708B0910808E0917E05F0E0EA0FBF
:1009EA00FB1FE0930708F0930808E0917F05F0E009
:1009FA000E94D564F0919507E0E00E94D564E091E9
:100A0A008005F0E00E94DA64EA0FFB1F0E94D564B9
:100A1A00E0918105FF27662777270E94DF640E94FD
:100A2A00E864E8E00E942A7D0E94DF64E091820582
:100A3A00F0E00E94E8640E94F1640E94DF64E091A1
:100A4A008305E0935905E0918405F0E00E94F6647D
:100A5A00F091A107E0E00E94F664E0918505F0E0DC
:100A6A000E94FB64EA0FFB1F0E94F664E091860570
:100A7A00E0930705E0918705E0930905E091880571
:100A8A00E0930A05E0918905E0930B05E0918A0558
:100A9A00E0930C05E0918B05E0930D05E0918C0540
:100AAA00E0937307E0918D05E0937407E0918E055A
:100ABA00EB8FE0918F05EA8FE0919005EF8BE09143
:100ACA009105EE8BE0919205ED8BE0919305EC8B0D
:100ADA00E0919405EB8BE0919505EA8BE091960500
:100AEA00F0E00E940065F091A907E0E00E9400652D
:100AFA00E0919705F0E00E940565EA0FFB1F0E944E
:100B0A000065E0919805F0E00E940A65F091B70748
:100B1A00E0E00E940A65E0919905F0E00E940F6505
:100B2A00EA0FFB1F0E940A65E0919A05E0932107EC
:100B3A00E0919B05E0931505E0919C05EC87E09117
:100B4A009D05F0E00E941465F091FD07E0E00E9427
:100B5A001465E0E0E0935D05E6E40E941965AAE306
:100B6A000E949964F0E00E942865EA0FFB1F0E9428
:100B7A001465E0916005E0934005E0916105E0931A
:100B8A004205E0916205E0934705E0916305EEA313
:100B9A00E0916405EAA3E0916505ECA3E09166059E
:100BAA00EDA3E0916705E0931905E0916805FF2739
:100BBA00662777270E942D650E9436650E943F6549
:100BCA00E09169050E9443650E944665E0916A05C5
:100BDA000E9443650E944665E0916B050E94436549
:100BEA000E942D65E0916C05E0935405E0916D0536
:100BFA00E0935505E0916E05E0935605E0916F0587
:100C0A00E0935805E0917005E0933405E091710591
:100C1A00E0933805E0917205E0933905E091730598
:100C2A00F0E00E944965F091AB07E0E00E94496557
:100C3A00E0917405F0E00E944E65EA0FFB1F0E94E6
:100C4A004965A0912107A23098F0E0917505F0E07E
:100C5A000E945365F0918907E0E00E945365E09194
:100C6A007605F0E00E945865EA0FFB1F0E94536563
:100C7A00F698F198A09121070E945D65A09121073D
:100C8A00E3E00E94727DE02921F0D0907705C090C0
:100C9A007805E0917905E0937A09E0917A05E09385
:100CAA007B09E0917B05F0E00E946265F0917D0985
:100CBA00E0E00E946265E0917C05F0E00E946765D1
:100CCA00EA0FFB1F0E946265E0917D05F0E00E9439
:100CDA006C65F0917F09E0E00E946C65E0917E0509
:100CEA00F0E00E947165EA0FFB1F0E946C65E091BB
:100CFA007F05F0E00E947665F091CE08E0E00E9460
:100D0A007665E0918005F0E00E947B65EA0FFB1FA3
:100D1A000E947665E0918105F0E00E948065F0917D
:100D2A008109E0E00E948065E0918205F0E00E947E
:100D3A008565EA0FFB1F0E948065E0918305F0E05C
:100D4A000E948A65F0918309E0E00E948A65E09139
:100D5A008405F0E00E948F65EA0FFB1F0E948A65F6
:100D6A00E0918505F0E00E949465F0918509E0E044
:100D7A000E949465E0918605F0E00E949965EA0F69
:100D8A00FB1F0E949465E0918705F0E00E949E6532
:100D9A00F0918709E0E00E949E65E0918805F0E005
:100DAA000E94A365EA0FFB1F0E949E65E0918905D8
:100DBA00E093F105E0918A05E093C305E0918B0584
:100DCA00E093F205E0918C05E093F305E0918D053F
:100DDA00E093F405E0918E05E093F706E0918F0524
:100DEA00E093F806E0919005E093FC06A9E0B8E0EC
:100DFA00E0919105F0E0ED93FC93F0910908E0E0B1
:100E0A00E0930908F0930A08A0910908B0910A082A
:100E1A00E0919205F0E0EA0FFB1FE0930908F093D6
:100E2A000A08ABE0B8E0E0919305F0E0ED93FC939B
:100E3A00F0910B08E0E0E0930B08F0930C08A09106
:100E4A000B08B0910C08E0919405F0E0EA0FFB1F43
:100E5A00E0930B08F0930C08E0919505E093FD06EA
:100E6A0050919605E0919705E0930107E091980566
:100E7A00F0E00E94A865E0E0E0935D05E0E80E94EA
:100E8A001965AFE30E949964E0933A05E091600521
:100E9A00F0E00E94AD65F091FF07E0E00E94AD65C9
:100EAA00E0916105F0E00E94B265EA0FFB1F0E9423
:100EBA00AD65E0916205E093CD05E03019F4E0916B
:100ECA00630502C0E091CD05E0932B07E09164052C
:100EDA00E0934305E0916505E0934805E0916605D6
:100EEA00E0934405E0916705E0934905E0916805C0
:100EFA00E98FE0916905E88FE0916A05E09375074B
:100F0A00E0916B05E0937607E0916C05ED83E09143
:100F1A006D05EE83E0916E05E0930707E0916F059A
:100F2A00E0930807E0917005E0930907E0917105E5
:100F3A00E0930C07E0917205E0933505E0917305A3
:100F4A00E0933605E0917405E0930D07E09175058D
:100F5A00E0930E05E0917605E0930F05E0917705A1
:100F6A00E0931005E0917805E0931105E091790589
:100F7A00E0931205E0917A05E0936907E0917B0519
:100F8A00E0936E07E0917C05E0934505E0917D05CD
:100F9A00E0934A05E0917F05EF83E0918005E093B5
:100FAA003705E0918105FF27662777270E94B765F5
:100FBA000E94C065E8E00E942A7D0E94B765E09120
:100FCA008205F0E00E94C0650E94F1640E94B76544
:100FDA000E94C065E8E00E942A7D0E94B765E09100
:100FEA008305F0E00E94C0650E94F1640E94B76523
:100FFA00E0918405F0E00E94C965F091D907E0E02C
:10100A000E94C965E0918505F0E0A091D907B091E9
:10101A00DA07EA0FFB1F0E94C965E0918605FF27E0
:10102A00662777270E94CE650E94D7650E94E065F1
:10103A00E09187050E94E4650E94E765E0918805D2
:10104A000E94E4650E94E765E09189050E94E465D3
:10105A000E94CE65E0918A05FF27662777270E94BE
:10106A00EA650E94F365E8E00E942A7D0E94EA652B
:10107A00E0918B05F0E00E94F3650E94F1640E9402
:10108A00EA650E94F365E8E00E942A7D0E94EA650B
:10109A00E0918C05F0E00E94F3650E94F1640E94E1
:1010AA00EA65E0918D05FF27662777270E94FC6590
:1010BA000E940566E8E00E942A7D0E94FC65E09194
:1010CA008E05F0E00E9405660E94F1640E94FC65AC
:1010DA000E940566E8E00E942A7D0E94FC65E09174
:1010EA008F05F0E00E9405660E94F1640E94FC658B
:1010FA00E0919005F0E00E940E66F091AD07E0E005
:10110A000E940E66E0919105F0E00E941366EA0FD4
:10111A00FB1F0E940E66E0919205FF27662777273C
:10112A000E9418660E942166E8E00E942A7D0E94B9
:10113A001866E0919305F0E00E9421660E94F1642E
:10114A000E9418660E942166E8E00E942A7D0E9499
:10115A001866E0919405F0E00E9421660E94F1640D
:10116A000E941866E0919505FF27662777270E9457
:10117A002A660E943366E8E00E942A7D0E942A6657
:10118A00E0919605F0E00E9433660E94F1640E94A5
:10119A002A660E943366E8E00E942A7D0E942A6637
:1011AA00E0919705F0E00E9433660E94F1640E9484
:1011BA002A66E0919805FF27662777270E943C66F2
:1011CA000E944566E8E00E942A7D0E943C66E09102
:1011DA009905F0E00E9445660E94F1640E943C660F
:1011EA000E944566E8E00E942A7D0E943C66E091E2
:1011FA009A05F0E00E9445660E94F1640E943C66EE
:10120A00E0919B05FF27662777270E944E660E947A
:10121A005766E8E00E942A7D0E944E66E0919C058E
:10122A00F0E00E9460660E944E660E945766E8E0FF
:10123A000E942A7D0E944E66E0919D05F0E00E9480
:10124A0060660E944E66E1E0E0935D05E0E00E9480
:10125A001965AAE00E949964E0937B07E091600512
:10126A00E0937C07E0916105E0937D07E0E0E0937D
:10127A007E07AFE0B8E0E0916205F0E0ED93FC9301
:10128A00A1E1B8E0E0916305F0E0ED93FC93A3E1FE
:10129A00B8E0E0916405F0E0ED93FC93A5E1B8E0D5
:1012AA00E0916505F0E0ED93FC93E0916605E0932B
:1012BA007F07E0916705E0938007E0916805E09376
:1012CA002A07A091F706A43618F0E0E0E093F706A3
:1012DA00A091F806A43618F0E0E0E093F806EC8155
:1012EA00E03009F071C0689432F8E1E0EEA7E9E174
:1012FA00EC83E3E2E0936607E2E3E0936707E4E660
:10130A00E0936807E5E0F8E00E946266E7E0F8E04B
:10131A000E946266E9E0F8E00E946266EBE0F8E0AB
:10132A000E946266EFE0F8E00E946766E1E1F8E099
:10133A000E946766E3E1F8E00E946766E5E1F8E08B
:10134A000E946766EFE0E0931905ECE2F1E00E9483
:10135A00B764E4EFF1E00E941465E4E6E093010764
:10136A00ECEFF0E00E94A865EEE7F2E00E94D56497
:10137A00EEE1EAA7E3E1E0933A05E4E6E8A7EEA3A3
:10138A00E4E0EC87E8EEF3E00E949E64E3E8E09391
:10139A005405E7E4E0935505E0E5E0935605E2E3FA
:1013AA00F0E00E94A864E8ECF0E00E94AD64E2E399
:1013BA00F0E00E94B264E4E2F0E00E940A65E8E02C
:1013CA00E0937F07E09380074A9912C00E946C66F7
:1013DA000E9475660E947C66E5E00E946F640E9426
:1013EA009466E5E00E946F640E947964E0935A056E
:1013FA00F498F398F298A0912B070E945D650E94D9
:10140A00B86609F0F29AA0912B07A23009F4F39A70
:10141A00A0912B07A33009F4F49AAC85A43019F0F3
:10142A000E94BF6602C00E94CD66E0932705AAE02B
:10143A000E947964E09330050E94D766E091F9062C
:10144A00F0E0AE0FBF1FE091FA06F0E0AE0FBF1F4B
:10145A000E94D97E14F4E1E001C0E0E0E093FB06CB
:10146A00E1E07E2E0E94E0662D98A0912207AE3020
:10147A00E0F3E0E0E09322072D9AA09132050E9462
:10148A005D65A09132050E94E66609F49FC5A091A8
:10149A003205A13019F4E0E0E0933205A091850706
:1014AA00B0918607E5E0F0E00E94B37D0E2EAC8D88
:1014BA00EEE00E948B7DE02119F0EC8DEF5F03C016
:1014CA0024FC02C0E0E0EC8FAC8DAE3011F46894DD
:1014DA0024F8A0912005A13029F4F69B02C0F698C1
:1014EA0001C0F69AF79B02C0F79801C0F79A0E94CA
:1014FA00EB66E0E0F0E064E374E40E94767CE0935B
:10150A003209F093330960933409709335090E94C4
:10151A00F4660E94D87B0E94FD660E9406670E94BC
:10152A000F670E94287C0E9414670E94D87B0E9441
:10153A001D670E94F4660E94266709F008F42BC012
:10154A00E0911209F091130960911409709115093B
:10155A000E942D670E94FD66E0918907F0918A0733
:10156A0031960E945365E0918B07F0918C07319672
:10157A00E0938B07F0938C070E9434670E943D67C3
:10158A000E942D65E0918D07F0918E073196E093C8
:10159A008D07F0938E070E9414670E94266709F050
:1015AA0008F411C0E0915E09F0915F096091600949
:1015BA00709161090E942D670E941D670E9442670F
:1015CA0031960E94C965E0918F07F091900739968C
:1015DA000E945865EA17FB07E8F4E0918907F09141
:1015EA008A07E0938F07F0939007E0E00E9447672D
:1015FA00E6E00E946F640E9484630E9462670E9410
:10160A00A563AAE00E9484630E9470670E94A56392
:10161A000E947A670E947E670E947A630E948367AB
:10162A000E948867E02161F10E948D67A0911609E6
:10163A00B091170980911809909119090E94767C36
:10164A00E0933E09F0933F09609340097093410982
:10165A000E949667ADE9B7E00E949F67A0913E0994
:10166A00B0913F0980914009909141090E94A46775
:10167A00E0932A09F0932B0960932C0970932D09A2
:10168A000E94AB67A0918D07B0918E07AE17BF0776
:10169A0008F07AC00E9406670E94B067A0912A09E2
:1016AA00B0912B0980912C0990912D090E94D17B30
:1016BA000E94B7670E94D87BE0931E09F0931F0926
:1016CA0060932009709321090E9496670E94B76768
:1016DA000E94767CA0E0B0E081E695E40E94287C36
:1016EA00A6E8B8E00E94C0670E940667E091220956
:1016FA00F091230960912409709125090E94D17BF8
:10170A000E94C5670E94CE67A5E6B8E086EB9AE319
:10171A000E94D17B0E94D7670E94CE67A0912209BE
:10172A00B091230980912409909125090E94767C21
:10173A00A8E8B8E00E94C0670E94E067E3E6F0E02C
:10174A000E94A77D0E2E0E94E067E0E0F0E00E9472
:10175A00A17DE029B9F0E3E6F0E0E0938808F09390
:10176A008908E0E0E0931609E0931709E093180965
:10177A00E0931909E0931A09E0931B09E0931C0905
:10178A00E0931D09689403C0E894F799689423F8D4
:10179A000E94E5670E94EE670E94F5670E94FE6755
:1017AA000E9409680E941D680E942668A09131095A
:1017BA00AA23DAF40E94E5670E94EE67A091420923
:1017CA00B091430980914409909145090E9431687A
:1017DA000E940968A0914A09B0914B0980914C096D
:1017EA0090914D090E943C6812C00E94E5670E94D0
:1017FA00EE670E9447680E94D87B0E9450680E9448
:10180A0009680E9459680E94D87B0E946268E1E0D8
:10181A00E0932D07A0912D07AF3008F0EBC00E948E
:10182A00F5670E94266709F008F417C00E946B68E2
:10183A000E942D67E0933609F093370960933809BF
:10184A00709339090E9421660E94DD7E34F40E9459
:10185A0074680E947D680E9418660E941D680E9432
:10186A00266709F008F417C00E9482680E942D6753
:10187A00E0933A09F0933B0960933C0970933D0960
:10188A000E9433660E94DD7E34F40E948B680E94B7
:10189A007D680E942A66A0913909AA238AF40E94C7
:1018AA006B680E9494680E94FE670E9421660E94EB
:1018BA00996834F40E9474680E943D670E94186611
:1018CA00A0913D09AA238AF40E9482680E94946822
:1018DA000E9426680E9433660E94996834F40E9426
:1018EA008B680E943D670E942A66A0914509AA2337
:1018FA00CAF4E0914209F091430960914409709158
:10190A0045090E9494680E9431680E944E65AF3F63
:10191A00EFEFBE0738F4E091AB07F091AC073196D0
:10192A000E944965A0914D09AA23CAF4E0914A0987
:10193A00F0914B0960914C0970914D090E9494688D
:10194A000E943C680E941366AF3FEFEFBE0738F46F
:10195A00E091AD07F091AE0731960E940E660E94A3
:10196A0047680E94266709F008F41DC0E0914609FD
:10197A00F091470960914809709149090E942D67C1
:10198A000E9450680E94F3650E94996864F4E0918D
:10199A00F208F091F3086091F4087091F5080E943A
:1019AA003D670E94EA650E9459680E94266709F00D
:1019BA0008F41DC0E0914E09F0914F096091500959
:1019CA00709151090E942D670E9462680E94056603
:1019DA000E94996864F4E091F608F091F708609122
:1019EA00F8087091F9080E943D670E94FC650E9400
:1019FA00A16810CF0E94E567E0E0F0E068EC72E4CD
:101A0A000E94A7680E94A4670E94AC680E94D87BC3
:101A1A00E0935209F093530960935409709355095E
:101A2A000E946C660E94B5680E94E97D0E94AC68BB
:101A3A000E949C7B0E94BB7C70F0E0E0E09352091C
:101A4A00E0935309E0935409E09355090E94BA6858
:101A5A0031960E9400650E94BF680E94E77C0E2EA4
:101A6A000E94E5670E940F670E94C5680E94A77DD1
:101A7A00E02151F1E091E208F091E3086091E40875
:101A8A007091E5080E94B5680E94147EDF01CB01BF
:101A9A000E94CF680E94C57E0E94767C0E94D86808
:101AAA000E94D17B0E94E1680E94D8680E94D87B7C
:101ABA00E0936209F093630960936409709365097E
:101ACA00A0E9B8E00E94C0670E943665A038E6E93E
:101ADA00BE07E8E98E07E0E09E0748F0E0E0E09301
:101AEA005708E0935808E0935908E0935A080E946F
:101AFA00E8680E2EE091F906A091F7060E94727D21
:101B0A000E22A091F806E091FA060E94727DE02169
:101B1A0069F0A0911E07A33030F4E0911E07EF5F31
:101B2A00E0931E0703C0E0E0E093FB06AE8DAC3302
:101B3A0019F4E2E0E093FB06A0913205A23009F025
:101B4A0045C2E1E02E26E0E0E09332050E94ED680E
:101B5A000E943D670E94B7650E94EB660E94DD7E87
:101B6A00A4F40E94F6680E94D7650E94C37E0E9470
:101B7A00D87BABE4B8E00E94657B0E94AF7E0E94EE
:101B8A00FB680E943D670E943C660E944566E0E150
:101B9A00FEE060E070E00E94317EE0936308F0931B
:101BAA00640860936508709366080E944566ECE3D2
:101BBA00F0E060E070E00E94317E7F936F93FF93C4
:101BCA00EF930E9404690E940D69AF91BF918F91B2
:101BDA009F910E94F77CA0935F08B093600880935E
:101BEA00610890936208E0915F08F0916008609143
:101BFA006108709162080E940D690E9445660E9400
:101C0A00C87E0E94F27C7F936F93FF93EF930E94AA
:101C1A000469A0E1BEE080E090E00E94E97DAF9116
:101C2A00BF918F919F910E94F77CA0935B08B0931C
:101C3A005C0880935D0890935E080E9414690E2EDA
:101C4A000E9457660E941B690E94D97DE02931F0E3
:101C5A00EFA5F8A90E9460660E944E66E0913F08CF
:101C6A00F09140086091410870914208A091D9070B
:101C7A00B091DA07882799270E94E37E21F10E9412
:101C8A00426766277727E0933F08F09340086093FE
:101C9A00410870934208E091AD07F091AE070E94A7
:101CAA0005660E9420690E941B690E94147EDF015A
:101CBA00CB010E944267662777270E94567EE093EF
:101CCA00D707F093D807AF8D0E9425690E94BF6895
:101CDA000E94B97D0E220E94E8680E942A690E9429
:101CEA002F6969F0EE8DEF5FEE8FEF8DF0E032969F
:101CFA00AE8DB0E0EA17FB0711F4ECE3EE8FA0918A
:101D0A002C07A33629F4E1E0EE8FE0E0E093FB062E
:101D1A00A394A0911405A13028F4E0911405EF5F73
:101D2A00E09314050E943969E8E5F2E00E94AD7D6E
:101D3A000E2E0E94FB640E9488670E22A091FB0669
:101D4A000E94C563A0911A050E943E6999F0E0912C
:101D5A00A307F091A4073196E093A307F093A40791
:101D6A000E9439690E944369EA1BFB0BE093A707AB
:101D7A00F093A807ECE3EA1509F0E6C0AA24D39485
:101D8A00E091E307E17091F00E944869EE7F0E94BA
:101D9A004D69E0E6E0936005E0917A090E94556991
:101DAA00E3E00E946F64B0E00E94287BE091E307C1
:101DBA00E27091F00E944869ED7F0E944D69E1E668
:101DCA00E0936005E0917B090E945569E3E00E9477
:101DDA006F64B0E00E94287BE091E307E470A1F011
:101DEA000E944869EB7F0E944D69EEE6E093600528
:101DFA00E0918809E0936105E09187090E9458699A
:101E0A000E94A5630E947A67E091E307E870A1F057
:101E1A000E944869E77F0E944D69E2E6E093600507
:101E2A00E0917E09E0936105E0917D090E9458697D
:101E3A000E94A5630E947A67E091E307E071A1F02E
:101E4A000E944869EF7E0E944D69E4E6E0936005CE
:101E5A00E0918009E0936105E0917F090E94586949
:101E6A000E94A5630E947A67E091E307E072A1F0FD
:101E7A000E944869EF7D0E944D69E8E6E09360059B
:101E8A00E0918209E0936105E09181090E94586915
:101E9A000E94A5630E947A67E091E307E074A1F0CB
:101EAA000E944869EF7B0E944D69EAE6E09360056B
:101EBA00E0918409E0936105E09183090E945869E1
:101ECA000E94A5630E947A67E091E307E078A1F097
:101EDA000E944869EF770E944D69ECE6E09360053D
:101EEA00E0918609E0936105E09185090E945869AD
:101EFA000E94A5630E947A67E091E407E170D9F035
:101F0A00E091E407EE7FE093E407E0E0E0935F0509
:101F1A00E6E6E0936005E091CE08F091CF080E94D2
:101F2A00587DE0936105E091CE080E9458690E94AD
:101F3A00A5630E947A67ECE3ED1531F4DD24C394BE
:101F4A00E4E1EC1509F4CC24ED89E03019F4E0E081
:101F5A00E0931605AD89A130C9F4E0911705EF5F4A
:101F6A00E0931705A0911705A23080F0E0911605BD
:101F7A00EF5FE0931605E0E0E0931705ED89A09185
:101F8A001605EA1718F4E0E0E0931605AD89A230C9
:101F9A0049F40E945B69E02911F0E0E001C0E1E048
:101FAA00E0931605AD89A33059F40E945B690E2AA5
:101FBA000E94696911F0E0E001C0E1E0E0931605D2
:101FCA00AD89A43019F4E1E0E0931605E8EC5E1659
:101FDA0048F45394EEE1E51529F40E946D69E0E0B6
:101FEA00E0936F07A091E9050E945D65A091E10564
:101FFA000E943E691E2EA091EA050E945D65A0918D
:10200A00E2050E943E691E2AA091EB050E945D65C9
:10201A00A091E3050E943E691E2AA091EC050E9448
:10202A005D65A091E4050E943E69E12929F0E091ED
:10203A002507EF5FE0932507A0912507AB3028F02D
:10204A00E0E0E09325070E946D690E9473690E948F
:10205A00537D3B97A4F10E9473690E94687DE093C7
:10206A005308F093540860935508709356080E94D9
:10207A0078690E947D690E94E97D0E949C7BAFE697
:10208A00B2E183E89AE30E94287C0E948869A3E56A
:10209A00B8E00E94657B0E94AF7E0E948F69A6E02D
:1020AA00B9E00E949869E0910805EF5FE09308059E
:1020BA000E949D6920F00091530810915408E0E0B5
:1020CA003699E1E07E2EE091FB06E03059F4E0E03B
:1020DA004A99E1E06E2E0E94A3698E2EE0E03799BC
:1020EA00E1E0BE2EA091FB060E945D650E94D766C4
:1020FA000E94AB69E02159F1E0E03699E1E0E09312
:10210A00C405E0E04A99E1E0E093C5050E94A369AD
:10211A00E093C605E0E03799E1E0E093C705A091B6
:10212A00C4050E94C063A091C5050E94B069A09130
:10213A00C6050E94B069A091C705E0E00E94727DC1
:10214A00E02929F0E0E0E0931E07E0931F07A09141
:10215A00FB06A23039F40E94E066E0E0E093F9065B
:10216A00E093FA06A091C4050E94C063A091C80535
:10217A000E94C563A9A10E943E6989F0E1E0E0934B
:10218A00C805E091F906E65FE093F906A091F90621
:10219A00A43628F0E091F906E456E093F906A091F6
:1021AA00C5050E94C063A091C9050E943E6979F0E5
:1021BA00E1E0E093C905E091F906EF5FE093F906E3
:1021CA00A091F906A43618F0E0E0E093F906A09190
:1021DA00C6050E94C063A091CA050E943E6989F0A3
:1021EA00E1E0E093CA05E091FA06E65FE093FA06B9
:1021FA00A091FA06A43628F0E091FA06E456E09394
:10220A00FA06A091C7050E94C063A091CB050E945F
:10221A003E6979F0E1E0E093CB05E091FA06EF5FE1
:10222A00E093FA06A091FA06A43618F0E0E0E093EB
:10223A00FA06A091C405A13019F4E0E0E093C805BC
:10224A00A091C505A13019F4E0E0E093C905A09179
:10225A00C605A13019F4E0E0E093CA05A091C705CC
:10226A00A13019F4E0E0E093CB050E94B5690E9421
:10227A00BA690E94C1690E94537D0E94C669A091F1
:10228A003805A23029F5EDE2F0E00E94CB690E9400
:10229A00D069A130E2E0BE074CF00E94D069E0E0CC
:1022AA00F2E0EA1BFB0BF595E79501C0EFEFE0932F
:1022BA0079070E94D069A030E2E0BE072CF40E94A0
:1022CA00B569F595E79501C0EFEFE0937A0704C089
:1022DA000E94B5690E94BA69E0911505E03009F0DB
:1022EA00CEC0EAE0E51509F048C00E94D5697497A6
:1022FA000E94DA69AE17BF0710F4E1E0E88B0E948A
:10230A00D5690E94DA690E94B37D0E2E0E94DF69A8
:10231A000E94DA690E94AD7DE02111F0E2E0E88BCB
:10232A000E94DF6974960E94E46910F4E3E0E88B86
:10233A000E94E86974970E94ED69AE17BF0710F40E
:10234A00E1E0EF870E94E8690E94ED690E94B37D8F
:10235A000E2E0E94F2690E94ED690E94AD7DE02175
:10236A0011F0E2E0EF870E94F26974960E94ED692B
:10237A00EA17FB0710F4E3E0EF870E94D569749728
:10238A000E94DA690E94F769A8890E943E6911F0E1
:10239A00E4E00CC00E94DF6974960E94DA690E9428
:1023AA00006AA8890E943E6911F0E5E0E88B0E9464
:1023BA00E86974970E94ED690E94F769AF850E94E7
:1023CA003E6911F0E4E00CC00E94F26974960E9422
:1023DA00ED690E94006AAF850E943E6911F0E5E04E
:1023EA00EF87A8890E942569A8890E94096AC1F015
:1023FA00EF85E03029F40E940E6A0E94C66902C085
:10240A000E94136AAC85A43028F4E8E2F0E00E9446
:10241A00CB6902C00E94196A5C3511F40E94136AE2
:10242A00A8890E941F6AA8890E94246A11F00E9442
:10243A00136AAF850E942569AF850E94096A69F00F
:10244A00E8E2F0E00E94CB69A8890E942569A88980
:10245A000E94096A11F00E94136AAF850E941F6ADE
:10246A00AF850E94246A51F0AC85A43028F4ECE3CD
:10247A00F0E00E94CB6902C00E94196A03C0E0E042
:10248A00E88BEF870E94D5690E94E46990F40E9464
:10249A00296A0E942E6A0E94336A0E94296A0E944F
:1024AA00DF69EA1BFB0BD0010E94197E0E94C669F4
:1024BA0002C00E94136A0E94DA69A93CE0E0BE07E2
:1024CA0024F0E8ECF0E00E94C669E0916808E09325
:1024DA0004070E94E8690E94ED69EA17FB0790F475
:1024EA000E943B6A0E940E6A0E94336A0E943B6AFB
:1024FA000E94F269EA1BFB0BD0010E94197E0E941E
:10250A00CB6902C00E94196A0E94ED69A93CE0E009
:10251A00BE0710F00E94406A0E94436AA081A1305F
:10252A0030F10E94496AAFE6B2E183E09AE30E9481
:10253A00A7680E94436A0E944F6A0E94287C7F9380
:10254A006F93FF93EF930E94436A0E944F6A0E941F
:10255A00566AAF91BF918F919F910E945D6A0E94C6
:10256A00626A0E94666A0E94287C0E946C6AE091F4
:10257A005905E030C1F5AC85A33098F5AFA5B8A9E7
:10258A000E94D97ECCF40E946F6AE0912E09F091E4
:10259A002F096091300970913109A0E0B0E080EA1A
:1025AA0090E40E94D87BE0932E09F0932F09609360
:1025BA0030097093310914C0A8A9AA2342F4EFA5DF
:1025CA00F8A93597AEE2B9E00E947A6A09C0E0E05C
:1025DA00E0932E09E0932F09E0933009E093310943
:1025EA0002C00E946F6AA0915905A130B9F50E94F4
:1025FA00816AAAEFB8E00E947A6AA091FA08B091BB
:10260A00FB088091FC089091FD08E0E0F0E060E8AA
:10261A0074E40E94767CA0E0B0E48CE995E40E9420
:10262A00287CDF01CB010E94866A0E948B6A0E9485
:10263A005D6ADF01CB01E8EBFEE165ED70E40E9423
:10264A00767CDE019F960E94C067A0911405A13096
:10265A0018F4E0E0EFA7E8AB0E946F6A0E949D6958
:10266A0030F0EFA5F8A9E0938C08F0938D08EE8975
:10267A00E03009F09EC0A0917208B0917308A23DA3
:10268A00E1E0BE07F4F40E94816A0E94906A7F9397
:10269A006F93FF93EF930E94816AED51F140DF013E
:1026AA000E94816AED51F1400E949D6AAF91BF91EB
:1026BA008F919F910E94A56AA2E9B8E00E94C06723
:1026CA0006C0E3E9F0E0E0939208F09393080E94D1
:1026DA00AA6AE23DA1E0FA072CF50E94B56A0E94B7
:1026EA00BA6AFF93EF930E94AA6A0E94906A7F9344
:1026FA006F93FF93EF930E94AA6AED51F1400F0185
:10270A000E94AA6AED51F140D0010E949D6AAF91E0
:10271A00BF918F919F910E94A56AAF91BF910E942C
:10272A00677B09C00E94B56ADF01AA0FBB1FAC56BE
:10273A00B74FE3E9F0E0ED93FC930E94C26AE23DF1
:10274A00A1E0FA072CF50E94B56A0E94CD6AFF93B0
:10275A00EF930E94C26A0E94906A7F936F93FF93DD
:10276A00EF930E94C26AED51F1400F010E94C26AC2
:10277A00ED51F140D0010E949D6AAF91BF918F91B6
:10278A009F910E94A56AAF91BF910E94677B09C081
:10279A000E94B56ADF01AA0FBB1FAA56B74FE3E929
:1027AA00F0E0ED93FC93EDEAFFEFE093D608F093A7
:1027BA00D708AE89A13041F5A0917208B09173088B
:1027CA0011960E94D56AE0939208F09393080E94AA
:1027DA00B56A0E94BA6ABF010E94AA6A0E94DA6AAE
:1027EA00DB01ED93FC930E94B56A0E94CD6ABF019A
:1027FA000E94C26A0E94DA6ADB01ED93FC93E0E070
:10280A00E093D608E093D7080E94B56A3396A2E906
:10281A00B8E0EE0FFF1FEA0FFB1FBF010E94DD6A3F
:10282A000E94A57E0E94DA6ADB01ED93FC930E9466
:10283A00E66AA0915405E3E80E94EC6A09F458C0DC
:10284A00A0919408B09195080E94F56A1CF4E1E001
:10285A00E0931007E0919408F09195080E94FC6AB1
:10286A000E94046B19F0E1E0E0931107A0919A0825
:10287A00B0919B080E94F56A1CF4E2E0E09310070D
:10288A00E0919A08F0919B080E94FC6A0E940B6BE7
:10289A0019F0E2E0E0931107A091A008B091A10815
:1028AA000E94F56A1CF4E3E0E0931007E091A008A7
:1028BA00F091A1080E94FC6A0E94126B19F0E3E0F1
:1028CA00E0931107A091A608B091A7080E94F56AA3
:1028DA001CF4E4E0E0931007E091A608F091A70841
:1028EA000E94FC6A0E94196B19F0E4E0E093110758
:1028FA00A0915505E7E40E94EC6A09F458C0A0913A
:10290A009608B09197080E94206B1CF4E5E0E093CA
:10291A001007E0919608F09197080E94FC6A0E94BD
:10292A00046B19F0E5E0E0931107A0919C08B091BF
:10293A009D080E94206B1CF4E6E0E0931007E091EA
:10294A009C08F0919D080E94FC6A0E940B6B19F08A
:10295A00E6E0E0931107A091A208B091A3080E94B3
:10296A00206B1CF4E7E0E0931007E091A208F091D5
:10297A00A3080E94FC6A0E94126B19F0E7E0E09338
:10298A001107A091A808B091A9080E94206B1CF415
:10299A00E8E0E0931007E091A808F091A9080E94E6
:1029AA00FC6A0E94196B19F0E8E0E0931107A09104
:1029BA005605E5E60E94EC6A09F464C0A0919808FD
:1029CA00B09199080E94276B1CF4E9E0E093100784
:1029DA00E0919808F0919908309719F4E9E0E093AA
:1029EA001107A0919E08B0919F080E94276B1CF4C2
:1029FA00EAE0E0931007E0919E08F0919F080E9498
:102A0A002E6B1E2EA09138050E945D65A091380597
:102A1A00E2E00E94727D0E2A0E94336BE029E121D6
:102A2A0019F0EAE0E0931107A091A408B091A50873
:102A3A000E94276B1CF4EBE0E0931007E091A408D6
:102A4A00F091A5080E942E6B0E943D6BE02119F0BF
:102A5A00EBE0E0931107A091AA08B091AB080E949D
:102A6A00276B1CF4ECE0E0931007E091AA08F091C0
:102A7A00AB080E942E6B0E943D6BE02119F0ECE03E
:102A8A00E0931107AC85A43011F00E94E66A0E9417
:102A9A009D6908F4B0C0E0919208F0919308E09320
:102AAA00AC08F093AD08EEEAF8E00E94456BE0EB63
:102ABA00F8E00E94456BE2EBF8E00E94456BA091BA
:102ACA009408B09195080E944A6B34F4E0919408F6
:102ADA00F09195080E94516BA0919A08B0919B08B9
:102AEA000E944A6B34F4E0919A08F0919B080E9484
:102AFA00516BA091A008B091A1080E944A6B34F4CE
:102B0A00E091A008F091A1080E94516BA091A6083B
:102B1A00B091A7080E944A6B34F4E091A608F0919C
:102B2A00A7080E94516BA0919608B09197080E943D
:102B3A00566B34F4E0919608F09197080E945D6B09
:102B4A00A0919C08B0919D080E94566B34F4E091C4
:102B5A009C08F0919D080E945D6BA091A208B0911B
:102B6A00A3080E94566B34F4E091A208F091A308DE
:102B7A000E945D6BA091A808B091A9080E94566BAB
:102B8A0034F4E091A808F091A9080E945D6BA09125
:102B9A009808B09199080E94626B34F4E091980801
:102BAA00F09199080E94696BA0919E08B0919F08C4
:102BBA000E94626B34F4E0919E08F0919F080E9493
:102BCA00696BA091A408B091A5080E94626B34F4C5
:102BDA00E091A408F091A5080E94696BA091AA0847
:102BEA00B091AB080E94626B34F4E091AA08F091AC
:102BFA00AB080E94696BE091F1050E946E6B0E941E
:102C0A00A97EA0E0B1E080E090E00E94E97DDF01CA
:102C1A00CB01E091F105F0E0E95DFA4FE081F0E0E7
:102C2A000E94F164A2E0B9E00E9498690E94766B62
:102C3A00E0E0F0E66AEE76E40E94BB7C09F008F474
:102C4A000AC00E947F6BA0E0B0E080E897E40E948F
:102C5A00D17B0E94886BAC85A43081F50E94766B8B
:102C6A00E0E0F0E060EA71E40E94A768EAA50E9449
:102C7A00916B0E94767CE0935A09F0935B0960930A
:102C8A005C0970935D090E94976BA2E0B9E00E940B
:102C9A009C6B0E94766B0E94A06B0E94287C0E940B
:102CAA00886B0E94766BE0E0F0E563EC77E40E94C3
:102CBA00767C0E94A56B0E94AE6B2DC00E947F6B32
:102CCA000E94D57E31F4E0E0F0E86BE375E40E94FF
:102CDA00886B0E94766BA030E0E8BE07EBE38E07B4
:102CEA00E5E49E0779F00E947F6BA6E6B6E686E6E3
:102CFA0090E40E94767CDF01CB010E94B96B0E94AE
:102D0A00AE6B09C0E0E0E093FE08E093FF08E093B1
:102D1A000009E09301090E949D6918F10E94F66872
:102D2A00A2EDB8E00E94C0670E94BB6B0E94AB692B
:102D3A000E2E0E94BB6BE0E0F0E00E94A17DE0292C
:102D4A0011F0E5E001C0E0E0E0930E07E0E0E09377
:102D5A000805E091E208F091E308E093D408F093C3
:102D6A00D5080E94DA69E8ECF0E00E94957D0E2E03
:102D7A00A091CE05E2E30E948B7DE021D1F0E091A3
:102D8A00CE05EF5FE093CE05A091CE05A23389F47C
:102D9A000E94A56B0E94C06BDF01CB010E948F6964
:102DAA000E949C7B0E94767CAAE3B5E00E94657B28
:102DBA00EC93A0913A050E94C063A091CE05E2E38C
:102DCA000E94727DE02119F0E0E0E093CE05A09127
:102DDA003A050E942569A091CE050E943E6919F024
:102DEA00E2E3E093CE05E09105070E94C46B0E94DE
:102DFA00E77C0E94CB6B0E94727D0E220E94D06BF0
:102E0A000E220E9475630E948867E021B9F0E09162
:102E1A000507E65FE09305070E94D56B31960E948D
:102E2A00DA6B0E94DF6BEA0FFB1FBF010E94E56BA2
:102E3A00DB01ED93FC93E2E3E093CF050E94EC6B98
:102E4A000E94F46B0E220E94F66B0E94FB6B71F1DA
:102E5A00E1E0F0E0E093D107F093D207EDEBF7E081
:102E6A000E94016CEFEBF7E00E94016CE1ECF7E0E5
:102E7A000E94016CE3ECF7E00E94016CE5ECF7E0DC
:102E8A000E94016CE7ECF7E00E94016CE9ECF7E0C4
:102E9A000E94016CEBECF7E00E94016CEDECF7E0AC
:102EAA000E94016CEFECF7E00E94016C0E947563CE
:102EBA000E947A630E94066C0E940F6C29F0E0E07F
:102ECA00E093D107E093D2070E94116C0E94D97E49
:102EDA0004F50E948B680E94B5680E94147EDF0187
:102EEA00CB010E94166C0E94687D0E94567EAEE05D
:102EFA00B9E00E949E7B0E94AF7EE0910E09F0919C
:102F0A000F096091100970911109DE01D1960E9492
:102F1A00C0670E941B6C0E947D690E94C97DEF9365
:102F2A000E94206CE250F040604070400E9421668E
:102F3A000E94D17DAF91EA230E2EA52DEEE10E94CB
:102F4A00727DE02191F00E94206C0E947C66E5E08F
:102F5A000E946F640E949466E5E00E946F640E947A
:102F6A008463E0938907E0938A07AB2D0E94C063CC
:102F7A00A0E0F3FCA1E00E94C5630E94226CE0215C
:102F8A0079F1E4E1EA876894F3F8AC85A43011F4A6
:102F9A000E946D69A0912B07A13021F4F298F39A4F
:102FAA00E2E01CC0A0912B07A23089F4F398F49AAE
:102FBA00A09168070E942569A0916707E0E00E9436
:102FCA00727DE02919F0E3E0E0932B0709C0A09194
:102FDA002B07A33029F4F498F29AE1E0E0932B0747
:102FEA00AB2D0E94C0630E94226C0E220E94066CC6
:102FFA000E94286CE02111F1A0910F07A03128F45A
:10300A00E0910F07EF5FE0930F07A0910F07AF3032
:10301A00A9F4AC85A43011F40E946D69E4E1EA8751
:10302A00A0912B07A43038F4E4E0E0932B07F29A3E
:10303A00F398F49803C0E1E0E0932B07E1E0EB1585
:10304A0019F4E0E0E0930F07E0916808E093310596
:10305A000E94306C0E94376C09F441C00E943B6C9C
:10306A00E081AAE6B9E00E94416C0E94496C0E9484
:10307A00B0670E94526C0E94526CE0936A09F09306
:10308A006B0960936C0970936D090E94566CE0811C
:10309A000E945C6C0E94616C0E94C6690E94676C07
:1030AA000E94666A0E945D6A0E94496C0E94287C9E
:1030BA00A0916609B09167098091680990916909A0
:1030CA000E94D87BE0936609F093670960936809C8
:1030DA00709369090E94676C0E946C6A09C0E0E0FB
:1030EA00E0936609E0936709E0936809E093690948
:1030FA000E94706C0E94766CE081A2E7B9E00E949F
:10310A00416C0E94706CA081A13048F00E947B6CD7
:10311A00EE0FFF1F0E94876C0E948B6A06C00E94F6
:10312A00876CE0E0F0E068E472E40E94767CE09369
:10313A007209F09373096093740970937509AC85E9
:10314A00E2E00E94907D0E2EA0912B070E94096A50
:10315A0009F4B3C00E94306C0E220E94906CECE21B
:10316A00F1E00E94AD7DE02151F0E0918909F091F2
:10317A008A093196E0938909F0938A0902C00E946C
:10318A00956CE0910407A0910307AE1710F4E09341
:10319A000307E0910407A0910207EA1710F4E093ED
:1031AA0002070E94F668A091DD07B091DE070E942F
:1031BA009B6C30F40E94F668ADEDB7E00E949F6701
:1031CA000E94F668A091DB07B091DC070E949B6C15
:1031DA0009F008F406C00E94F668ABEDB7E00E9459
:1031EA009F67A0910307BB27E0910207F0E0AE1B9F
:1031FA00BF0BBD01A0910107E2E0EA9FF001DB01EC
:10320A000E94A77D0E2EA0910107E4E60E94A26CFF
:10321A00A091DB07B091DC07E091DD07F091DE07B2
:10322A00EA1BFB0BDF010E94A76C0E94B37D0E2EE6
:10323A000E94AC6CEBEFF0E00E94AD7D0E220E9482
:10324A00EB66E0E0F0E060E87FE30E94DB7CE021EF
:10325A00E12991F00E94956CE0910407E09303073D
:10326A00E09302070E94F668ABEDB7E00E949F6701
:10327A00E093DD07F093DE070E94B16C0E94E17CC7
:10328A006E2FA09122050E94B46CA09122050E9483
:10329A00BD6CEF930E94B16C0E94E77C6E2FA091E7
:1032AA0021050E94B46CA09121050E94BD6CAF91CA
:1032BA00EA2B19F0E1E0E0937007A72D0E94C063A2
:1032CA000E94226C0E22A0E0F0FCA1E00E94C563DD
:1032DA00A09170070E94C26C09F443C0E0E0E09339
:1032EA0070076894F0F80E94956C0E94C76C0E945F
:1032FA00D57E01F50E94F668A8EDB8E00E94C06785
:10330A00E0E0E0936E09E0936F09E0937009E093BF
:10331A0071090E94DA690E94D97E14F4E4E1E8870F
:10332A000E942E6AA6E5B9E00E947A6A689421F89A
:10333A00E894F4F8A091DA08B091DB080E94AB692E
:10334A000E2E0E94BF680E94C5680E94957DE021EA
:10335A0041F0E091DA08F091DB08E093D808F093A5
:10336A00D908AB89A130D9F50E94F46B0E2EA09131
:10337A003105E2E30E948B7D0E94D06C0E94DA6CD8
:10338A000E94E16C0E22A0E0F4FCA1E00E94E96C2C
:10339A0031F00E94C76C0E94626A0E94EE6C0E9421
:1033AA00F76C0E94ED69E2E3F0E00E94AD7D0E94B5
:1033BA00D06C0E94FA6C0E94E77C0E94E16CE021CA
:1033CA0071F00E94C76C0E942D670E94EE6C0E94E9
:1033DA00FF6C0E94036D19F0E3E00E94096D0E94E0
:1033EA00106D0E2EA09129070E943E6909F44CC067
:1033FA000E94EB660E940F670E94A7680E94156DE3
:10340A0033960E941A6D0E94E77CEF930E941F6D0B
:10341A00E0E0F0E060EA70E40E94E77CAF91EA2322
:10342A00EF930E94F6680E948869DF01CB010E942F
:10343A00156D0E941A6D0E94E17CEF930E941F6D28
:10344A000E94DA6CAF91EA23AF91EA2BE9F0A091DE
:10345A000109AA234AF00E94F6680E94346D0E946C
:10346A003D6D0E94D87B08C00E94F6680E94346DA8
:10347A000E943D6D0E945D6AE0936E09F0936F09A8
:10348A0060937009709371090E94496D0E944F6D93
:10349A000E94D06C0E94566D19F0E0E0EC8F05C0D6
:1034AA00AC8DA23010F4E89424F80E945B6D0E945F
:1034BA00DD7E3CF40E94C76CA5E8B7E00E949F67D6
:1034CA0006C00E942E6AE0938507F09386070E9441
:1034DA002E6A309729F4E89421F86894F4F83BC0EE
:1034EA00A0E021FCA1E00E94C0630E94F46B0E22BE
:1034FA00AB890E943E691E2E0E945B6D0E94FA6C87
:10350A000E94E77C0E94646DA0913105E1E30E946C
:10351A00907D0E22AB890E94E96C1E2AA091D808E0
:10352A00B091D908E0E0F0E00E949B7D0E94646DB2
:10353A000E94106DE021E12971F00E94156DE0935F
:10354A00DA08F093DB080E946A6D0E94136AE89415
:10355A0022F8689421F84B9908C00E946A6DE89491
:10356A0022F8689421F8E1E001C0E0E0E093FE0669
:10357A00E09105050E94DA69F0E0EA17FB0724F4F6
:10358A00E0916808E09305050E94786DEF930E9428
:10359A00B16C0E94E77CAF91EA230E2EA09121051F
:1035AA000E94C5630E94036DEF930E94786DEF93AA
:1035BA000E94B16C0E94E17CAF91EA230E2EA09189
:1035CA0022050E94C5630E94036DAF91EA2B61F048
:1035DA00E0916808E09305050E94FF6C0E94696902
:1035EA0019F0E2E00E94096D0E945B6D0E94DD7E87
:1035FA000CF043C022FC03C0E1E0E093300568947C
:10360A0022F80E942E6A0E945B6D0E941A6D0E9427
:10361A00BB7C90F10E94C76C0E946C6AAB89A23095
:10362A0059F5A0916E09B0916F0980917009909136
:10363A007109E0E0F0E068E473E40E94BB7C09F001
:10364A0008F402C00E94806D0E94896D0E945B6D21
:10365A000E94D87B0E946C6AA0916908AA2362F42E
:10366A00E1E0F0E00E94C6690E945B6D0E94896DEC
:10367A000E94D17B0E94806D02C0E89422F80E94C9
:10368A00926D0E94976D0E22A0E026FCA1E00E9496
:10369A00C5630E94036D31F0689426F80E942E6A71
:1036AA000E948F640E94926D0E94976DE02161F1E1
:1036BA000E94A96D0E94B16DA0F0A0915308B0912B
:1036CA0054080E94B96DEA1BFB0BA3E0B0E00E940C
:1036DA00E17D0E94BE6DAE1BBF0BA093DC08B093C8
:1036EA00DD080E94A96D0E94DD7E28F40E94C36D48
:1036FA0032970E948F64A091DD08AA232AF4E0E0A1
:10370A00E093DC08E093DD080E94926D0E94E37E5C
:10371A0060F50E94C86D0E94B16D70F00E94BC6491
:10372A00E0915308F0915408EA1BFB0B0E94BE6D0E
:10373A00EA0FFB1F0E948F640E94C86DA230E0E06E
:10374A00BE07E0E08E07E0E09E0728F00E94C36D06
:10375A0031960E948F640E94BE6DAB3FE0E0BE07C7
:10376A0024F0EAEFF0E00E948F640E94C36D0E9489
:10377A00DA690E94A17D0E2E0E94036D11F0E89471
:10378A0026F80E94C36D0E94DA690E94A77D0E2E58
:10379A000E94036D21F00E94C36D0E94C6690E94B7
:1037AA007B6CAFA5B8A90E94B37D0E2EA0915C05D3
:1037BA000E94C5630E94036D39F0E1E0E0935C0565
:1037CA000E94D26D0E9494640E947B6CAFA5B8A936
:1037DA00EA17FB0748F50E947B6C0E94D86D139785
:1037EA0070F00E947B6C0E94D86DE4E0F0E00E94C9
:1037FA00DD6DAE1BBF0BA0938408B09385080E94B1
:10380A007B6C0E94D86D0E94D97E28F40E94E46DD8
:10381A0035970E949464A0918508AA232AF4E0E0CF
:10382A00E0938408E09385080E947B6CAFA5B8A951
:10383A00AE17BF0750F50E947B6C0E94E96D149782
:10384A0060F00E947B6C0E94E96DE5E0F0E00E9466
:10385A00DD6DEA0FFB1F0E9494640E947B6C0E943C
:10386A00E96D0E94D97E28F40E94E46D35960E9483
:10387A009464A0918408B0918508A53CE9E0BE074C
:10388A0024F0E4ECF9E00E9494640E94D26DDF0116
:10389A000E94E46D0E94A17D0E2E0E94036D19F014
:1038AA00E0E0E0935C050E94D26DDF010E94E46DC6
:1038BA000E94A77D0E2E0E94036D41F0A0918408FC
:1038CA00B09185080E94EF6D0E94C6690E94F46D4E
:1038DA000E94C46B0E94E77CEF930E94F46DF0E0B3
:1038EA000E94FC7C0E94EB660E941A6D0E94E17C99
:1038FA00AF91EA2B11F0689430F80E94FD6D0E9496
:10390A00E77C0E2E0E94496DE02911F0E89430F808
:10391A0030FE6AC0A0910109AA23A2F00E94F46DA8
:10392A00F0E00E94EB660E94A56A7F936F93FF9373
:10393A00EF930E94876C0E94C06BAF91BF918F91E9
:10394A009F911DC00E94CF680E94327B7F936F9324
:10395A00FF93EF930E94F46DF0E0AF91BF918F91C6
:10396A009F910E94A56A7F936F93FF93EF930E94A2
:10397A00876C0E94C06BAF91BF918F919F910E94FB
:10398A00287CA0917609B091770980917809909165
:10399A0079090E945D6AE0937609F093770960934A
:1039AA00780970937909A0917909AA234AF4E0E089
:1039BA00E0937609E0937709E0937809E09379092F
:1039CA000E94FD6D0E94BB7C09F008F402C00E94AF
:1039DA00076EE0917609F091770960917809709104
:1039EA0079090E946C6A02C00E94076EE8ECF8E04E
:1039FA000E940B6EEAECF8E00E940B6EECECF8E029
:103A0A000E940B6EAC85A43060F0E8ECF8E00E94EE
:103A1A00106EEAECF8E00E94106EECECF8E00E94FE
:103A2A00106E0E94156E0E941F6EA0915405E3E865
:103A3A000E948B7DE02191F00E94156E0E94256EF6
:103A4A00E093C808F093C908A091C808B091C908C2
:103A5A00549724F4E8ECF8E00E94016C0E942A6E64
:103A6A000E941F6EA0915505E7E40E948B7DE0211C
:103A7A0091F00E942A6E0E94256EE093CA08F09384
:103A8A00CB08A091CA08B091CB08549724F4EAEC69
:103A9A00F8E00E94016C0E94346E0E941F6EA09191
:103AAA005605E5E60E948B7DE02191F00E94346E76
:103ABA000E94256EE093CC08F093CD08A091CC0823
:103ACA00B091CD08549724F4ECECF8E00E94016C14
:103ADA00E091C808F091C9080E94E46934F4E091C1
:103AEA00C808F091C9080E94C669E091CA08F09115
:103AFA00CB080E94E46934F4E091CA08F091CB083B
:103B0A000E94C669E091CC08F091CD080E94E46950
:103B1A0034F4E091CC08F091CD080E94C669E09196
:103B2A0018050E94DA69F0E0EA17FB0724F4E0912D
:103B3A006808E0931805E0911805F0E035970E94AF
:103B4A00DA690E94A17D6E2F0E2EA0E026FCA1E06C
:103B5A000E94E96C1E2E062EA0915C050E94E96C5B
:103B6A001E2A062EA0E030FCA1E00E94E96CE129A1
:103B7A0061F0E0916808E09318050E94FF6C0E94CA
:103B8A00036D19F0E2E00E94096DA0912405A130AD
:103B9A0078F00E94136AA0912405A13021F4EAE08A
:103BAA00F0E00E94C669E0912405E150E093240503
:103BBA000E94F76CAB890E943E691E2E0E94ED6935
:103BCA00E2E3F0E00E94B37D0E2EAB89E1E00E94B1
:103BDA00727D0E94E16CE0211E2A0E94F76CAB897B
:103BEA000E943E6E0E9469691E2A0E94F76C0E941A
:103BFA00106DE021E129A9F0E0E0E09306050E94BA
:103C0A005B6D0E94DD7E1CF4E2E0E0932405E0E0B7
:103C1A00E0935609E0935709E0935809E09359094C
:103C2A0002C00E94196A0E942E6AE093FB07F09371
:103C3A00FC070E94F76CAA8D0E94E96C11F02C9A7D
:103C4A0001C02C980E94F76CA091FE060E94C26CDB
:103C5A0011F0E3E001C0E0E0E0934B05A72D0E94DC
:103C6A00C0630E94226CE02121F0E091EF07E0930B
:103C7A005705A0915705A130A8F0E09157050E9479
:103C8A00ED69F0E0EA17FB0728F0E0915705F0E04C
:103C9A000E94CB690E94DA690E94D97E1CF4E0E096
:103CAA00E0935705A0911F07AF3F28F4E0911F0743
:103CBA00EF5FE0931F07A72D0E94C0630E94436E27
:103CCA000E94496D0E944A6E0E94286C0E22A091A1
:103CDA00FB060E94C5630E94D7660E94AB69E02179
:103CEA001E2EA0911F07E8EC0E94526E0E94777D5B
:103CFA000E220E94496D0E944A6E0E94286C0E2272
:103D0A00A091FB060E943E6E0E94D7660E94AB6994
:103D1A00E021E12969F0AD8DAF3F18F4ED8DEF5F39
:103D2A00ED8FAD8DA43119F4E2E0E093FB0602C0F9
:103D3A00E0E0ED8FA92D0E94C0630E94556E0E949B
:103D4A005A6EE3E30E94907D0E220E94606E51F04B
:103D5A000E94676EABE1B8E00E946C6EE1E0F0E0B1
:103D6A00ED93FC93A92D0E94C0630E94556E0E9498
:103D7A005A6EE8E30E94727DE02131F00E94C16927
:103D8A00E093DE08F093DF08A0916E08B0916F0807
:103D9A0015960E9473690E94A17D0E2EA0911A05A4
:103DAA000E94E96C81F0E0919F07F091A00731979A
:103DBA00E0939F07F093A007309721F49924E0E05D
:103DCA00E09320071FC0EAE0F0E0E0939F07F0933A
:103DDA00A007A0911A05A13019F4E0E0E0931F07AB
:103DEA00A091FB06E0E00E94777D0E2EA0912007AD
:103DFA000E943E6939F0E1E0E0932007E093FB0678
:103E0A00E0E0ED8FA92DE0E00E94727D6E2F0E2E6C
:103E1A00A0E0F099A1E00E943E6E0E94E8680E229E
:103E2A00A52FEDE50E94777D0E942A690E94727D86
:103E3A000E94376C1E2E062EA0E0F099A1E00E9487
:103E4A003E6E0E94E8680E942A690E942F691E2A13
:103E5A000E9443690E9439690E94957D0E2E0E9434
:103E6A00E8680E220E94FB640E948867E021E1292B
:103E7A0009F40BC1F09B09C1F098E0E00E94626767
:103E8A000E94A563AAE00E948463E0935F05E7E3CA
:103E9A00E0936005E091AA07E0936105E091A90724
:103EAA000E9458690E94A563AAE00E9484630E9446
:103EBA004767E6E00E946F640E9484630E9470670D
:103ECA000E94A563AAE00E948463E0935F05EAE585
:103EDA00E0936005E091AC07E0936105E091AB07E0
:103EEA000E9458690E94A563AAE00E948463E09335
:103EFA005F05E4E8E0936005E0912B070E945569AD
:103F0A00E3E00E946F640E948463E0935F05E2EA43
:103F1A00E09360050E94ED680E945D7DE093610573
:103F2A000E94C065E8E00E94427DE0936205E0914C
:103F3A004308E0936305E091DA07E0936405E091B2
:103F4A00D907E09365050E94D765E8E10E94427DA2
:103F5A00E0936605E0914B08F0914C0860914D089A
:103F6A0070914E080E945D7DE09367050E94D765B7
:103F7A00E8E00E94427DE0936805E0914B08E093F7
:103F8A0069050E94F365E0E10E94367DE0936A05C7
:103F9A000E94F365E8E00E94367DE0936B05E091AC
:103FAA00F208E0936C050E940566E0E10E94367D06
:103FBA00E0936D050E940566E8E00E94367DE09375
:103FCA006E05E091F608E0936F05E091AE07E09385
:103FDA007005E091AD07E09371050E942166E0E16A
:103FEA000E94367DE09372050E942166E8E00E94F5
:103FFA00367DE0937305E091EA08E09374050E9428
:10400A003366E0E10E94367DE09375050E943366CF
:10401A00E8E00E94367DE0937605E091EE08E093B1
:10402A0077050E94FB680E945D7DE09378050E94F7
:10403A004566E8E00E94427DE0937905E0914708F1
:10404A00E0937A05E0914F08F09150086091510889
:10405A00709152080E945D7DE0937B050E9457662D
:10406A00E8E00E94427DE0937C05E0914F08E093EE
:10407A007D050E946864EFE10E94716EA4E6B0E0DB
:10408A000E94287BE2E3E0933C05A82D0E945D652F
:10409A000E94226CE02139F0E894F2F8E0E0E09323
:1040AA005B05E0932E05A82D0E94C063A0915B05D5
:1040BA000E94C5630E94226CE02171F0E0912E05F6
:1040CA00EF5FE0932E05A0912E05AA3029F4E0E0D7
:1040DA00E0932E05E0932005A82D0E94C063A091CD
:1040EA005B050E94C563A0E0F2FCA1E00E94C563E3
:1040FA000E94226CE021E1F1E4E1E9876894F2F898
:10410A00E0912005EF5FE09320050E94796EA0E020
:10411A00F0FCA1E00E943E6919F0E1E0E09320057D
:10412A00A09120050E941F6AA0E0F0FCA1E00E9475
:10413A003E6919F0E2E0E09320050E94796EAA8DAB
:10414A000E94C563AC85E3E00E94777DE02119F007
:10415A00E1E0E0932005A09120050E941F6AA0E0FB
:10416A00F0FCA1E00E94E96C19F0E3E0E09320057D
:10417A00E091FB06E03009F0C9C1E0E0E0934C05AC
:10418A00E0934D050E94806EE0930007E0912005C0
:10419A00E030B1F4F6980E94846E0E22AA8D0E9435
:1041AA00246A11F00E948063A09140050E9425694B
:1041BA000E948D6E11F00E94946EE0E0E98B5FC060
:1041CA00A0912005A130E9F4A0914005A33010F494
:1041DA000E94946EA0914005A33019F4EBA1E093DC
:1041EA004C050E94996EE02121F00E949C6EE0E04D
:1041FA00E8BDAA8DA53021F40E949C6EEFEFE8BDC0
:10420A003EC0A0912005A230F1F4F69AA091400593
:10421A00A33010F40E94946EA0914005A33019F4C3
:10422A00ECA1E0934C050E94996EE02121F00E94D6
:10423A009C6EE0E0E8BDAA8DA53021F40E949C6E38
:10424A00EFEFE8BD1CC0A0912005A330C1F4F69A97
:10425A00A0914005A33018F4E091F20501C0EFEFF8
:10426A00E0934C050E94996EE02119F0EFEFE7BD4B
:10427A00E8BDAA8DA53019F4EFEFE7BDE8BDE6E980
:10428A00E0934D05A0914B05E3E00E94727D0E2E4E
:10429A00A0914005E1E00E94907D0E220E948D6E61
:1042AA0019F0EFEFE0934C050E94A66E0E94AA6EE9
:1042BA0029F00E94946EE1E0E093FF060E94B16E3D
:1042CA000E94AA6E11F00E94B46E0E94A66E0E940D
:1042DA00BB6E29F00E94946EE0E0E093FF060E9414
:1042EA00B16E0E94BB6E11F00E94C26E0E94A66E51
:1042FA000E94C96E29F00E94946EE1E0E093FF06E5
:10430A000E94B16E0E94C96E11F00E94C26E0E9494
:10431A00A66E0E94D06E31F00E94946E0E94806E4A
:10432A00E0933D050E94B16E0E94D06E41F00E945A
:10433A00B46EA0913D05AA3010F40E94D76E0E9477
:10434A00A66E0E94E06E51F0A0912005A13010F0F7
:10435A000E94946E0E94806EE0933D050E94B16EA9
:10436A000E94E06E41F00E94B46EA0913D05AA3011
:10437A0010F40E94D76E0E94E76EEC91E0938A00D7
:10438A00E98DE03019F4E0E0E093B400A98DA130A2
:10439A0019F4EFEFE093B400E88DE03009F41598D2
:1043AA00A88DA13009F4159AA88D0E945D650E9416
:1043BA00EF6EE4E6F0E00E94A17DE02111F0EFEF5C
:1043CA00E7BD0E945B690E220E9469691E2E0E9447
:1043DA00496D0E944F6D0E22A72D0E94C5630E944F
:1043EA00436E0E94BF680E94E77C0E22AA8D0E943B
:1043FA003E691E2AA091FE060E945D650E94F46B2A
:10440A00E0211E2AA88D0E945D650E94EF6EECE2F3
:10441A00F1E00E94A17D0E220E94EF6EE4E6F0E038
:10442A000E94A77DE021E12909F445C0E091040535
:10443A00EF5FE0930405A091FE06A13011F40E94FB
:10444A00136AAB8DA13019F4EFEFE0938800AB8DBE
:10445A00A33041F4E0910405E270AFEFEA02F00103
:10446A00E0938800A0910405E5E00E94907D0E2E5D
:10447A000E94F46EC1F0AA8DA33011F40E94F96E65
:10448A00AA8DA43029F40E94F96E0E94016FE8BD3A
:10449A000E94016FE0938A00AB8DA23021F40E9442
:1044AA00016FE0938800A0910405A03118F0E0E0C4
:1044BA00E09304052AC0E4E0E0930405E0E0E09319
:1044CA008800A0E025FCA1E00E945D65A09120057E
:1044DA000E943E69D1F0E0912D05EF5FE0932D0532
:1044EA00A0912D05A13019F4EFEFE0938A00A09175
:1044FA002D05A33019F4E0E0E0938A00A0912D0580
:10450A00A43019F4E0E0E0932D0507C00E9480630F
:10451A00E0E0E0938800E0938A00A091FB06A230D5
:10452A0008F087C00E94086F3597EA17FB0708F45E
:10453A0042C0A0917C09A83230F4E0917C09EF5F77
:10454A00E0937C0930C0E091B300A8A50E94526EA6
:10455A000E948B7DE02171F0A091B300E8A50E9432
:10456A00116F0E94566A0E94626A0E94146FEA0FD3
:10457A00A02DEC93E091B300A8A50E948B7D0E9428
:10458A00CB6B0E948B7DE02171F0E091B300A8A56E
:10459A000E94116F0E94566A0E94626A0E94146FFA
:1045AA00EA1BA02DEC930E941F6F19F0E8A5E09377
:1045BA00B3006894F6F80E94086F3596EA17FB076D
:1045CA00B8F5E0E0E0937C09E091B300AEA10E9467
:1045DA00526E0E948B7DE02161F0A091B300EEA1A2
:1045EA000E94116F0E942B6F0E94146FEA0FA02D78
:1045FA00EC93E091B300AEA10E948B7D0E94CB6B3D
:10460A000E948B7DE02161F0E091B300AEA10E948F
:10461A00116F0E942B6F0E94146FEA1BA02DEC935E
:10462A000E941F6F19F0EEA1E093B300E894F6F828
:10463A0006C0E0E0E093B300E8E2E0937C09E1E041
:10464A00E61529F4E894F1F8E0E0E0935A05A62D7E
:10465A000E94C063A0915A050E94C563A0E0F1FCC4
:10466A00A1E00E94C5630E94226CE02149F168948E
:10467A00F1F8E0911305EF5FE0931305E0E0EE87B0
:10468A00AE85A53088F40E94326FA081A13018F05F
:10469A00E5E0EE8705C0E0911305EF5FE0931305AF
:1046AA00EE85EF5FEE87ECCFA0911305A53018F0E9
:1046BA00E0E0E09313050E94326FE081E0932C075B
:1046CA00A62D0E94C063A8A1EFEF0E948B7DE02176
:1046DA0021F0E8A1EF5FE8A309C0A8A1A13030F05A
:1046EA00E894F1F8E0E0E8A3E0933005A8A1A53149
:1046FA0019F4E1E0E0933005A8A1A43109F08FC2D2
:10470A00A52FE0E00E94867D0E94CB6B0E948B7DE4
:10471A00E02129F05150E091D405E0933E05A091A3
:10472A002C07A33620F4E3E6E0932C0778C2E1E0F5
:10473A00E0932C07E0E0E09313050E949863EEA54E
:10474A00E0936105EC81E0936205ECA5E0936305D3
:10475A00EAA5E0936405E0916607E0936505E091B8
:10476A006707E0936605E0916807E0936705E9A5A6
:10477A00E0936805E8A5E0936905EBA1E0936A0573
:10478A00EF8DE0936B05E0919207E0936C05E09161
:10479A009107E0936D05E0918107E0936E05E09142
:1047AA008307E0936F05E091F107E0937005E091CC
:1047BA006B07E0937105E0916C07E0937205E09155
:1047CA006D07E0937305E091FA07E0937405E091B1
:1047DA00F907E0937505E0912105E0937605E091EC
:1047EA002305E0937705E0912205E0937805E091AF
:1047FA000608E0937905E0910508E0937A05E091CF
:10480A00F607E0937B05E091F507E0937C05E091DC
:10481A000208E0937D05E0910108E0937E05E091AE
:10482A000808E0937F05E0910708E0938005E0918E
:10483A009607E0938105E0919507E09382050E942F
:10484A00E864E8E00E94427DE0938305E0912B084A
:10485A00E0938405E0915905E0938505E091A2076C
:10486A00E0938605E091A107E0938705E0910705AB
:10487A00E0938805E0910905E0938905E0910A052E
:10488A00E0938A05E0910B05E0938B05E0910C0516
:10489A00E0938C05E0910D05E0938D05E091730797
:1048AA00E0938E05E0917407E0938F05EB8DE0931A
:1048BA009005EA8DE0939105EF89E0939205EE89E0
:1048CA00E0939305ED89E0939405EC89E0939505CF
:1048DA00EB89E0939605EA89E0939705E091AA07A8
:1048EA00E0939805E091A907E0939905E091B8074C
:1048FA00E0939A05E091B707E0939B05E0912107C1
:10490A00E0939C05E0911505E0939D05EC85E09305
:10491A009E05E091FE070E9424640E942D64E093A4
:10492A005F05E6E4E0936005E091FD07E093610529
:10493A00E0914005E0936205E0914205E09363054A
:10494A00E0914705E0936405EEA1E0936505EAA1CD
:10495A00E0936605ECA1E0936705EDA1E093680595
:10496A00E0911905E09369050E943665E8E10E9425
:10497A00427DE0936A050E9434670E945D7DE09360
:10498A006B050E943665E8E00E94427DE0936C0563
:10499A00E0915708E0936D05E0915405E0936E05A8
:1049AA00E0915505E0936F05E0915605E093700597
:1049BA00E0915805E0937105E0913405E0937205A2
:1049CA00E0913805E0937305E0913905E0937405A9
:1049DA000E946864E6E10E946F640E948463E09327
:1049EA005F05E0E7E0936005E091F105E09361057A
:1049FA00E091C305E0936205E091F205E093630557
:104A0A00E091F305E0936405E091F405E093650510
:104A1A00E091F706E0936605E091F806E0936705F2
:104A2A00E091FC06E0936805E0910A08E0936905C5
:104A3A00E0910908E0936A05E0910C08E0936B05A0
:104A4A00E0910B08E0936C05E091FD06E0936D059B
:104A5A0050936E05E0910107E0936F05E091DF073F
:104A6A00E09370050E946864E2E10E946F640E940C
:104A7A008463E0935F05E0E8E0936005E0913A051E
:104A8A00E0936105E0910008E0936205E091FF0779
:104A9A00E0936305E091CD05E09364050E946864A4
:104AAA00E6E00E946F640E948463E0935F05E5E894
:104ABA00E0936005E0914305E0936105E0914805C4
:104ACA00E0936205E0914405E0936305E0914905AE
:104ADA00E0936405E98DE0936505E88DE09366054A
:104AEA00E0917507E0936705E0917607E093680522
:104AFA00ED81E0936905EE81E0936A05E09107078D
:104B0A00E0936B05E0910807E0936C05E0910907D3
:104B1A00E0936D05E0910C07E0936E05E091350591
:104B2A00E0936F05E0913605E0937005E0910D077B
:104B3A00E0937105E0910E05E0937205E0910F058F
:104B4A00E0937305E0911005E0937405E091110577
:104B5A00E0937505E0911205E0937605E091690707
:104B6A00E0937705E0916E07E0937805E0914505BB
:104B7A00E0937905E0914A05E0937A05EF81E093A5
:104B8A007C05E0913705E0937D050E946864EFE1BA
:104B9A000E946F640E947964E0935F05E0E0E0930D
:104BAA006005E0917B07E0936105E0917C07E09363
:104BBA006205E0917D07E0936305E0910F08E093B9
:104BCA006405E0911108E0936505E0911308E0930C
:104BDA006605E0911508E0936705E0917F07E09389
:104BEA006805E0918007E0936905E0912A07E09360
:104BFA006A050E946864ECE00E946F640E9479640E
:104C0A004E2EE0E0E0933B05A52FE8E30E94727D7B
:104C1A000E2E0E943D6F19F0E1E0E0933F05A62DAC
:104C2A000E94C063A0E0F1FCA1E00E94C563A52F29
:104C3A00E4E60E94817D0E942A690E94727DE02139
:104C4A0031F06894F1F85F5F543609F450E0E1E01E
:104C5A00E71511F4E894F0F8A72D0E94C063A0E0CC
:104C6A00F0FCA1E00E94C563A52FE0E00E947C7DD4
:104C7A000E942A690E94727DE02131F06894F0F85E
:104C8A0051505F3F09F453E6AB2D0E94C0630E9466
:104C9A00406FC1F00E94476FA9F4A0912B05A4317F
:104CAA0019F4E7E0E0932B05E0E0E0932C05E894A3
:104CBA00F3F8A0912B05A33028F0E0912B05E150E1
:104CCA00E0932B05A82D0E94C0630E94406FC1F09B
:104CDA000E94476FA9F4A0912B05A43119F4E7E0CB
:104CEA00E0932B05E0E0E0932C05E894F2F8A0911C
:104CFA002B05A33028F0E0912B05E150E0932B051A
:104D0A00A82D0E945D65AB2D0E94E96C31F0E0E0B0
:104D1A00E0932C05E4E1E0932B05AB2D0E945D6541
:104D2A00A0E0F3FCA1E00E94E96C29F0E894F3F812
:104D3A00E0E0E0933005AB2D0E94C063A0E0F3FCF5
:104D4A00A1E00E94C5630E94406F09F497C5E1E0A3
:104D5A00E09330056894F3F8503049F4A881A43000
:104D6A0030F4E881EF5FE883E0E0E093300551300A
:104D7A0049F4AEA5A13030F4EEA5EF5FEEA7E0E06E
:104D8A00E0933005523041F40E94526FAF3520F45F
:104D9A000E94F46D0E945B6F533049F40E94616F68
:104DAA00A83C28F40E94686FEB5F0E946F6F543032
:104DBA0041F40E94746FAF3020F40E947B6F0E940E
:104DCA005B6F553049F40E94566CA081A43620F4DA
:104DDA000E94826F0E945B6F563069F40E947B6C5E
:104DEA00E43FA1E0FA0738F40E94896FED91FD9142
:104DFA003A960E948F6F573061F4A0911905A83C2A
:104E0A0040F4E0911905EF5FE0931905E0E0E093C3
:104E1A003005583061F4A0913805A23040F4E09191
:104E2A003805EF5FE0933805E0E0E093300559304C
:104E3A0049F40E943B6CA081AA3020F40E94956F2D
:104E4A000E945B6F5A3049F40E94706CA081A330B3
:104E5A0020F40E949C6F0E945B6F5B3039F40E94C1
:104E6A00A36F20F40E94AB6F0E945B6F5C3099F4D1
:104E7A000E940F65A535E0E0BE0768F40E94B26F94
:104E8A0031960E94B76F0E94C56F0E94C76F0E9439
:104E9A00D16F0E94D66F5D3071F40E94A364A43C66
:104EAA00E9E0BE0740F40E94786931960E949E6448
:104EBA00E0E0E09330055E3079F40E94DD6F0E94F5
:104ECA00BC64AE17BF0740F40E94B96D31960E94C8
:104EDA00B764E0E0E09330055F30A9F40E94C56F43
:104EEA00A6E6B6E686E491E40E94287C0E9428653C
:104EFA000E949B6C40F40E94D16F31960E94146507
:104F0A00E0E0E0933005503171F40E943B6AAF3F14
:104F1A00E0E0BE0740F40E94E86931960E94B2645C
:104F2A00E0E0E0933005513179F40E94DF690E9494
:104F3A00296AAE17BF0740F40E94D56931960E94CC
:104F4A00A864E0E0E0933005523171F40E94E36F07
:104F5A00AF3FE0E0BE0740F40E94DF6931960E944D
:104F6A00AD64E0E0E0933005533149F40E94436AAE
:104F7A00A081AA3020F40E94E86F0E945B6F54312E
:104F8A0061F4A0915805A13040F4E0915805EF5F13
:104F9A00E0935805E0E0E0933005553161F4A091C3
:104FAA002205AA3040F4E0912205EF5FE093220542
:104FBA00E0E0E0933005563161F4A0912105AA3072
:104FCA0040F4E0912105EF5FE0932105E0E0E093F2
:104FDA003005573161F4A0912305A23340F4E091E2
:104FEA002305EF5FE0932305E0E0E09330055831B5
:104FFA0061F4A0910107A43640F4E0910107EB5F48
:10500A00E0930107E0E0E0933005593171F40E9422
:10501A00AC6CAC3FE0E0BE0740F40E94A76C32964D
:10502A000E94A865E0E0E09330055A3149F4A9A549
:10503A00A13030F4E9A5EF5FE9A7E0E0E09330059D
:10504A005B3149F4AB89A23030F4EB89EF5FEB8B2B
:10505A00E0E0E09330055C3149F4AC89A33030F4E8
:10506A00EC89EF5FEC8BE0E0E09330055D3179F499
:10507A000E947E67AE3DE3E0BE0748F40E94AB673C
:10508A003A960E94EF6F0E9405700E940E705E3180
:10509A0079F40E948367A835E2E0BE0748F40E94CB
:1050AA0029703A960E942E700E9405700E940E7016
:1050BA005F3161F4A0910705AA3040F4E091070539
:1050CA00EF5FE0930705E0E0E0933005503289F4A2
:1050DA000E944470A081AB3160F40E9444700E9427
:1050EA004A70E0910E07E03021F4E0910905E0935F
:1050FA000E05513289F40E944D70A081AA3160F4E4
:10510A000E944D700E944A70E0910E07E03021F42F
:10511A00E0910A05E0930F05523289F40E94537018
:10512A00A081AA3160F40E9453700E944A70E091F3
:10513A000E07E03021F4E0910B05E093100553329D
:10514A0089F40E945970A081AA3160F40E945970B2
:10515A000E944A70E0910E07E03021F4E0910C05BC
:10516A00E0931105543289F40E945F70A081AA313C
:10517A0060F40E945F700E944A70E0910E07E0306E
:10518A0021F4E0910D05E0931205553249F4AB8DF7
:10519A00A33030F4EB8DEF5FEB8FE0E0E093300566
:1051AA00563249F4AA8DA53030F4EA8DEF5FEA8FC2
:1051BA00E0E0E0933005573249F4A98DA13030F48C
:1051CA00E98DEF5FE98FE0E0E0933005583249F46A
:1051DA00A88DA13030F4E88DEF5FE88FE0E0E0932E
:1051EA003005593261F4A0914005A83040F4E091AD
:1051FA004005EF5FE0934005E0E0E09330055A3266
:10520A0061F4A0913905A83C40F4E0913905EB5FBF
:10521A00E0933905E0E0E09330055B3239F50E940E
:10522A00E864AE3DE3E0BE07E0E08E07E0E09E07FB
:10523A00E8F40E946C66E65FFF4F6F4F7F4F0E9453
:10524A00DF640E947468E851FC4F6F4F7F4F0E94E1
:10525A0018660E94DD6F0E943366662777270E94D0
:10526A00ED7C0E942A66E0E0E09330055C3261F44E
:10527A00AA890E9465700E94036D31F0EA89EF5F86
:10528A00EA8BE0E0E09330055D3291F40E943665E6
:10529A00AF37E6E9BE07E8E98E07E0E09E0740F48B
:1052AA000E943467EC59FF4F6F4F7F4F0E946A701C
:1052BA005E3271F40E940565A031E7E2BE0740F450
:1052CA000E94BA683A960E940065E0E0E0933005D1
:1052DA005F3261F4A0912107A43040F4E0912107E4
:1052EA00EF5FE0932107E0E0E0933005503361F48B
:1052FA00A0911505A13040F4E0911505EF5FE09308
:10530A001505E0E0E0933005513349F4AC85A4304B
:10531A0030F4EC85EF5FEC87E0E0E0933005523340
:10532A0049F4AF89A33030F4EF89EF5FEF8BE0E007
:10533A00E0933005533349F4AD89A43030F4ED8954
:10534A00EF5FED8BE0E0E0933005543361F4A09118
:10535A005405A33840F4E0915405EF5FE0935405F7
:10536A00E0E0E0933005553361F4A0915505A73488
:10537A0040F4E0915505EF5FE0935505E0E0E093D6
:10538A003005563361F4A0915605A53640F4E091F4
:10539A005605EF5FE0935605E0E0E093300557339A
:1053AA0089F4A0913E05E3E00E948B7D0E2E0E94B7
:1053BA003D6F41F0E0913E05EF5FE0933E05E0E08E
:1053CA00E0933005583369F4ACA5A63950F4ECA53E
:1053DA00EF5FECA70E94916B0E947D70E0E0E09382
:1053EA003005593379F40E94DA64A03BE4E0BE0741
:1053FA0048F40E94976B31960E94D5640E94B96B5B
:10540A000E948D705A3349F4AAA5AC3330F4EAA548
:10541A00EF5FEAA7E0E0E09330055B3361F4A09127
:10542A00F105A33040F4E091F105EF5FE093F10557
:10543A00E0E0E09330055C3361F4A0913A05AA3FBD
:10544A0040F4E0913A05EF5FE0933A05E0E0E0933B
:10545A0030055D33E9F4E0910005EF5FE093000564
:10546A00A0910005AC3318F0E0E0E09300050E943B
:10547A0098630E94A270E295E07F6E2F0E94A67048
:10548A00E60FE09361050E949E63E3E00E94716E5D
:10549A005E3361F4A091C305A13040F4E091C305E5
:1054AA00EF5FE093C305E0E0E09330055F3379F402
:1054BA000E94D16F0E94B265AE17BF0740F40E94E6
:1054CA001B6C31960E94AD65E0E0E09330055034E4
:1054DA0071F4E091F806EF5FE093F806E0E0E093FC
:1054EA003005A091F806A43610F0E093F80651347E
:1054FA0079F4A091FC060E9465700E94AE7041F09A
:10550A00E091FC06EF5FE093FC06E0E0E0933005F3
:10551A00523479F4A091FD060E9465700E94AE7023
:10552A0041F0E091FD06EF5FE093FD06E0E0E093D5
:10553A003005533449F4AE89A13030F4EE89EF5F77
:10554A00EE8BE0E0E0933005543471F40E94C664B7
:10555A00A83BEBE0BE0740F40E94866A31960E949F
:10556A00C164E0E0E0933005553461F4A091590537
:10557A00A13040F4E0915905EF5FE0935905E0E06E
:10558A00E0933005563471F40E94FB64A835E2E0DA
:10559A00BE0740F40E9443697E960E94F664E0E0EA
:1055AA00E0933005573449F4AF8DAC3330F4EF8DC6
:1055BA00EF5FEF8FE0E0E0933005583459F4A091A3
:1055CA000C07A13038F4E0910C07E0930C07E0E0F7
:1055DA00E0933005593461F4A0910D07A43040F4EA
:1055EA00E0910D07EF5FE0930D07E0E0E0933005EF
:1055FA005A3461F4A091CD05A43040F4E091CD0570
:10560A00EF5FE093CD05E0E0E09330055B3469F4A9
:10561A000E94706C0E94766CA081AA3030F40E94BD
:10562A00706C0E94766C0E944A705C3479F40E9415
:10563A00B0700E94A57EE336A0E0FA0738F40E9413
:10564A00B070ED91FD9131960E948F6F5D3461F4D7
:10565A00A0911B05A13040F4E0911B05EF5FE09398
:10566A001B05E0E0E09330055E3461F4A0917F070A
:10567A00AF3040F4E0917F07EF5FE0937F07E0E00F
:10568A00E09330055F3461F4A0918007AF3040F4B5
:10569A00E0918007EF5FE0938007E0E0E093300558
:1056AA00503561F4A0912A07A23040F4E0912A070C
:1056BA00EF5FE0932A07E0E0E09330055A35E1F422
:1056CA000E94F66BEAE0F0E00E94AD7D0E2E0E9489
:1056DA00F66BAA0FBB1FA354B84F0E94A57EDF0129
:1056EA000E948867E02141F00E94D56B31960E94A2
:1056FA00DA6BE0E0E09330055B3561F4A09167086E
:10570A00AF3744F4E0916708EF5FE0936708E0E0A1
:10571A00E09330055C3561F4A0910605AA3F40F498
:10572A00E0910605EB5FE0930605E0E0E0933005C3
:10573A005D3591F4A0916407A83340F4E0916407C1
:10574A00EF5FE0936407E0E0E09330050E94C169EF
:10575A00E093DE08F093DF085E3561F4A09152050C
:10576A00A13140F4E0915205EF5FE0935205E0E089
:10577A00E09330050E94B6700E94E96C61F0A09136
:10578A00F305AF3F40F4E091F305EF5FE093F305D3
:10579A00E0E0E09330050E94B6700E943E6961F035
:1057AA00A091F405AF3F40F4E091F405EF5FE09378
:1057BA00F405E0E0E0933005503671F40E94D064BD
:1057CA00A83EE3E0BE0740F40E94BF703A960E94EA
:1057DA00CB64E0E0E0933005513691F4A091F205F4
:1057EA00AA3F70F4AA3020F0E091F205E65F03C008
:1057FA00E091F205EF5FE093F205E0E0E093300517
:10580A005236B1F40E94E76EAC91AA3F31F40E947D
:10581A00E76EEC91EB5F0E946F6F0E94E76EAC91AE
:10582A00AA3F30F40E94E76EEC91E65F0E946F6F28
:10583A000E94C4700E94E96C71F0A8A5AA3F58F4AE
:10584A00AA3018F0E8A5E65F02C0E8A5EF5FE8A76E
:10585A00E0E0E09330050E94C4700E943E6971F056
:10586A00AEA1AA3F58F4AA3018F0EEA1E65F02C032
:10587A00EEA1EF5FEEA3E0E0E0933005A82D0E94D1
:10588A005D65A0E0F2FCA1E00E94E96C29F0E894D1
:10589A00F2F8E0E0E0933005A82D0E94C063A0E092
:1058AA00F2FCA1E00E94C5630E94406F09F4BBC5E7
:1058BA00E1E0E09330056894F2F8503049F4A881A9
:1058CA00A13030F0E881E150E883E0E0E093300570
:1058DA00513049F4AEA5A13030F0EEA5E150EEA763
:1058EA00E0E0E0933005523049F40E94526FA23052
:1058FA0028F00E94F46DE1500E946F6F533099F4C2
:10590A000E94616FA53020F00E94686FE55007C0C1
:10591A000E94616FA13038F00E94686FE150EC93E9
:10592A00E0E0E0933005543049F40E94746FA130EE
:10593A0028F00E947B6FE1500E946F6F553051F43E
:10594A000E94566CA081A13028F00E94826FE1501B
:10595A000E946F6F563059F40E947B6C3B9738F067
:10596A000E94896FED91FD913A970E948F6F57308F
:10597A0061F4A0911905A23040F0E0911905E150B7
:10598A00E0931905E0E0E0933005583061F4A09106
:10599A003805A13040F0E0913805E150E093380530
:1059AA00E0E0E0933005593051F40E943B6CA0814D
:1059BA00A23028F00E94956FE1500E946F6F5A3012
:1059CA0051F40E94706CA081A13028F00E949C6F53
:1059DA00E1500E946F6F5B3041F40E94A36F28F080
:1059EA000E94AB6FE1500E946F6F5C3089F40E9495
:1059FA000F65559768F00E94B26F31970E94B76F92
:105A0A000E94C56F0E94C76F0E94D16F0E94D66F15
:105A1A005D3071F40E94A364A538E3E0BE0740F04C
:105A2A000E94786931970E949E64E0E0E093300515
:105A3A005E30B9F40E94C56FA6E6B6E686EE90E43B
:105A4A000E94287C0E94BC640E949B6C09F008F4A6
:105A5A0008C00E94B96D31970E94B764E0E0E093F4
:105A6A0030055F3079F40E94DD6F0E942865EA17DD
:105A7A00FB0740F40E94D16F31970E941465E0E061
:105A8A00E0933005503169F40E943B6A0E94D97E46
:105A9A0040F40E94E86931970E94B264E0E0E09322
:105AAA003005513169F40E94296A0E94D97E40F476
:105ABA000E94D56931970E94A864E0E0E09330051E
:105ACA00523179F40E94D5690E94E36FEA17FB0705
:105ADA0040F40E94DF6931970E94AD64E0E0E093F0
:105AEA003005533151F40E94436AA081A13028F055
:105AFA000E94E86FE1500E946F6F543161F4A091E7
:105B0A005805A13040F0E0915805E150E09358055E
:105B1A00E0E0E0933005553161F4A0912205A1300F
:105B2A0040F0E0912205E150E0932205E0E0E093A5
:105B3A003005563161F4A0912105A13040F0E09181
:105B4A002105E150E0932105E0E0E093300557316B
:105B5A0061F4A0912305A23040F0E0912305E150C1
:105B6A00E0932305E0E0E0933005583161F4A09119
:105B7A000107A63040F0E0910107E550E0930107E4
:105B8A00E0E0E0933005593161F40E94AC6C139760
:105B9A0040F00E94A76C32970E94A865E0E0E0936B
:105BAA0030055A3149F4A9A5A13030F0E9A5E150F0
:105BBA00E9A7E0E0E09330055C3149F4AC89A13013
:105BCA0030F0EC89E150EC8BE0E0E09330055B319A
:105BDA0049F4AB89A13030F0EB89E150EB8BE0E07E
:105BEA00E09330055D3171F40E947E670E94D97E90
:105BFA0048F40E94AB6731970E94EF6F0E940570CC
:105C0A000E940E705E3171F40E9483670E94D97EF1
:105C1A0048F40E94297031970E942E700E940570E4
:105C2A000E940E705F3161F4A0910705A23040F026
:105C3A00E0910705E150E0930705E0E0E0933005C5
:105C4A00503289F40E944470A081A23060F00E9410
:105C5A0044700E94CD70E0910E07E03021F4E0918B
:105C6A000905E0930E05513289F40E944D70A08116
:105C7A00A13060F00E944D700E94CD70E0910E0735
:105C8A00E03021F4E0910A05E0930F05523289F4DD
:105C9A000E945370A081A13060F00E9453700E944C
:105CAA00CD70E0910E07E03021F4E0910B05E0930E
:105CBA001005533289F40E945970A081A13060F016
:105CCA000E9459700E94CD70E0910E07E03021F4D5
:105CDA00E0910C05E0931105543289F40E945F703B
:105CEA00A081A13060F00E945F700E94CD70E091A7
:105CFA000E07E03021F4E0910D05E09312055532CC
:105D0A0049F4AB8DA13030F0EB8DE150EB8FE0E040
:105D1A00E0933005563249F4AA8DA13030F0EA8D6D
:105D2A00E150EA8FE0E0E0933005573249F4A98D5B
:105D3A00A13030F0E98DE150E98FE0E0E0933005E1
:105D4A00583249F4A88DA13030F0E88DE150E88F3F
:105D5A00E0E0E0933005593261F4A0914005A130AA
:105D6A0040F0E0914005E150E0934005E0E0E09327
:105D7A0030055A32A1F4A0913905A53020F0E091FE
:105D8A003905E55007C0A0913905A13040F0E091EE
:105D9A003905E150E0933905E0E0E09330055B32E4
:105DAA0049F50E94E864AB30E0E0BE07E0E08E0708
:105DBA00E0E09E07F8F00E946C660E947D680E94EF
:105DCA00DF640E947468E456F040604070400E94AC
:105DDA0018660E94B26F0E9433660E942069A093DF
:105DEA00EE08B093EF088093F0089093F108E0E092
:105DFA00E09330055C3249F4AA89A13030F0EA898F
:105E0A00E150EA8BE0E0E09330055D3269F40E94EC
:105E1A0036650E94D17040F00E943467EA50F04023
:105E2A00604070400E946A705E3269F40E940565A3
:105E3A000E94D97E40F40E94BA6831970E94006598
:105E4A00E0E0E09330055F3261F4A0912107A130D0
:105E5A0040F0E0912107E150E0932107E0E0E09370
:105E6A003005503361F4A0911505A13040F0E0915E
:105E7A001505E150E0931505E0E0E0933005513354
:105E8A0049F4AC85A13030F0EC85E150EC87E0E0D4
:105E9A00E0933005523349F4AF89A13030F0EF89ED
:105EAA00E150EF8BE0E0E0933005533349F4AD89DC
:105EBA00A13030F0ED89E150ED8BE0E0E093300560
:105ECA00543361F4A0915405A53140F0E091540592
:105EDA00E150E0935405E0E0E0933005553361F476
:105EEA00A0915505A53140F0E0915505E150E093A8
:105EFA005505E0E0E0933005563361F4A09156056C
:105F0A00A53140F0E0915605E150E0935605E0E0F6
:105F1A00E0933005573379F4A0913E050E94256934
:105F2A000E943D6F41F0E0913E05E150E0933E054D
:105F3A00E0E0E0933005583369F4ACA5AD3350F096
:105F4A00ECA5E150ECA70E94916B0E947D70E0E005
:105F5A00E0933005593379F40E94DA64A73DE1E011
:105F6A00BE0748F00E94976B31970E94D5640E9441
:105F7A00B96B0E948D705A3349F4AAA5AB3030F040
:105F8A00EAA5E150EAA7E0E0E09330055B3361F46B
:105F9A00A091F105A13040F0E091F105E150E093C4
:105FAA00F105E0E0E09330055C3361F4A0913A0535
:105FBA00A13040F0E0913A05E150E0933A05E0E083
:105FCA00E09330055D3331F5E0910105EF5FE09331
:105FDA000105A0910105AD3018F0E1E0E09301055B
:105FEA00E2E0E0935F05A0910105B0E00E94EF6D49
:105FFA00E295E07F6E2F0E94D970E60FE09360056C
:10600A00E0916005E05CE09360050E949E63E2E037
:10601A000E94716E5E3361F4A091C305A13040F015
:10602A00E091C305E150E093C305E0E0E093300559
:10603A005F3379F40E94DD6F0E94B265EA17FB07AD
:10604A0040F40E941B6C31970E94AD65E0E0E0933A
:10605A003005503471F4E091F706EF5FE093F706EC
:10606A00E0E0E0933005A091F706A43610F0E09343
:10607A00F706513479F4A091FC060E9425690E9422
:10608A00AE7041F0E091FC06E150E093FC06E0E0DE
:10609A00E0933005523479F4A091FD060E942569F7
:1060AA000E94AE7041F0E091FD06E150E093FD06DA
:1060BA00E0E0E0933005533449F4AE89A13030F082
:1060CA00EE89E150EE8BE0E0E0933005543471F450
:1060DA000E94C664A13DE7E0BE0740F00E94866ABE
:1060EA0031970E94C164E0E0E0933005553461F4D1
:1060FA00A0915905A13040F0E0915905E150E09393
:10610A005905E0E0E0933005563469F40E94FB64D7
:10611A000E94D97E40F40E9443697E970E94F664E9
:10612A00E0E0E0933005573449F4AF8DA13030F008
:10613A00EF8DE150EF8FE0E0E0933005583461F4E1
:10614A00A0910C07A13040F0E0910C07E150E093D8
:10615A000C07E0E0E0933005593461F4A0910D0793
:10616A00A13040F0E0910D07E150E0930D07E0E027
:10617A00E09330055A3461F4A091CD05A13040F086
:10618A00E091CD05E150E093CD05E0E0E0933005E4
:10619A005B3469F40E94706C0E94766CA081A23014
:1061AA0030F00E94706C0E94766C0E94CD705C3454
:1061BA0069F40E94B0700E94A57E329738F00E945E
:1061CA00B070ED91FD9131970E948F6F5D3461F44B
:1061DA00A0911B05A13040F0E0911B05E150E0932E
:1061EA001B05E0E0E09330055E3461F4A0917F077F
:1061FA00A13040F0E0917F07E150E0937F07E0E0B3
:10620A00E09330055F3461F4A0918007A13040F03B
:10621A00E0918007E150E0938007E0E0E0933005E9
:10622A00503561F4A0912A07A13040F0E0912A0785
:10623A00E150E0932A07E0E0E09330055A35D9F4BB
:10624A000E94F66B0E94D97EB0F40E94D56B3197FA
:10625A000E94DA6BE0E0E09330050E94D56B30973C
:10626A0051F4E9E0E0930507E0E0E093D107E09319
:10627A00D207E093CF055B3569F4A0916708E1E89E
:10628A00EA1744F4E0916708E150E0936708E0E018
:10629A00E09330055C3561F4A0910605A13040F029
:1062AA00E0910605E550E0930605E0E0E09330054D
:1062BA005D3561F4A0916407A13040F0E091640774
:1062CA00E150E0936407E0E0E09330055E3561F465
:1062DA00A0915205A13040F0E0915205E150E093BF
:1062EA005205E0E0E09330050E94B6700E94E96C26
:1062FA0061F0A091F305A13040F0E091F305E1507F
:10630A00E093F305E0E0E09330050E94B6700E9446
:10631A003E6961F0A091F405A13040F0E091F405E6
:10632A00E150E093F405E0E0E0933005503661F483
:10633A000E94D064559740F00E94BF703A970E941D
:10634A00CB64E0E0E0933005513691F4A091F20578
:10635A00A13070F0AB3020F0E091F205EA5003C0B2
:10636A00E091F205E150E093F205E0E0E0933005B8
:10637A00523639F5E0912005F0E0BF01DE01929630
:10638A00AE0FBF1FAC910E942569FB01DE019296F8
:10639A00AE0FBF1FAC91EFEF0E948B7DE02131F071
:1063AA000E94E76EEC91EA500E946F6F0E94E76EBE
:1063BA00AC91AF3F31F40E94E76EEC91E5500E9438
:1063CA006F6F0E94C4700E94E96C71F0A8A5A13099
:1063DA0058F0AB3018F0E8A5EA5002C0E8A5E15041
:1063EA00E8A7E0E0E09330050E94C4700E943E698D
:1063FA0071F0AEA1A13058F0AB3018F0EEA1EA501E
:10640A0002C0EEA1E150EEA3E0E0E0933005A52F33
:10641A00ECE30E94727D0E2EA0913A050E943E691D
:10642A0011F0E1E04E2EA72D0E94C063A9A1EFEF63
:10643A000E948B7D0E942A690E948B7D0E22AD8D5F
:10644A000E943E6919F0E9A1EF5FE9A3A72D0E9416
:10645A005D650E94226C0E22AD8D0E943E6921F07C
:10646A00E894F0F8E0E0E9A3A9A1EEE10E94727DC8
:10647A000E94CB6B0E948B7D0E22A091FB06E2E06C
:10648A000E94727DE02121F0E1E0E093FB06EE8FAD
:10649A00EF8DE03011F4E0E0EE8F0E94BF680E94B9
:1064AA00E77C0E2E0E94E8680E22AE8D0E94BD6C1B
:1064BA0011F0E1E0EE8FAE8DAC3311F40E94406A28
:1064CA00A0910605A13028F0E0910605F0E00E94AF
:1064DA00C669AA890E945D650E94ED690E94886763
:1064EA00E02141F1EB85EF5FEB87F0E03196BF01E8
:1064FA000E94E170E617F70798F40E94D16F0E9494
:10650A007D690E94C17D0E2E0E94E770E4EAF1E0E7
:10651A0060E070E00E94B97DE02911F00E94196ADA
:10652A000E94E170AB85B0E0EA17FB0710F4E0E0E7
:10653A00EB8702C0E0E0EB870E94F76C0E94D16F04
:10654A000E947D690E94D97D0E220E942865E4EA94
:10655A00F1E00E949B7D0E22AC850E94096A51F0EF
:10656A000E94ED69A639E0E0BE0720F4E6E9F0E012
:10657A000E94CB69E8ECE51509F018C1E0917A09A7
:10658A000E94C46B0E94BB7C09F008F40CC00E94F4
:10659A004869E1600E94F0700E94CF68AAE7B9E0FA
:1065AA000E94657BEC93E0917B09ABA9BCA9F0E062
:1065BA000E94A77D0E2EE0917B09ADA9BEA90E947B
:1065CA00F570AFA9B8AD0E94F570A9ADBAADF0E00B
:1065DA000E94A77DE02989F10E944869E2600E9431
:1065EA00F070E0917B09ABA9BCA9F0E0EA17FB07C0
:1065FA001CF4EBA9E0937B09E0917B09ADA9BEA944
:10660A00F0E0EA17FB071CF4EDA9E0937B09E0919F
:10661A007B09AFA9B8ADF0E0EA17FB071CF4EFA9B4
:10662A00E0937B09E0917B09A9ADBAADF0E0EA17E6
:10663A00FB071CF4E9ADE0937B09E0918709F0912F
:10664A008809AFA5B8A90E94B37D0E2E0E941469CD
:10665A00E02149F00E944869E4600E94F070EFA5C9
:10666A00F8A90E949E65E0917D09F0917E09D80102
:10667A000E94AD7D0E2EE8ECF0E00E94A77DE0219D
:10668A0049F00E944869E8600E94F07000937D0911
:10669A0010937E09E0917F09F0918009E017F107D4
:1066AA0048F40E944869E0610E94F07000937F09F3
:1066BA00109380090E94FC70E0918109F09182098F
:1066CA000E9401710E220E940F6C59F00E944869C3
:1066DA00E0620E94F070E091AE08F091AF080E946B
:1066EA0080650E940471E0918309F09184090E94F7
:1066FA0001710E220E940F6C59F00E944869E064F1
:10670A000E94F070E091B008F091B1080E948A6589
:10671A000E940971E0918509F09186090E94017130
:10672A000E220E940F6C59F00E944869E0680E948C
:10673A00F070E091B208F091B3080E949465EFA559
:10674A00F8A90E94687D0E940E71F8010E941771D3
:10675A000E94687D0E94147E0E940E710E94177129
:10676A000E942071E093E208F093E3086093E40842
:10677A007093E508E091CE08F091CF08A091E20865
:10678A00B091E3088091E4089091E5080E94687D41
:10679A000E94E37E5CF4E091E407E160E093E407A1
:1067AA00E091E208F091E3080E947665A0912C0737
:1067BA00A33610F00C941240A0E026FCA1E00E943F
:1067CA005D65A0915C050E942571A0E030FCA1E006
:1067DA000E94C26C21F0E894F799689401C0E89489
:1067EA00F5F8E0912605E170EE0FAE2FE09126054F
:1067FA00E6950E942A71EA0F0E2EE0912605E6958B
:10680A00E695E170AE2FE0E0F5FCE1E0EA2BEE0F51
:10681A00EE0FE00DE0936207A8890E942569AF8513
:10682A000E942F7129F0E0916207EF5FE0936207FF
:10683A000E94326FE081E0932C07A09125050E9407
:10684A002569AC85E4E00E94727DE02949F4F79954
:10685A0007C0A0E0F699A1E0EA2FE295E07F19C00F
:10686A00A0E0F699A1E0EA2FE295E07F0E2EA0E0E3
:10687A00F299A1E0EA2FEE0FEE0F0E0EA0E0F399C7
:10688A00A1E0EA2FEE0FA02DAE0FE0E0F499E1E0CF
:10689A00EA0FE0936307A8A9AA231AF4E05AE0933F
:1068AA0063070E9434710E9448710E945071E894F3
:1068BA0031F8A091FE06A13011F46894F5F8EC893C
:1068CA00E03019F4E9E0E0936107AC89A13081F482
:1068DA00A0E022FCA1E0EA2FEE0FE75F0E2EA0E077
:1068EA0022FCA1E0EA2FEE0FEE0FE00DE093610724
:1068FA00AC89A23069F4E9E0E0936107A0E022FCE8
:10690A00A1E00E945871A0E022FCA1E00E945F7100
:10691A00AC89A33031F4E0E022FCE1E0E85FE093E7
:10692A006107E0E0F799E1E0E09302050E94C56F94
:10693A00AEEAB7E489E091E40E946A7109F008F4CA
:10694A0003C0E1E0E09302050E94C56FABE7B4E142
:10695A0082E191E40E946A7109F008F403C0E3E05D
:10696A00E09302050E94C56FADE3BAE08BE191E4C2
:10697A000E946A7109F008F403C0E7E0E093020597
:10698A000E94C56FAFE1B5E88FE191E40E946A7198
:10699A0009F008F403C0EFE0E09302050E94C56F16
:1069AA00A1EEBAE788E291E40E946A7109F008F45C
:1069BA0003C0EFE1E0930205A0912B07A43019F57B
:1069CA00A0E0F799A1E00E945871A0E0F799A1E030
:1069DA000E945F71A0E0F799A1E00E945D65A09115
:1069EA0030050E943E6911F0E1E00BC0A0E0F79982
:1069FA00A1E00E94C063A09130050E94E96C19F0E1
:106A0A00E0E0E0933005A0910305A431D0F50E949F
:106A1A00BB6BA83EE3E0BE0734F0E7EEF3E0E09399
:106A2A00D208F093D3080E94BB6BAD39EFEFBE07D3
:106A3A0034F4EDE9FFEFE093D208F093D308A09184
:106A4A00D308AA2372F00E94BB6BA436E0E0BE070B
:106A5A0024F00E947471E09331070E947F710E94B2
:106A6A008171A091D308AA235AF4EDE0E09331078B
:106A7A00E091D208F091D3080E9489710E94817135
:106A8A000AC0F79B04C0E0E4E093310702C00E9409
:106A9A008D71E0933207AA85A13098F0EA85E1501A
:106AAA00EA87EEE5E0933107A0912B07A43018F4AA
:106ABA00E0912B0704C0E0E5E0933107EAE0E093B8
:106ACA003207A985A13050F0E985E150E987E8E36A
:106ADA00E0933107E0912005E0933207A885A130C1
:106AEA0048F0E885E150E887E9E3E0933107E0E51B
:106AFA00E0933207E0911605E03009F03FC0E091DB
:106B0A006207E058E0936207EAE0E0932F07E0E0CB
:106B1A00E09330070E9491710E94D97E84F40E940A
:106B2A0091710E94EF6D0E9496710E949B711A9753
:106B3A0024F00E94A0710E94A2710E94AA71A091E1
:106B4A008D08AA23DAF40E94B2710E9489710E9408
:106B5A009671E0E4E0932F07E0918E08E093300706
:106B6A000E949B711A9744F00E94A0710E94A27120
:106B7A000E94AA71689401C0E89431F8A0911605A0
:106B8A00A13009F049C0E0916307E85FE093630729
:106B9A000E94B7710E94A57EFF238AF4E0E4E09385
:106BAA002F070E94B7710E94BC7114F4689401C047
:106BBA00E89431F80E94B7710E94C27106C0E89445
:106BCA0031F80E94B7710E94A57EE0938E08F09377
:106BDA008F080E949B711A9724F00E94A0710E944C
:106BEA00A2710E94AA710E94B7710E94A57EBF017C
:106BFA00DF01E3E6F0E00E94A77D0E2EDB01EDE95E
:106C0A00FFEF0E94A17DE02939F0E89431F8E0E431
:106C1A00E0932F07E0933007E0910D07E030F9F495
:106C2A00D8010E94C771E0933307D8010E94EF6D23
:106C3A000E94D171E0933407D8010E94D771E09382
:106C4A0035070639E0E01E0754F4E0E4E093330721
:106C5A00E0933407E0933507E0E0E0930205A09162
:106C6A000D07A13008F4D9C0A13079F50E94C56F8B
:106C7A00A2E5B8EB8AE391E40E94287C7F936F93A4
:106C8A00FF93EF930E94C56F0E94DC71AF91BF9191
:106C9A008F919F910E945D6A0E94E3710E94EC713C
:106CAA007F936F93FF93EF930E94C56F0E94DC71ED
:106CBA00D8010E946D7D0E94C57E0E945D6AAF91D7
:106CCA00BF918F919F910E94FB71A0910D07A230F5
:106CDA00E9F40E94BC640E94D16FEA1BFB0BAAE094
:106CEA00B9E00E949C6B0E94EC717F936F93FF93B3
:106CFA00EF930E94BC64F801EA1BFB0BAF91BF91B2
:106D0A008F919F910E948B6A0E94FB71A0910D073F
:106D1A00A33081F40E94206CAAE0B9E00E9498692D
:106D2A000E94EC71DF01CB010E9474680E949E7B75
:106D3A000E94FB71A0910D07A430B1F40E94B26FBA
:106D4A000E94E864662777270E94E97DAAE0B9E0F5
:106D5A000E9498690E94EC71DF01CB010E948B6846
:106D6A000E949E7B0E94FB71E0910A09F0910B0937
:106D7A0060910C0970910D090E94677B9F01EAE0FE
:106D8A00E09335072436E0E03E072CF023E630E0B6
:106D9A00E3E2E093350733232AF420E030E0ECE124
:106DAA00E0933507D9010E94EF6D0E94D171E093FB
:106DBA003307E0913307E03019F4EAE0E093330750
:106DCA00D9010E94D771E0933407E0E0F799E1E036
:106DDA00E09302050024021603061CF4E1E0E093A6
:106DEA0002052431E0E03E071CF0E3E0E0930205EF
:106DFA002832E0E03E071CF0E7E0E09302052C337E
:106E0A00E0E03E071CF0EFE0E09302052035E0E009
:106E1A003E071CF0EFE1E0930205A0916E08B091E5
:106E2A006F08E2E3F0E00E94A17D0E2EA0917008A7
:106E3A00B0917108E2E3F0E00E94A17D0E22A52D37
:106E4A00E6E40E948B7DE02119F0E0E0E0932C0754
:106E5A00E0912C07E03079F4EEE3E0933707E5E0C0
:106E6A00E0933807ECE70E94FE71E7E30E940472A0
:106E7A00EEE5E0933D07A0912C07A13009F063C02D
:106E8A00A8890E94C063AF850E94C5630E940A72E6
:106E9A000E940E720E9412720E94167229F00E94BB
:106EAA001A72EA2BE09362070E945865A83EE3E053
:106EBA00BE0790F0E0916107E05EE09361070E94EF
:106ECA0058650E942372E0933B070E942D72E0935B
:106EDA003C070E94397217C0E0916107E056E093BF
:106EEA0061070E945865A436E0E0BE0720F00E94C0
:106EFA002D72E0933B070E9439720E944172E0931F
:106F0A003C070E945865EAE0F0E00E945B7EE0934D
:106F1A003D07E9E0EC1518F4E2E0E0933607AC2D02
:106F2A00BB270E94D771E0933707AD2DB0E00E94CE
:106F3A00EF6D0E94D171E0933807AD2DBB270E94F7
:106F4A00D771E0933907A0912C07A23009F05EC0EF
:106F5A00E0916107E054E09361070E943665A0342E
:106F6A00E2E4BE07EFE08E07E0E09E0750F00E94E1
:106F7A003665E0E4F2E46FE070E00E944672E09366
:106F8A0037070E943665A03AE6E8BE07E1E08E07B9
:106F9A00E0E09E0750F00E943665E0EAF6E861E01C
:106FAA0070E00E944672E09338070E9436650E949C
:106FBA00517240F00E9436650E9459720E944672D0
:106FCA00E09339070E9436650E945E7240F00E9483
:106FDA0036650E9466720E944672E0933A070E94E2
:106FEA0036650E946B7240F00E9436650E941B69EA
:106FFA000E944672E0933B070E9473720E94467297
:10700A00E0933C070E9473720E947A72A0912C0747
:10701A00A33089F5E7E70E947F720E9421660E94E9
:10702A00517224F00E9421660E9485720E94216694
:10703A000E945E7224F00E9421660E9493720E944E
:10704A0021660E946B7244F00E9421660E942071A0
:10705A000E94A172E0933B070E9421660E94D170B0
:10706A0034F00E94AA720E94B172E0933C070E9417
:10707A00AA720E94B472A0912C070E941F6AA09162
:10708A002C07E9E00E94727DE02999F10E94B97209
:10709A00A93019F4E2E0E0933607EEE30E947F722A
:1070AA000E9433660E94517224F00E9433660E9445
:1070BA0085720E9433660E945E7224F00E943366D3
:1070CA000E9493720E9433660E946B7244F00E947F
:1070DA0033660E9420710E94A172E0933B070E94CE
:1070EA00C1720E94B172E0933C070E94C1720E9471
:1070FA00B472A0912C07E5E00E94727D0E2EEAE0A0
:10710A000E94727DE02909F457C00E94B972AA3020
:10711A0019F4E2E0E0933607EEE30E947F72E0E5BD
:10712A00E0933907A0919108AA231AF4E0E4E093C6
:10713A003B070E94116CAD39EFEFBE071CF4E0E487
:10714A00E0933A07A0919108AA23BAF00E94116C21
:10715A00A436E0E0BE0734F00E94116C0E94C771A9
:10716A00E0933B070E94116C0E94EF6D0E94D1715F
:10717A00E0933C070E94116C19C00E94C872E43661
:10718A00A0E0FA0744F00E94C8720E94616C0E9453
:10719A00D171E0933B070E94166C0E9489710E948C
:1071AA00D171E0933C070E94C872DF01EAE0F0E087
:1071BA000E945E7EE0933D07A0912C07A630C9F598
:1071CA000E94CC72E0E0E09337070E94D272A9A92C
:1071DA00BAA9A031E7E2BE0724F0EFE0F7E2E9AB93
:1071EA00FAABAAA9AA231AF4E0E0E9ABEAABA9A987
:1071FA00BAA9A83EE3E0BE0724F00E94D972E09340
:10720A003A07A9A9BAA9A436E0E0BE0724F00E9469
:10721A00C771E0933B07A9A9BAA90E94EF6D0E9422
:10722A00D171E0933C07A9A9BAA90E94D771E0934A
:10723A003D07A0912C07A73009F04DC00E94ED69C7
:10724A000E94D97E00F5ECE0E09337070E940E6AAF
:10725A00F695E795E436A0E0FA0730F00E94ED696A
:10726A000E94DE72E09338070E940E6AF695E7954F
:10727A003A9730F00E94ED690E94E472E093390770
:10728A000E940E6A21C0EBE0E09337070E94EA727F
:10729A00E436A0E0FA0740F0A091FB07B091FC07A2
:1072AA000E94DE72E09338070E94EA723A9740F031
:1072BA00A091FB07B091FC070E94E472E0933907A2
:1072CA00E091FB07F091FC07F695E795DF010E9434
:1072DA004172E0933A07A0912C07A83009F085C0C3
:1072EA00A8890E94C063AF850E94C5630E940A7282
:1072FA000E940E720E9412720E94167229F00E9457
:10730A001A72EA0FE0936207A0918608B091870883
:10731A00A135EBEFBE0734F4E1E5FBEFE093860815
:10732A00F0938708A0918608B0918708A03BE4E013
:10733A00BE0734F0EFEAF4E0E0938608F09387089A
:10734A00A0918708AA2352F4E0E4E0933A07E09177
:10735A008608F09187080E94FC7C04C0E0918608A8
:10736A00F0918708E0938A08F0938B08A0918A0825
:10737A00B0918B08ECE3F0E00E942C7EE093990731
:10738A00F0939A070E94F172ECE30E94097EA091A1
:10739A008A08B0918B08AE1BBF0BA0939B07B093D2
:1073AA009C0723FE1DC00E94F1721A9718F0E2E0B2
:1073BA00E09336070E94F1720E944172E093370708
:1073CA00A0919B07B0919C070E94F672E093380740
:1073DA00A0919B07B0919C070E944172E0933907E4
:1073EA000E94FC72E8E7E0933D07A0912C07AB30BE
:1073FA0061F5E0916107E054E0936107E9E30E94D7
:10740A0003730E940565A83EE3E0BE0730F00E94C0
:10741A0005650E942372E0933A070E940565A43627
:10742A00E0E0BE0730F00E9405650E940973E09310
:10743A003B070E9405650E94F672E0933C070E9492
:10744A0005650E944172E0933D07A0912C07AC307C
:10745A0009F08BC0E2E0E0933607EEE3E0933707EA
:10746A00A091D508AA239AF10E940F731A9744F0A3
:10747A000E940F730E94EF6D0E94D171E0933C0746
:10748A000E940F73A436E0E0BE0734F00E940F7327
:10749A000E94C771E0933B070E940F73A83EE3E086
:1074AA00BE0734F00E940F730E94D972E0933A0724
:1074BA000E940F73A031E7E2BE0734F00E940F73F7
:1074CA000E941473E09339070E940F7348C0EAE0E0
:1074DA00E0933C070E940F73A73FEFEFBE075CF4EF
:1074EA000E9419730E9489710E94D171E0933C072E
:1074FA00EDE0E0933B070E940F73AD39EFEFBE0753
:10750A005CF40E941E730E94616C0E94D171E09328
:10751A003B07EDE0E0933A070E940F73A931ECEFC5
:10752A00BE0754F40E941E73DF010E94D972E093D1
:10753A003A07EDE0E09339070E940F73A13FE8EDA7
:10754A00BE0754F40E941E73DF010E941473E09375
:10755A003907EDE0E09338070E941E73DF01EAE085
:10756A00F0E00E945E7EE0933D07A0912C07AD30CB
:10757A0071F50E942273E3E6E0933D07A091AF08FC
:10758A00AA233AF4E0E4E0933B07E091AE08E195E0
:10759A0004C00E94FC700E94D771E0933C070E94CD
:1075AA00FC70A436E0E0BE0734F00E94FC700E9432
:1075BA00C771E0933A070E94FC701A9744F00E9440
:1075CA00FC700E94EF6D0E94D171E0933B07A0917D
:1075DA002C07AE3089F50E942C73E8E7E09339074F
:1075EA00E3E6E0933D07A091B108AA233AF4E0E468
:1075FA00E0933B07E091B008E19504C00E94047152
:10760A000E94D771E0933C070E940471A436E0E01F
:10761A00BE0734F00E9404710E94C771E0933A07D2
:10762A000E9404711A9744F00E9404710E94EF6D3F
:10763A000E94D171E0933B07A0912C07AF3071F5FE
:10764A000E943373E3E6E0933D07A091B308AA23AF
:10765A003AF4E0E4E0933B07E091B208E19504C014
:10766A000E9409710E94D771E0933C070E94097138
:10767A00A436E0E0BE0734F00E9409710E94C77187
:10768A00E0933A070E9409711A9744F00E9409711F
:10769A000E94EF6D0E94D171E0933B07A0912C07E5
:1076AA00A03171F5A8890E94C063AF850E94C563A5
:1076BA000E940A720E940E720E9412720E94167230
:1076CA0029F00E941A72EA0FE0936207E0E00E9432
:1076DA0089630E943D73A0910105AA3018F0E2E087
:1076EA00E09336070E94D970E09337070E94A27090
:1076FA000E94D171E09338070E94A670E09339077F
:10770A00A0912C07A13109F042C00E94CC72E091ED
:10771A007408F09175080E9463737F936F93FF93C7
:10772A00EF93E0917408F09175080E946B73AF9122
:10773A00BF918F919F910E945D6AA7E1B8E00E9474
:10774A009F670E947573129728F4E0E0E093170888
:10775A00E09318080E947A73E1E0E09339070E94E7
:10776A007573A436E0E0BE0730F00E9475730E947C
:10777A000973E0933B070E9475730E94F672E093C7
:10778A003C070E9475730E944172E0933D07A091E5
:10779A002C07A23109F042C00E94CC72E09176080F
:1077AA00F09177080E9463737F936F93FF93EF932F
:1077BA00E0917608F09177080E946B73AF91BF91C0
:1077CA008F919F910E945D6AA9E1B8E00E949F672C
:1077DA000E948173129728F4E0E0E0931908E0937D
:1077EA001A080E947A73E2E0E09339070E948173D3
:1077FA00A436E0E0BE0730F00E9481730E9409734C
:10780A00E0933B070E9481730E94F672E0933C0763
:10781A000E9481730E944172E0933D07A0912C0758
:10782A00A33109F061C00E948673A0EDB8E00E94FE
:10783A00C067E0E50E948F73E4E5E0933907A09101
:10784A00D108AA2312F4EDE001C0EAE0E0933C0774
:10785A000E949573A73FEFEFBE0714F4EDE001C055
:10786A00EAE0E0933B070E949573AD39EFEFBE075C
:10787A0014F4EDE001C0EAE0E0933A07A091D108E0
:10788A00AA2342F40E9486730E94327BA0EDB8E0DC
:10789A000E94C0670E949573A83EE3E0BE0734F0D9
:1078AA000E9495730E94D972E0933A070E949573D9
:1078BA00A436E0E0BE0734F00E9495730E94C771B7
:1078CA00E0933B070E9495731A9744F00E949573C0
:1078DA000E94EF6D0E94D171E0933C070E9495735C
:1078EA000E94D771E0933D07A0912C07A43109F0BB
:1078FA0055C0A72D0E94C0630E94496D0E220E94A6
:10790A00ED69E0E0F0E00E94957D0E94376C29F075
:10791A00E0E0E0938B07E0938C07E2E0E09337071F
:10792A000E949A73A83EE3E0BE07C8F0E09161079F
:10793A00E05EE09361070E949A730E942372E093CB
:10794A003B070E949A730E940973E0933C070E94C6
:10795A009A73EAE0F0E00E94197EDF0119C0E09113
:10796A006107E056E09361070E949A73A436E0E04B
:10797A00BE0730F00E949A730E940973E0933B0796
:10798A000E949A730E94F672E0933C070E949A73CF
:10799A00EAE0F0E00E945B7EE0933D07A0912C07AD
:1079AA00A531C1F40E94B972A93019F4E2E0E0935A
:1079BA0036070E949F7330F00E94B0730E940973C9
:1079CA00E0933B070E94B0730E94F6720E94B5735F
:1079DA00E0933D07A0912C07E6E10E94727D0E2EEE
:1079EA00E7E10E94727DE029C1F10E94B972A930D3
:1079FA0019F4E2E0E0933607E5E00E948F730E94F3
:107A0A00B973A0912C07E7E10E94C47329F0E4E559
:107A1A00E09338070E94CE73EDE00E94D973A83E26
:107A2A00E3E0BE0730F00E94E0730E942372E09305
:107A3A003A070E94E073A436E0E0BE0730F00E94E5
:107A4A00E0730E940973E0933B070E94E0730E946F
:107A5A00F6720E94E573E0933D07A0912C07A831C6
:107A6A0011F5A0E023FCA1E00E94C063A0E0F79911
:107A7A00A1E00E943E6991F40E94E0671A9744F0DF
:107A8A000E94E0670E94EF6D0E94D171E09338076F
:107A9A000E94E0670E94D771E09339070E94FC7246
:107AAA00E5E0E0933D07A0912C07A931D9F40E94A3
:107ABA00CC720E9445660E94DD7E10F40E94E97332
:107ACA000E94F4730E94FB730E94037419F4EAE0A3
:107ADA00E0933B070E9409740E94F6720E940E749A
:107AEA00E0933D07A0912C07AA3161F40E94127419
:107AFA0018F0E1E0E09336070E9426740E9436747B
:107B0A000E945874A0912C07AB3109F04FC00E9413
:107B1A00CC72E2E0E09336070E942C730E949171C6
:107B2A000E94D9720E94677419F4EAE0E0933A0756
:107B3A000E9491710E94C7710E946D7419F0EAE067
:107B4A00E0933B070E9491710E94EF6D0E94D171F0
:107B5A00E0933C070E9491710E94D771E0933D0720
:107B6A00A0918D08AA2312F50E94B2710E94FC7C92
:107B7A000E94616C0E94D1710E94037421F4EDE0AD
:107B8A00E0933B0703C0EDE0E0933A070E94B2712D
:107B9A000E9489710E94D171E0933C070E94B271E0
:107BAA000E94FC7C0E94D171E0933D07A0911607C8
:107BBA000E945D65A09117070E942571A091180780
:107BCA000E942571A09119070E94C26C09F43BC05A
:107BDA00F79928C00E947974ECE70E948274E0E069
:107BEA00E0933907E5E00E948874EAE0E0933C07F5
:107BFA00E1E0E0933005A09112070E945D65A09133
:107C0A0013070E942571A09114070E942571A09163
:107C1A0015070E94C26C11F0E8E301C0EAE0E093A4
:107C2A003D0711C0E0E0E0931607E0931707E093E1
:107C3A001807E0931907E0931207E0931307E093FC
:107C4A001407E0931507A0912907A13029F4E0E071
:107C5A00F799E1E0E0933005A0E020FCA1E00E9462
:107C6A008E74A0911C050E945D65A0911D050E945D
:107C7A002571A0911E050E942571A0911F050E94E1
:107C8A00C26CE12181F00E947974EAE0E09337073F
:107C9A000E944871E9E3E0933B07E6E7E0933C077B
:107CAA00EDE3E0933D07A0E020FCA1E0E1E00E94C3
:107CBA00727D1E2EA0911C050E945D65A0911D0576
:107CCA000E942571A0911E050E942571A0911F0591
:107CDA000E94C26CE121B9F1E0916107EF77E0936C
:107CEA006107A0912C07A33618F4EAE0E0930B078A
:107CFA00E2E0E0933607E4E5E0933707A091E50771
:107D0A00B091E6070E940973E0933807A091E5074E
:107D1A00B091E6070E94F672E0933907EEE3E0932A
:107D2A003A07ABA9BCA91A9744F0ABA9BCA90E940F
:107D3A00EF6D0E94D171E0933B07ABA9BCA90E94E9
:107D4A00D7710E949374A8890E942569AF850E9401
:107D5A002F7109F48DC00E947974EAE0E093370725
:107D6A000E9448710E945071AF850E942569A889B6
:107D7A000E94BD6C49F1AF85A13029F40E94997423
:107D8A00ECE0E0933A07AF85A23029F40E94997497
:107D9A00EDE0E0933A07AF85A33029F40E94997485
:107DAA00EBE0E0933A070E94A07429F00E949974CC
:107DBA00ECE0E0933A070E94AA7429F00E949974B1
:107DCA00EBE0E0933A0728C0AF85A13029F40E947E
:107DDA00B474ECE0E0933D07AF85A23029F40E9429
:107DEA00B474EDE0E0933D07AF85A33029F40E9417
:107DFA00B474EBE0E0933D070E94A07429F00E945E
:107E0A00B474ECE0E0933D070E94AA7429F00E9442
:107E1A00B474EBE0E0933D07A889A13029F40E94ED
:107E2A00BB74ECE0E0933D07A889A23029F40E94D4
:107E3A00BB74EDE0E0933D07A889A33029F40E94C2
:107E4A00BB74EBE0E0933D07A889E4E00E94C274AA
:107E5A0029F00E94BB74ECE0E0933D07A889E5E0B5
:107E6A000E94C27429F00E94BB74EBE0E0933D07C4
:107E7A00A09110070E942569A0911107E0E00E94D5
:107E8A00907D0E2AA09128070E94F46E29F0E091B5
:107E9A002807EF5FE0932807A09110070E94C063AC
:107EAA00A09111070E943E6919F0E0E0E0932807CB
:107EBA00A09110070E9425690E94CA740E94D57475
:107ECA001E2EA09111070E9425690E94CA740E9461
:107EDA00D574E129D1F00E9479740E942273A0918D
:107EEA001007A13030F0E09110070E94DC740E9464
:107EFA00E274A0911107A13030F0E09111070E94BD
:107F0A00DC740E94E9740E94F074A0911007E4E006
:107F1A000E94907D0E2E0E94F7740E94D5741E2E28
:107F2A00A0911107E4E00E94907D0E2E0E94F77442
:107F3A000E94D574E129F9F00E9479740E942C7389
:107F4A00E8E7E0933907A0911007A13038F0E091F3
:107F5A001007E4500E94DC740E94E274A091110799
:107F6A00A13038F0E0911107E4500E94DC740E94BD
:107F7A00E9740E94F074A09110070E9400750E9493
:107F8A00D5741E2EA09111070E9400750E94D57407
:107F9A00E129E1F00E9479740E943373A0911007DD
:107FAA00A13038F0E0911007E8500E94DC740E947A
:107FBA00E274A0911107A13038F0E0911107E8505E
:107FCA000E94DC740E94E9740E94F074A091110767
:107FDA000E942569A0E0F799A1E0E1E00E94727D84
:107FEA000E942A690E948B7DE02119F0E0E0E0936B
:107FFA003005A091FB06A13081F4E0916207EB7F86
:10800A00E0936207EF7EE0936207EF5FE093620717
:10801A00E0916107EF77E09361070E94616FA436F0
:10802A0038F4E4E6E09377070E940975E09378074D
:10803A000E94616FA53648F00E94616FE8ECEA1B66
:10804A00E0937707E4E6E09378070E94616FA4362D
:10805A0029F4E4E6E0937707E0937807A0913905DD
:10806A00A43638F4E4E6E0932607E0913905E09374
:10807A002707A0913905A53638F0E8ECEA1BE0930A
:10808A002607E4E6E0932707A0913905A43629F4E8
:10809A00E4E6E0932607E0932707A0912C07A3368E
:1080AA0011F00C941C54E1E0E0932D07A0912D07E8
:1080BA00A03148F40E941075AAE0A083E89431F830
:1080CA000E94A168F3CFA52FE9E50E941675E8E59D
:1080DA000E94727DE02909F050E5513509F45AE50C
:1080EA00503089F4E881E03019F4E42F0E941B75BE
:1080FA00A881A13040F0E881F0E03197E053FA4FCF
:10810A00E0810E941B75513019F4EEA50E941B757F
:10811A00523021F40E94F46D0E941B75533021F4F1
:10812A000E9409750E941B75543021F40E94217522
:10813A000E941B75553029F40E94566CE0810E94FA
:10814A001B75563051F40E947B6C0E948B6A0E9408
:10815A00566AA7EFB7E00E949F67573039F4A0919B
:10816A001905E2E0EA9FF0010E942875583021F4CF
:10817A00E09138050E941B75593029F40E943B6C26
:10818A00E0810E941B755A3029F40E94706CE081CC
:10819A000E941B755B3021F40E942D750E941B758D
:1081AA005C3021F40E94B26F0E9428755D3021F480
:1081BA000E9478690E9428755E3021F40E94B96D88
:1081CA000E9428755F3021F40E94D16F0E942875A1
:1081DA00503121F40E943B6A0E943475513121F4D6
:1081EA000E94296A0E943475523121F40E94E36F79
:1081FA000E943475533129F40E94436AE0810E9437
:10820A001B75543121F4E09158050E941B755531B4
:10821A0021F4E09122050E941B75563121F4E09168
:10822A0021050E941B75573121F4E09123050E9414
:10823A001B75583121F4E09101070E941B755931D1
:10824A0021F40E94A76C0E9428755A3119F4E9A5F5
:10825A000E941B755B3119F4EB890E941B755C3116
:10826A0019F4EC890E941B755D3121F40E94AB67F9
:10827A000E9428755E3121F40E9429700E94287597
:10828A005F3121F4E09107050E941B75503229F4F1
:10829A000E944470E0810E941B75513229F40E94A9
:1082AA004D70E0810E941B75523229F40E9453706E
:1082BA00E0810E941B75533229F40E945970E081B3
:1082CA000E941B75543229F40E945F70E0810E945B
:1082DA001B75553219F4EB8D0E941B75563219F431
:1082EA00EA8D0E941B75573219F4E98D0E941B759D
:1082FA00583219F4E88D0E941B75593221F4E09125
:10830A0040050E941B755A3221F4E09139050E94FA
:10831A001B755B3231F4E0912B08F0912C080E9416
:10832A0028755C3219F4EA890E941B755D3251F492
:10833A000E9434670E949C7B0E94566AA7EFB7E0AE
:10834A000E949F675E3221F40E94BA680E942875D3
:10835A005F3221F4E09121070E941B75503321F40A
:10836A00E09115050E941B75513319F4EC850E94A2
:10837A001B75533319F4ED890E941B75543321F48C
:10838A00E09154050E941B75553321F4E09155057F
:10839A000E941B75563321F4E09156050E941B7505
:1083AA00573331F4E0913E05F0E031960E9428758A
:1083BA00583319F4ECA50E941B75593321F40E9415
:1083CA00976B0E9428755A3319F4EAA50E941B7507
:1083DA005B3321F4E091F1050E941B755C3321F4B3
:1083EA00E0913A050E941B755D3321F4E091010585
:1083FA000E941B755E3321F4E091C3050E941B7530
:10840A005F3321F40E941B6C0E942875513421F4B9
:10841A00E091FC060E941B75523421F4E091FD069E
:10842A000E941B75533419F4EE890E941B7554344B
:10843A0021F40E94866A0E942875553421F4E0913D
:10844A0059050E941B75563421F40E9443690E9403
:10845A002875573419F4EF8D0E941B75583421F48E
:10846A00E0910C070E941B75593421F4E0910D0725
:10847A000E941B755A3421F4E091CD050E941B75A8
:10848A005B3439F40E94706C0E94766CE0810E9421
:10849A001B755D3421F4E0911B050E941B755E3447
:1084AA0021F4E0917F070E941B755F3421F4E0916B
:1084BA0080070E941B75503521F4E0912A070E941B
:1084CA001B755A3531F40E94DF6B0E9438750E9481
:1084DA0028755C3521F4E09106050E941B750E94FF
:1084EA00B6700E94E96C21F0E091F3050E941B75B9
:1084FA000E94B6700E943E6921F0E091F4050E9444
:10850A001B75503621F40E94BF700E94287551369F
:10851A0021F4E091F2050E941B75523629F40E945B
:10852A00E76EEC910E941B750E94C4700E94E96C70
:10853A0019F0E8A50E941B750E94C4700E943E694A
:10854A0019F0EEA10E941B75A52F0E94C063A52FEA
:10855A00EEE00E943D75EFE00E94727DE0291E2E3A
:10856A00A52FE9E10E94727D0E2E0E944275EBEF63
:10857A00F0E00E94AD7DE021E1290E2EA52FEDE16C
:10858A000E943D75EBE20E943D75EEE20E943D7548
:10859A00E8E30E943D75E9E30E943D75EFE30E941E
:1085AA00727DE0291E2E0E94D06B0E2E0E947563EA
:1085BA000E948867E0211E2A0E94D06B0E2E0E941C
:1085CA00F66B0E9488670E944775E5E00E94517524
:1085DA00E8E00E948B7D0E944775E0E00E94517599
:1085EA00E3E00E948B7D0E944775E4E00E94727D61
:1085FA000E944775EDE00E945175E1E10E948B7D72
:10860A00E021E12911F0F59A01C0F598A0E0F59969
:10861A00A1E0EA2FE795E0E0E7950E945775A52FBC
:10862A00B0E0A7FDBFEF0E94EF6D0E94D171E09309
:10863A003107A52FB0E0A7FDBFEF0E94D771E093E5
:10864A003207A52FE1E00E946175E7E00E94817D73
:10865A00E0211E2EA52FE8E00E946175ECE00E9441
:10866A00817DE021E1290E2EA52FE3E10E943D75CF
:10867A00ECE40E94727DE02961F1A0912B070E942F
:10868A005D650E94B86699F0E0916307EC5FE0933C
:10869A006307A0912B07A43051F4A0E0F799A1E059
:1086AA000E945871A0E0F799A1E00E945F71A09121
:1086BA002B07A23029F4E0916307EE5FE09363078A
:1086CA00A0912B07A33029F4E0916307EF5FE093B1
:1086DA0063070E944275A031E7E2BE0730F00E94AC
:1086EA0042750E946675E09339070E944275A83E5A
:1086FA00E3E0BE0730F00E9442750E942372E093C5
:10870A003A070E946C7530F00E9442750E94097304
:10871A00E0933B070E9442751A9720F00E947175F8
:10872A00E0933C070E947375E0933D07503049F58A
:10873A00ECE10E947575E0E5E0933507E881E030E9
:10874A0049F4EEE5E0933807E5E0E0933907E3E71B
:10875A00E0933A07A881A13028F00E943373E88198
:10876A00E0933A070E947175E0933C07E881F0E0D4
:10877A0031970E947B75A8810E94BD6C11F00E94FE
:10878A008075513079F4EBE50E947575EDE60E942B
:10879A00867511F40E948E750E944275119711F424
:1087AA000E949775523031F4EDE60E949E75E8E317
:1087BA00E0933507533009F04AC0E9E30E94A475F3
:1087CA00A0917707A43628F0B0E00E94C771E09321
:1087DA003707A0917707AA3038F0B0E00E94EF6D12
:1087EA000E94D171E0933807A0917707BB270E94B6
:1087FA00D7710E94AD750E94B375E0933B07A091B3
:10880A007807AA3058F0B0E00E94EF6D0E94D1714B
:10881A00E0933B070E94B375E0933C07EAE0E093DC
:10882A003D07A0917807A43690F0B0E00E94C77186
:10883A00E0933B07A0917807B0E00E94EF6D0E9499
:10884A00D171E0933C070E94B375E0933D07543021
:10885A0049F4E7E30E94B775E1E70E94867511F4CF
:10886A000E948E75553031F4E3E7E0933307ECE16B
:10887A000E94BD75563091F4ECE70E94C375E9E396
:10888A00E09335070E9442751A9720F00E9471758D
:10889A00E0933B070E9473750E9493745730D9F492
:1088AA00E3E7E0933307E4E70E94C9750E946C7519
:1088BA0030F00E9442750E940973E0933A070E94C1
:1088CA0042751A9720F00E947175E0933B070E9447
:1088DA0073750E9493745830E9F4EEE30E94CF75E1
:1088EA00E5E0E0933507E0913805E03019F4E2E07D
:1088FA000E94D575A0913805A13019F4E4E00E94D0
:10890A00D575A0913805A23029F4ECE70E94DE75EE
:10891A000E94E475593031F4E7E7E0933407E5E063
:10892A00E09335075A3009F044C00E94EB75E4E53C
:10893A000E94867561F4EEE3E0933707E0E00E9457
:10894A000373E8E70E94F275EDE30E94F8750E944E
:10895A004275119761F4E9E3E0933707EEE30E9469
:10896A00FE75E0E50E940476E4E50E940A760E941C
:10897A004275129759F4EEE30E941076E8E70E94D6
:10898A00AD75E9E3E0933B070E9416760E944275B3
:10899A00139779F4E6E7E0933707EBE5E0933807B6
:1089AA00EAE0E0933907E7E30E94DE75EEE50E940C
:1089BA00F8755B3019F5EDE60E941D76EDE30E942D
:1089CA00867561F4EDE6E0933807E7E6E093390748
:1089DA00EEE30E94F275E0E50E94F8750E94427586
:1089EA00119761F4EDE6E0933907E0E30E942376FC
:1089FA00EEE3E0933C07EDE6E0933D075C30C1F41B
:108A0A00EEE30E942976ECE7E0933507EEE3E09384
:108A1A003A070E9442751A9720F00E947175E093F6
:108A2A003C070E947375E0933D07E0E2E093630719
:108A3A00A52FEDE10E941675EEE20E94727DE029F3
:108A4A0021F00E947175E0933C075D30B9F40E94F1
:108A5A00E7700E941B690E944672E09333070E94E6
:108A6A002F760E944672E09334070E942F760E9466
:108A7A006C7EE0933507E0E2E09363075E3031F401
:108A8A00EEE3E0933307ECE00E9435765F3031F491
:108A9A00EEE3E0933307EBE00E943576503121F59F
:108AAA00ECE70E943B76ECE0E09339070E94D0693C
:108ABA00A436E0E0BE0734F00E94D0690E94C77174
:108ACA00E09333070E94D0691A9744F00E94D06954
:108ADA000E94EF6D0E94D171E09334070E94D06921
:108AEA000E94D771E09335075131F1F40E94417623
:108AFA00ECE00E94487634F00E9452760E94C771D8
:108B0A00E09333070E9452761A9744F00E945276F5
:108B1A000E94EF6D0E94D171E09334070E94527651
:108B2A000E94D771E09335075231F1F40E944176E1
:108B3A00EBE00E94487634F00E9452760E94C77198
:108B4A00E09333070E9452761A9744F00E945276B5
:108B5A000E94EF6D0E94D171E09334070E94527611
:108B6A000E94D771E0933507533111F5E8E30E946B
:108B7A001D76E7E70E94867511F40E9457760E94D7
:108B8A005F7648F4E8E3E0933907E0E0E0933A07D8
:108B9A00EDE3E0933B070E9442751A9748F0E8E339
:108BAA00E0933807E0E0E0933907EDE30E94DC74D4
:108BBA005431C1F4E8E30E941D76ECE70E94867501
:108BCA0059F40E94D272E4E5E0933A07EEE5E093A5
:108BDA003B07E0E50E940A760E944275119711F45C
:108BEA000E9457765531B9F40E946376ECE00E94F0
:108BFA006D7611F40E948E750E945F7660F40E9471
:108C0A0042751A9720F00E947175E0933B070E9403
:108C1A0073750E9475765631B9F40E946376EBE05B
:108C2A000E946D7611F40E948E750E945F7660F440
:108C3A000E9442751A9720F00E947175E0933B07D3
:108C4A000E9473750E947576573129F40E946376E3
:108C5A00E0E4E0933707583149F40E94EB750E942B
:108C6A007B760E946C7511F40E948E75593189F4D5
:108C7A00E5E00E949E750E947B760E947175E093E2
:108C8A003C070E944275AB3FE0E0BE0710F00E942D
:108C9A008E755A3171F40E948276EEE30E948675CF
:108CAA0011F40E9497750E944275119711F40E945F
:108CBA008E755B3129F40E948276EEE0E0933507E7
:108CCA005C3149F4E9E30E94CF75EAE00E948675B7
:108CDA0011F40E948E75A52FEDE10E941675EEE142
:108CEA000E94727DE029D1F0E3E70E9410765D319F
:108CFA0011F4EEE501C0E8E7E09339070E948976AE
:108D0A001A9730F00E9489760E94F672E09334072F
:108D1A000E9489760E944172E09335075F3149F4D7
:108D2A00E8E3E0933307EDE6E0933407E3E7E09303
:108D3A003507A52FEFE10E946175E5E20E94817D6A
:108D4A00E02109F43FC1EDE60E948E76E52FEF514E
:108D5A000E94867561F4E1E0E0933807EDE3E09361
:108D6A003907E4E50E94DE75E0E50E94F8750E9485
:108D7A004275119711F40E9494760E9442751297D7
:108D8A0049F4E0E0E0933B07EEE5E0933C07E0E0DE
:108D9A00E0933D070E944275139761F4E7E3E0937D
:108DAA003807E7E7E0933907E4E70E94DE75E5E074
:108DBA000E940A760E944275149721F40E94A176B5
:108DCA000E94A6760E944275159711F40E94AB760E
:108DDA000E944275169711F40E94A6760E94427567
:108DEA00179759F4E7E7E0933807E9E3E09339077F
:108DFA000E94DC74ECE70E94B5760E9442751897CF
:108E0A0049F4E3E70E940373E7E70E942376EAE066
:108E1A000E940A760E944275199721F40E94A1764F
:108E2A000E94A6760E9442751A9711F40E94AB76A8
:108E3A000E9442751B9761F4E9E3E0933907E8E37E
:108E4A000E94DC74E7E7E0933C07ECE7E0933D0718
:108E5A000E9442751C9759F4E3E7E0933907E0E072
:108E6A00E0933A07EEE3E0933B070E94E9740E941D
:108E7A0042751D9719F4E7E30E94BB760E9442757A
:108E8A001E9719F4ECE70E94BB760E9442751F9761
:108E9A0019F4E9E30E94BB760E944275509711F4D7
:108EAA000E94CD760E944275519729F40E94D57688
:108EBA00E1E0E0933D070E944275529729F40E942F
:108ECA00D576E2E0E0933D070E944275539731F46C
:108EDA00E0E5E0933B07E3E70E94DC760E944275F7
:108EEA00549761F4E8E70E94FE75E1E0E0933A07DF
:108EFA00E3E70E94E276E2E0E0933D070E944275D2
:108F0A00559731F4E9E7E0933B07E0E50E94E876FC
:108F1A000E944275569761F4E5E0E0933807E3E76B
:108F2A00E0933907E9E70E940476EEE50E94E876C5
:108F3A000E944275579761F4E5E00E948F73E9E752
:108F4A000E94EE76EEE5E0933B07E4E50E94E876C0
:108F5A000E944275589749F4E3E70E940373E7E7D2
:108F6A000E942376EAE00E94F4760E94427559979D
:108F7A0061F4E1E0E0933807ECE7E0933907E7E7CB
:108F8A000E948874E8E70E94E8760E9442755A9720
:108F9A0061F4E8E7E0933807E1E0E0933907E4E5B4
:108FAA000E940476EAE00E94DC760E9442755B9792
:108FBA0049F4E1E0E0933907ECE70E94F275E8E74B
:108FCA000E940A76553249F4EAE00E948E76E5E07C
:108FDA000E94867511F40E948E75563249F4EAE0B1
:108FEA000E948E76E8E00E94867511F40E948E75C2
:108FFA00573241F40E94FA76E0E00E94867511F435
:10900A000E948E75583241F40E94FA76E4E00E947A
:10901A00867511F40E948E75593231F4E0E00E948F
:10902A00B775E8E7E09335075A3209F04AC0ECE72A
:10903A000E94A475A0912607A43628F0B0E00E94E9
:10904A00C771E0933707A0912607AA3038F0B0E03D
:10905A000E94EF6D0E94D171E0933807A091260714
:10906A00BB270E94D7710E94AD750E940177E093D9
:10907A003B07A0912707AA3058F0B0E00E94EF6D95
:10908A000E94D171E0933B070E940177E0933C076D
:10909A00EAE0E0933D07A0912707A43690F0B0E0FC
:1090AA000E94C771E0933B07A0912707B0E00E9496
:1090BA00EF6D0E94D171E0933C070E940177E09323
:1090CA003D075B3269F4ECE70E942976E8E7E09312
:1090DA0035070E947175E0933C07E0E2E09363076D
:1090EA005C32C9F4ECE70E94057741F4E4E5E093C9
:1090FA003807E0E00E94FE710E940B770E944275D9
:10910A00119749F4E0E50E94EE76E5E0E0933B072B
:10911A00E9E70E940A765D3259F4E0916107E05C62
:10912A00E0936107E0E00E94CF75E0E0E093350745
:10913A005E3231F4E9E3E0933307E8E30E943576DF
:10914A005F32B9F5E8E70E94C375E5E00E948675CB
:10915A0011F40E948E750E944275119711F40E94B3
:10916A00CD760E944275129711F40E9494760E945D
:10917A004275139791F4E8E7E0933707E1E0E0934B
:10918A003807E4E5E0933907EDE00E948874E0E5EA
:10919A00E0933C07E3E7E0933D070E94427514978A
:1091AA0041F4E8E70E943B76E3E70E94FE710E94E1
:1091BA000B77503361F4E9E70E94057711F40E94B6
:1091CA0097750E944275119711F40E948E7551335A
:1091DA00B1F4E3E7E0933307E0E50E941077A0914A
:1091EA000305A43160F0E4E5E0933707EDE6E09388
:1091FA003807E0E3E0933907EDE3E0933A075233A7
:10920A00A9F5EDE60E941677E3E6E0933507EF89C4
:10921A00E03061F4EEE5E0933A07E0E3E0933B07E0
:10922A00EDE6E0933C07E3E7E0933D07AF89A13021
:10923A0049F4E7E3E0933907ECE50E948874ECE52A
:10924A000E94B576AF89A23029F4ECE7E0933B0798
:10925A000E94E475AF89A33049F4E9E3E093390742
:10926A00ECE50E942376E8E70E94B5765333A1F530
:10927A00E7E7E0933307E0E40E941077ED89E030F6
:10928A0019F4E7E7E0933D07AD89A13031F4E7E748
:10929A00E0933B07E0E40E940A76AD89A23041F4EC
:1092AA000E941C77E6E70E942477EEE5E0933D07EB
:1092BA00AD89A33059F40E941C77E9E3E0933B0798
:1092CA00E0E5E0933C07ECE1E0933D07AD89A4308B
:1092DA0019F4E8E7E0933D07543369F4E8E70E949C
:1092EA0016770E9422730E944275A338E0E0BE07F7
:1092FA0011F40E948E75553381F4E8E70E941677BF
:10930A000E942C73E8E7E09339070E944275A7345C
:10931A00E0E0BE0711F40E948E75563369F4E8E75F
:10932A000E9416770E9433730E944275A536E0E0C8
:10933A00BE0711F40E948E755733A9F4E4E5E09351
:10934A003307E9E30E941077A091CC05E1E00E947F
:10935A00777D0E2EA0E0F799A1E00E94E96C19F042
:10936A00EAE0E0933D07583331F4EEE50E941D76BA
:10937A00E7E7E09335075933F9F4A091D308AA2314
:10938A002AF4E0E0E093D208E093D3080E94BB6B92
:10939A00A436E0E0BE0724F00E947471E09333071C
:1093AA000E947F710E94D171E09334070E94BB6BC7
:1093BA000E94D771E09335075A3331F4E7E3E0931B
:1093CA003307E9E30E942A775B3369F4E5E0E09327
:1093DA003307E0933407E8E3E0933507E091F105BA
:1093EA00EF5FE0933D075C3399F4E6E70E94B775B7
:1093FA00EAE00E94867561F4E7E7E0933A07ECE158
:10940A00E0933B07E8E7E0933C07ECE5E0933D0790
:10941A005D3351F5E0E00E9489630E943D73E9E300
:10942A000E941677E0E0E0933507EAE0E0933C0714
:10943A00E0933D070E941A72EA0FE0936207A09137
:10944A000105AA3018F0E2E0E09336070E94D970CD
:10945A00E09337070E94A2700E94D171E093380707
:10946A000E94A670E09339075E3301F5E091620726
:10947A00E061E0936207E8E3E0933307E9E3E0930E
:10948A003407EEE5E0933507E1E0E0933707A09172
:10949A00C305E3E0EA1BE0933807ECE7E0933A07F9
:1094AA00E1E0E0933B07E7E70E94F4765F3349F493
:1094BA00E1E70E94B775EAE0E0933507E0E6E0935A
:1094CA006307503449F5E9E3E0933307E0E0E093BA
:1094DA003407EEE5E0933507A091F706B0E00E9465
:1094EA00EF6D0E94D171E0933A07A091F706BB276E
:1094FA000E94D771E0933B07A091F806B0E00E9462
:10950A00EF6D0E94D171E0933C07A091F806B0E09C
:10951A000E94D771E0933D075134E9F4E4E70E94D1
:10952A002976E1E00E94867561F4E4E50E9482747E
:10953A00E4E50E94FE71E1E00E942477ECE1E09309
:10954A003D070E944275119731F4E1E00E942477A9
:10955A00ECE1E0933D07523419F5E4E70E942976DD
:10956A00E3E60E94867579F4E4E7E0933807EAE0D7
:10957A00E0933907E1E0E0933A07E2E00E940472DF
:10958A00E3E6E0933D070E944275119749F4E4E748
:10959A000E94FE71E6E00E940472E3E6E0933D0752
:1095AA00533469F5EDE6E0933307E8E30E94107758
:1095BA00EE89E03091F4E8E7E0933807EEE6E093CD
:1095CA003907E8E0E0933A07E1E0E0933B07EDE092
:1095DA00E0933C07E1E0E0933D07AE89A13079F4DE
:1095EA00E8E3E0933907E7E3E0933A07E3E0E0933F
:1095FA003B07E5E0E0933C07EEE5E0933D07543492
:10960A0009F5EFA5F8A90E949671A8A9AA2342F420
:10961A00E0918E08F0918F080E94FC7C0E9496715E
:10962A000E949B710E94C771E09333070E94A07148
:10963A000E94D171E09334070E949B710E94D771F6
:10964A00E09335075534B9F4E0E3E0933307EDE6E8
:10965A00E0933407E4E50E94867519F4E1E00E947C
:10966A00DC760E944275119731F4E0E0E0933B0703
:10967A00EEE30E940A765634A9F40E9430770E94DB
:10968A000973E09333070E9430770E94F672E093E1
:10969A0034070E9430770E9441720E94867511F445
:1096AA000E948E755734D9F4E8E3E0933307E0E07B
:1096BA00E0933407E9E30E94867511F40E948E75DF
:1096CA000E945F7660F40E9442751A9720F00E9409
:1096DA007175E0933B070E9473750E947576583442
:1096EA0049F4E7E70E941677E4E50E94867511F4CB
:1096FA000E948E75593409F03FC0EEE30E94167736
:10970A00E4E50E94867531F4EEE30E94DE75E8E333
:10971A000E940A760E944275119759F4E3E70E9463
:10972A003B760E943577EAE0E0933C07EEE3E0936C
:10973A003D070E944275129739F4E3E70E943B768F
:10974A000E9435770E9416760E944275139741F45B
:10975A00E3E70E943B760E943577E4E50E94937422
:10976A000E944275149741F4E3E70E943B760E94F7
:10977A003577EEE30E940A765A3419F5E8E7E09362
:10978A003307E0E5E0933407E5E00E94867531F49B
:10979A00EDE60E94F275ECE10E94F8750E944275AE
:1097AA00149779F4E0E5E0933707E9E7E09338079F
:1097BA00ECE10E94EE76E0E5E0933B07E5E00E94EB
:1097CA00F8755B3431F4E9E30E949E75E1E0E093B9
:1097DA0035075C34C1F4ECE7E0933307E0E50E9417
:1097EA00C9750E94B0700E94A57E3A9730F00E9417
:1097FA00B0700E943A77E0933B070E94B0700E94D3
:10980A003E770E9493745D3471F40E944277ECE1D2
:10981A000E94867511F40E948E750E9442751197F6
:10982A0011F40E9497755E3431F4E3E7E09333074D
:10983A00E9E30E94BD755F3431F4E1E0E093330758
:10984A00E9E30E94BD75503511F5ECE70E94757584
:10985A00E3E70E94867511F40E948E750E94427594
:10986A00119749F4E9E30E94FE75E1E00E948874C9
:10987A00E1E00E9475760E944275129741F4E7E78B
:10988A00E0933B07E8E3E0933C07E0933D075A3552
:10989A0009F05BC0E0E50E941677E0E0E093350747
:1098AA00A091CF050E94907D1E2E0E94EC6B0E9413
:1098BA00F66B0E948867E021E12971F0E091B9070F
:1098CA000E9482740E947175E0933C07E091CF0573
:1098DA00E150E093CF0539C00E94E56BE093D307CE
:1098EA00F093D4070E947471E09337070E947F7146
:1098FA000E94D171E09338070E9449770E94097348
:10990A00E0933B070E9449770E94F672E0933C0776
:10991A000E9449770E944172E0933D070E94EC6BD6
:10992A000E94F66B0E94FB6B81F0F79B08C0EAE08D
:10993A00E0933B07E3E2E0933C07E4E504C0EAE096
:10994A000E942477E3E2E0933D075B3509F042C0C9
:10995A00E8E7E0933307E5E00E941077A0916708F3
:10996A00A03044F0E0916708F0E0E7FDFFEF0E94C5
:10997A00287530C0E0916708F0E0E7FDFFEF0E942C
:10998A00FC7C0E9428750E9442750E947A630E949C
:10999A004275EAE0F0E00E94AD7DE02119F0EDE0C9
:1099AA00E0933C070E944275E9E0F0E00E94B37D33
:1099BA000E2E0E944275E4E6F0E00E94AD7DE021A1
:1099CA0019F0EDE0E0933B070E946C7518F0EDE0AA
:1099DA00E0933A075C3531F4E7E7E0933307E9E3CC
:1099EA000E94C9755D3509F033C4A0916407A83097
:1099FA0008F043C0E7E70E94CF75E09164070E9430
:109A0A004E770E946F630E943875E83EA3E0FA071A
:109A1A004CF00E9453770E943875DF010E94D97278
:109A2A00E0933A070E9453770E943875E436A0E023
:109A3A00FA0754F00E9453770E9438750E94616CAD
:109A4A000E94D171E0933B070E9453770E943875B8
:109A5A003A975CF00E9453770E943875DF010E94A2
:109A6A00EF6D0E94D171E0933C070E9453770E94E8
:109A7A0038750E94D171E0933D070E94577749F1EA
:109A8A00E6E70E941677E0916407E750E09335070E
:109A9A00E7E7E0933707ECE7E0933807E9E3E09379
:109AAA0039070E946277E170E0933B070E94627770
:109ABA00E695E170E0933C070E946277E695E695A9
:109ACA000E946A7738970E94717719F4EDE00E9434
:109ADA0076770E947977C1F10E944277E091640714
:109AEA00EB500E944E770E948477E170E09338072A
:109AFA000E948A77E695E170E09339070E948A7797
:109B0A00E695E695E170E0933A070E948A770E940B
:109B1A008D77E0933B070E948A77E295E170E093A4
:109B2A003C070E948A77E295EF70E6950E946A7771
:109B3A003C970E94717741F4EDE0E09338070E9468
:109B4A00AD75EDE00E9476770E949277D1F10E947E
:109B5A009A77EEE30E94A077EF50E09334070E94D1
:109B6A00A5770E94A57EE83EA3E0FA0748F00E9486
:109B7A00A5770E94A57EDF010E942372E0933A072F
:109B8A000E94A5770E94A57EE436A0E0FA0730F08D
:109B9A000E94A5770E94AD77E0933B070E94A577C4
:109BAA000E943A77E0933C070E94A5770E943E778D
:109BBA000E94B17770970E94717719F4EAE00E94C7
:109BCA007677A0916407E3E10E94B777E8E10E9403
:109BDA008B7DE02109F464C00E949A77E7E70E942E
:109BEA00A077E351E09334070E94BD770E94A57ED7
:109BFA00FF2332F10E94BD770E94A57EDF010E94F9
:109C0A00D9720E94677419F4EAE0E0933A070E9455
:109C1A00BD770E94C5770E94D1710E94037419F41E
:109C2A00EAE0E0933B070E94BD770E94C9770E9451
:109C3A00D171E0933C070E94BD770E94A57E21C0A6
:109C4A00EDE0E0933B070E94BD770E94CE776CF46B
:109C5A00EDE0E0933A070E94BD770E94C2710E942C
:109C6A00616C0E94D171E0933B070E94BD770E940C
:109C7A00D4770E94D171E0933C070E94BD770E947D
:109C8A00C271DF010E94D771E0933D07E09164073A
:109C9A00F0E074970E94717719F4EAE00E947677EF
:109CAA00A0916407E7E10E94B777ECE10E948B7DFF
:109CBA00E02109F46EC0E7E70E949E75E09164070F
:109CCA00E7510E944E770E94D7770E94A57EFF2314
:109CDA0002F10E94DD770E94C5770E94D1710E942D
:109CEA00037419F4EAE0E0933B070E94DD770E94CF
:109CFA00C9770E94D1710E94E07719F0EAE0E093F7
:109D0A003C070E94DD770E94A57E0E94D171E093F4
:109D1A003D070E94DD770E94A57EFF236AF5EDE0EC
:109D2A00E0933C070E94DD770E94CE776CF4EDE069
:109D3A00E0933A070E94DD770E94C2710E94616C2B
:109D4A000E94D171E0933B070E94DD770E94BC71AB
:109D5A005CF4EDE0E0933B070E94DD770E94D47744
:109D6A000E94D171E0933C070E94DD770E94C27184
:109D7A000E94D171E0933D07E0916407F0E0789783
:109D8A000E94717731F4EAE00E94DC74EAE00E94F2
:109D9A00E876A0916407EBE10E94B777E8E20E94B7
:109DAA008B7DE02109F4BEC0A0916407A03268F45B
:109DBA00E7E30E94A077EB510E944E77EC51A3E0B3
:109DCA00EA02F001EF5FE0930A07A0916407EFE16E
:109DDA000E94B777E4E20E948B7DE02169F0ECE70C
:109DEA000E94A077EF510E944E77E052A3E0EA0268
:109DFA00F001EE5FE0930A07A0916407A43268F0CD
:109E0A00E9E30E94A077E3520E944E77E452A3E06E
:109E1A00EA02F001ED5FE0930A07E8E7E09334070E
:109E2A000E94EC770E94A57EFF230AF10E94EC773C
:109E3A000E94C5770E94D1710E94677419F4EAE002
:109E4A00E0933A070E94EC770E94C9770E94D17189
:109E5A000E946D7419F0EAE0E0933B070E94EC77E8
:109E6A000E94A57E0E94D171E0933C072DC00E94FA
:109E7A00EC770E94C2710E94D171E0933C07EDE039
:109E8A00E0933B070E94EC770E94BC715CF40E944D
:109E9A00EC770E94D4770E94D171E0933B07EDE002
:109EAA00E0933A070E94EC770E94CE776CF40E9406
:109EBA00EC770E94C2710E94616C0E94D171E0939A
:109ECA003A07EDE0E0933907E3E60E94B177BF0174
:109EDA007C970E947B75A0916407E0E20E94A26CC5
:109EEA00FB01B0970E947B75A0916407EFE10E9485
:109EFA00907D0E22E4E20E948B7DE0211E2AFB0166
:109F0A00B4970E947B75A0916407E3E20E94F377FD
:109F1A0049F0EAE00E94FE71EAE0E0933B07EDE0D7
:109F2A00E0933C07A0916407E7E20E94B777ECE26E
:109F3A000E948B7DE02191F1E3E70E94B775E091E1
:109F4A006407E7520E944E770E94F8770E94C77111
:109F5A000E94037419F4EAE0E0933B07E091640776
:109F6A000E94F8770E94EF6D0E94D1710E94E077FB
:109F7A0019F0EAE0E0933C07E09164070E94F87761
:109F8A000E94D7710E94B177B8970E94717731F415
:109F9A00EAE00E94E276EDE0E0933D070E94FF7757
:109FAA000E940378A9F1E3E7E0933307E6E7E09339
:109FBA003407E0916407EB520E944E770E940878BA
:109FCA000E94C7710E94037419F4EAE0E0933B0708
:109FDA00E09164070E9408780E94EF6D0E94D17197
:109FEA000E94E07719F0EAE0E0933C07E091640709
:109FFA000E9408780E94D7710E94B177BC970E948C
:10A00A00717731F4EAE00E94E276EDE0E0933D07F1
:10A01A000E940F78E4E30E948B7DE02159F10E94AF
:10A02A009A77EEE30E949E75E0916407EF520E94D0
:10A03A004E770E9413780E94AD770E94037419F438
:10A04A00EAE0E0933B07E09164070E9413780E94DC
:10A05A003A77E0933C07E09164070E9413780E94E4
:10A06A003E770E94B177F0970E94717719F4EAE07F
:10A07A000E947677A0916407E3E30E94907D0E2EFA
:10A08A000E94606E09F45CC0E0E50E947575E0917B
:10A09A006407E353E09335070E94676E0E941978BC
:10A0AA000E94A57EE031A7E2FA0758F00E94676E87
:10A0BA000E9419780E94A57EDF010E946675E093CE
:10A0CA0039070E94676E0E9419780E94A57EE83EB1
:10A0DA00A3E0FA0758F00E94676E0E9419780E945E
:10A0EA00A57EDF010E942372E0933A070E94676E01
:10A0FA000E9419780E94A57EE436A0E0FA0740F093
:10A10A000E94676E0E9419780E94AD77E0933B0720
:10A11A000E94676E0E9419780E94A57E3A9740F0C5
:10A12A000E94676E0E9419780E943A77E0933C0772
:10A13A000E94676E0E9419780E943E77E0933D075D
:10A14A00A0916407A83309F083C0E4E50E94C375AF
:10A15A00E8E3E09335070E945276E091DE08F09139
:10A16A00DF08AE17BF070CF041C00E94C169A09179
:10A17A00DE08B091DF08AE1BBF0BA093E008B093D6
:10A18A00E108EDE0E0933C070E941D781A971CF065
:10A19A00EDE0E0933B070E9422781CF0EDE0E093AB
:10A1AA003A070E9427781CF0EDE0E09339070E94F5
:10A1BA00277834F00E941D780E94D972E0933A07FA
:10A1CA000E94227834F00E941D780E94C771E093A1
:10A1DA003B070E941D781A9744F00E941D780E943E
:10A1EA00EF6D0E94D171E0933C072AC00E94C169B9
:10A1FA00A091DE08B091DF08EA1BFB0BE093E008B0
:10A20A00F093E1080E94277834F00E941D780E949A
:10A21A00D972E0933A070E94227834F00E941D789E
:10A22A000E94C771E0933B070E941D781A9744F079
:10A23A000E941D780E94EF6D0E94D171E0933C0745
:10A24A00A091E008B091E1080E94D771E0933D0720
:10A25A005E3509F09EC2EDE60E94C375E7E7E0931A
:10A26A003507E0915205E03029F5EDE60E948F733B
:10A27A00EBE0E0933907A0917A09B0E00E94C77138
:10A28A000E94037419F4EAE0E0933B07A0917A096B
:10A29A00B0E00E94EF6D0E94D1710E94E07719F040
:10A2AA00EAE0E0933C07A0917A09BB270E94D771A4
:10A2BA00E0933D07A09152050E945D65A091520569
:10A2CA000E94E66639F10E94B973A0915205E2E054
:10A2DA000E94C47311F00E94CE73E5E00E948F734E
:10A2EA00A0915205A23019F4E4E5E0933807E0E4BE
:10A2FA000E94D9730E9409730E94037419F4EAE058
:10A30A00E0933B070E94E0730E94F6720E94E57395
:10A31A00E0933D07A0915205A330A9F40E94F4737B
:10A32A00EBE0E09338070E94A3650E9409730E943C
:10A33A00037419F4EAE0E0933B070E94A3650E94C4
:10A34A00F6720E949374A0915205A430C9F40E9437
:10A35A0045660E94DD7E10F40E94E9730E94F47340
:10A36A000E94FB730E94037419F4EAE0E0933B072E
:10A37A000E9409740E94F6720E940E74E0933D07CF
:10A38A00A0915205A53021F5E2E0E09336070E943C
:10A39A002C78A0917B09B0E00E94C7710E94677473
:10A3AA0019F4EAE0E0933A07A0917B09B0E00E9431
:10A3BA00EF6D0E94D1710E946D7419F0EAE0E0938A
:10A3CA003B07A0917B09BB270E94D7710E94937417
:10A3DA00A0915205A630B9F40E947A73ECE0E0939A
:10A3EA0039070E9467650E940973E0933B070E9440
:10A3FA0067650E94F672E0933C070E9467650E94B7
:10A40A004172E0933D07A0915205A730B9F40E942A
:10A41A007A73EBE0E09339070E9471650E94097331
:10A42A00E0933B070E9471650E94F672E0933C0735
:10A43A000E9471650E944172E0933D07A091520506
:10A44A00A830E1F50E942C780E947B650E94D9729F
:10A45A00E0933907E0913907E03019F4EAE0E09334
:10A46A0039070E947B650E94C771E0933A070E94F0
:10A47A0033780E943E6919F0EAE0E0933A070E94B5
:10A48A007B650E94EF6D0E94D171E0933B070E94A9
:10A49A003378EAE00E94727D0E22A0913B070E9467
:10A4AA003E6919F0EAE0E0933B070E947B650E944F
:10A4BA00D771E0933C07EEE3E0933D07A091520584
:10A4CA00A930F1F40E9422730E948565A436E0E067
:10A4DA00BE0730F00E9485650E940973E0933A072F
:10A4EA000E9485651A9730F00E9485650E94F6726F
:10A4FA00E0933B070E9485650E9441720E943C7866
:10A50A00A0915205AA3009F50E942C73E8E7E0935E
:10A51A0039070E948F65A436E0E0BE0730F00E943A
:10A52A008F650E940973E0933A070E948F651A9714
:10A53A0030F00E948F650E94F672E0933B070E94FA
:10A54A008F650E9441720E943C78A0915205AB30FF
:10A55A00F1F40E9433730E949965A436E0E0BE07C5
:10A56A0030F00E9499650E940973E0933A070E94AD
:10A57A0099651A9730F00E9499650E94F672E093E5
:10A58A003B070E9499650E9441720E943C78A09103
:10A59A005205AC30A1F5E7E7E0933707E1E7E0932E
:10A5AA0038070E94F3650E94517224F00E94F365F5
:10A5BA000E9485720E94F3650E945E7224F00E94D6
:10A5CA00F3650E9493720E94F3650E946B7244F0D5
:10A5DA000E94F3650E9420710E94A172E0933B07DA
:10A5EA000E94F3650E94D17034F00E9442780E9462
:10A5FA00B172E0933C070E9442780E94B472A09123
:10A60A005205AD30B9F5E7E70E943B760E944E65E8
:10A61A00A031E7E2BE0730F00E944E650E946675DF
:10A62A00E09339070E944E65A83EE3E0BE0730F08A
:10A63A000E944E650E942372E0933A070E944E657B
:10A64A00A436E0E0BE0730F00E944E650E9409730E
:10A65A00E0933B070E944E651A9730F00E944E65C0
:10A66A000E94F672E0933C070E944E650E94417276
:10A67A00E0933D07A0915205AE3079F5EEE3E09301
:10A68A003707E1E7E09338070E9405660E94517296
:10A69A0024F00E9405660E9485720E9405660E9447
:10A6AA005E7224F00E9405660E9493720E940566FB
:10A6BA000E946B7244F00E9405660E9420710E94FB
:10A6CA00A172E0933B070E9449780E94B172E0931D
:10A6DA003C070E9449780E94B472A0915205AF309B
:10A6EA0099F5EEE30E943B760E941366A031E7E2F9
:10A6FA00BE0730F00E9413660E946675E093390720
:10A70A000E941366A83EE3E0BE0730F00E9413667B
:10A71A000E942372E0933A070E941366A436E0E08F
:10A72A00BE0730F00E9413660E940973E0933B074C
:10A73A000E9413660E94F672E0933C070E94136619
:10A74A000E944172E0933D07A0915205A03189F41D
:10A75A000E949F7330F00E94B0730E940973E093C5
:10A76A003B070E94B0730E94F6720E94B573E09391
:10A77A003D07A0915205A13161F40E94127418F0AC
:10A78A00E1E0E09336070E9426740E9436740E9424
:10A79A0058745F35C1F4E8E30E947575EEE5E093FD
:10A7AA003507F6FC03C0ECE0E0933707F6FE03C07A
:10A7BA00EBE0E0933707E091F707F091F80730975D
:10A7CA0011F40E948E75503631F4E8E30E94CF7579
:10A7DA00EDE0E0933507513661F4E3E7E0933307A0
:10A7EA00ECE7E0933407EAE00E94867511F40E94D0
:10A7FA008E75523651F4E8E3E0933307E091200571
:10A80A00E0933407E0E1E0936307533681F4E8E329
:10A81A00E0933307ECE7E0933407F6FC03C0ECE07F
:10A82A00E0933507F6FE03C0EBE0E0933507A0E0BE
:10A83A00F099A1E00E94C063A92D0E94C563A0916E
:10A84A003C050E942F71A1F1E0E00E945775E8943F
:10A85A0031F80E943471E0E0E0933807E1E7E093D1
:10A86A003907E0933A070E945071A0913C05A13044
:10A87A00F8F0A13319F4E1E0E0933005A0913C052A
:10A88A00A03319F4E0E0E0933005A0913C05AC3226
:10A89A0019F4E1E0E0933005A0913C05AD3219F4DA
:10A8AA00E0E0E0933005E0913C05E150E0933C059F
:10A8BA00A0913C05E8E20E948B7D0E2EE0E00E940A
:10A8CA00907D0E22A52DE2E30E94907DE02109F001
:10A8DA002998A091FB06A13081F5E0E00E94577506
:10A8EA000E9450780E945878EAE0E0933607E3E73E
:10A8FA00E0933707A091F906B0E00E94EF6D0E943D
:10A90A00D171E0933807A091F906B0E00E94D7719F
:10A91A00E0933907A091FA06B0E00E94EF6D0E9419
:10A92A00D171E0933A07A091FA06B0E00E94D7717C
:10A93A000E94E276EAE0E0933D07A0916F07A1301A
:10A94A00C9F4E0E00E9457750E9450780E94587836
:10A95A00EAE0E0933607E8E30E948274E7E7E093CF
:10A96A003907EEE5E0933A07E1E00E942477EDE348
:10A97A00E0933D07A0E032FCA1E00E945D650E94E1
:10A98A00226CE02159F0E1E70E941076E5E0E093BD
:10A99A003907E6E70E94DC740E94E974E1E0E0937B
:10A9AA002D07A0912D07A03108F08AC00E941075CA
:10A9BA00E081E03021F40E941075AFE3A0830E9489
:10A9CA001075A081A63021F40E941075ADE7A0830E
:10A9DA000E941075A081A13021F40E941075A6E092
:10A9EA00A0830E941075A081A23021F40E941075E4
:10A9FA00ABE5A0830E941075A081A33021F40E94C8
:10AA0A001075AFE4A0830E941075A081A43021F4D0
:10AA1A000E941075A6E6A0830E941075A081A53039
:10AA2A0021F40E941075ADE6A0830E941075A081E2
:10AA3A00A73021F40E941075A7E0A0830E94107528
:10AA4A00A081A83021F40E941075AFE7A0830E946C
:10AA5A001075A081A93021F40E941075AFE6A08379
:10AA6A000E941075A081AA3021F40E941075A0E0FE
:10AA7A00A0830E941075A081AB3021F40E9410754A
:10AA8A00A1E0A0830E941075A081AC3021F40E943D
:10AA9A001075A8E0A0830E941075A081AD3021F442
:10AAAA000E941075A0E4A0830E941075A081AE30A8
:10AABA0021F40E941075A9E0A0830E94A16871CFB9
:10AACA00A0912A070E945D65A0913005E2E00E94EC
:10AADA00777DE02119F0E0E0E0933005E0912A0764
:10AAEA00E03019F4E0E0E0933005E0910205E695E4
:10AAFA00E6950E945E78E09133070E946378E091C0
:10AB0A0033070E946D78E09133070E947978E091CB
:10AB1A003307E1700E948178E695E170EE0F0E949A
:10AB2A0081780E9486780E9481780E948C78EA2B2C
:10AB3A00E0934007E09102050E948D77E295E07F5D
:10AB4A00AE2FE09134070E946378E09134070E94A7
:10AB5A006D78E09134070E947978E0913507E170C9
:10AB6A000E949078E695E170EE0F0E9490780E941C
:10AB7A0086780E9490780E948C78EA2BE0934107AD
:10AB8A00E0910205E6950E945E78E09135070E9401
:10AB9A006378E09135070E946D78E09135070E944D
:10ABAA007978E0913407E1700E949578E695E17032
:10ABBA00EE0F0E9495780E9486780E9495780E94EE
:10ABCA008C78EA2BE0934207E09136070E945E7880
:10ABDA00E09137070E946378E09137070E946D7809
:10ABEA00E09137070E947978E0916107E1700E944D
:10ABFA009A78E695E170EE0F0E949A780E9486781C
:10AC0A00EA2BAE2FE09102050E942A71EA2BE0930B
:10AC1A004307E0913B070E945E78E0913B070E9460
:10AC2A009F78E0913B070E94A778E0913B070E943A
:10AC3A008D770E94B1780E948D770E94B5780E9424
:10AC4A00BA780E94B5780E94C0780E94B578E295D9
:10AC5A000E942A71EA2BE0934407E0913A070E9486
:10AC6A005E78E0913A070E949F78E0913A070E9445
:10AC7A00A778E0913A070E948D770E94B178E29511
:10AC8A00E1700E94C8780E94BA780E94C8780E942F
:10AC9A00C0780E94C878E2950E942A71EA2BE09354
:10ACAA004507E09161070E94CD78E0913A070E943A
:10ACBA006378E0913A070E946D78E0913A070E9422
:10ACCA007978E0913907E1700E94D178E695E170D0
:10ACDA00EE0F0E94D1780E9486780E94D1780E9455
:10ACEA008C78EA2BE0934607E0913C070E945E7855
:10ACFA00E0913C070E949F78E0913C070E94A77868
:10AD0A00E0913C070E948D770E94B1780E94D67824
:10AD1A00E1700E94D1780E94BA780E94D1780E948C
:10AD2A00C0780E94D178E2950E942A71EA2BE093BA
:10AD3A004707E09138070E945E78E09138070E9441
:10AD4A009F78E09138070E94A778E09138070E941F
:10AD5A008D770E94B178EE1FE0E0EE1FE1700E944D
:10AD6A00DB780E94BA780E94DB780E94C0780E9441
:10AD7A00DB78E2950E942A71EA2BE0934807E0917A
:10AD8A006207E2950E945E78E09138070E94637834
:10AD9A00E09138070E946D78E09138070E9479782F
:10ADAA00E0913707E1700E94E078E695E170EE0FD6
:10ADBA000E94E0780E9486780E94E0780E948C784F
:10ADCA00EA2BE0934907E0913D070E945E78E09103
:10ADDA003D070E949F78E0913D070E94A778E09185
:10ADEA003D070E948D770E94E578E0E031FCE1E0C2
:10ADFA000E94EB78E295E170EE0F0E94EB780E94D8
:10AE0A00C0780E94EB78E295EF70E6950E942A716D
:10AE1A00EA2BE0934A07E0912F070E948D77E2958B
:10AE2A00E07FAE2FE0912F07E695E6950E94F07835
:10AE3A000E94EB780E94F5780E94EB78E1700E94FC
:10AE4A00E578E09162070E948D770E94FC780E9463
:10AE5A0001790E94FC78E170EE0FEE0F0E94FC78F7
:10AE6A00E6950E942A71EA2BE0934B07E09162076C
:10AE7A000E94CD78E0913007E2950E94F0780E9416
:10AE8A0006790E946D78E09130070E940B79E09173
:10AE9A0030070E948D770E9406790E9401790E94EC
:10AEAA0006790E9410790E9406790E942A71EA2B7B
:10AEBA00E0934C07E09162070E94D6780E945E7880
:10AECA00E09163070E94F0780E9415790E94F57854
:10AEDA000E941579E695E695E1700E94E578E09181
:10AEEA000205E295E1700E94FC78EE1FE0E0EE1F99
:10AEFA00E170EE0F0E9415790E948D77EE0FEE0F2A
:10AF0A000E941579E2950E942A71EA2BE0934D0777
:10AF1A00E09163070E94CD78E0913107E2950E94A3
:10AF2A00F0780E941A790E946D78E09131070E94A8
:10AF3A000B79E09132070E948D770E941F790E9457
:10AF4A0001790E941F790E9410790E941F790E943C
:10AF5A002A71EA2BE0934E07E09163070E94D678A4
:10AF6A000E945E78E0913207E2950E94F0780E9492
:10AF7A001F790E946D78E09132070E940B79E09167
:10AF8A0031070E948D770E941A790E9401790E94E6
:10AF9A001A790E9410790E941A790E942A71EA2B62
:10AFAA00E0934F07A091FB06A230A1F4E1E0E09301
:10AFBA002D07A0912D07A13150F4E0912D07F0E063
:10AFCA00E15CF84FA0E0A0830E94A168F2CFE4E020
:10AFDA00E0934B0727FE11C0E1E0E0932D07A09113
:10AFEA002D07A13150F4E0912D07F0E0E15CF84F14
:10AFFA00AFEFA0830E94A168F2CF0E942479A091AA
:10B00A002D07AD3010F50E942C79A091C305A1300F
:10B01A0061F40E943179A0E5B8E00E94217DE170D7
:10B02A0011F4429801C0429A0BC00E943179A2E5FC
:10B03A00B8E00E94217DE17011F4429801C0429A61
:10B04A000E9436790E94A168DACF0E943E79A091C7
:10B05A002D07AD3090F40E942C790E943179A0E33B
:10B06A00B8E00E94217DE17011F4429801C0429A31
:10B07A000E9436790E94A168EACF0E943E79A09187
:10B08A002D07AD3090F40E942C790E943179A2E00C
:10B09A00B8E00E94217DE17011F4429801C0429A01
:10B0AA000E9436790E94A168EACF0E943E79A09157
:10B0BA002D07AD3090F40E942C790E943179A6E0D8
:10B0CA00B8E00E94217DE17011F4429801C0429AD1
:10B0DA000E9436790E94A168EACF0E943E79A09127
:10B0EA002D07AD3010F50E942C79A0913005A230C1
:10B0FA0060F00E943179A0E8B8E00E94217DE170F9
:10B10A0011F4429801C0429A0BC00E943179A0EC16
:10B11A00B8E00E94217DE17011F4429801C0429A80
:10B12A000E9436790E94A168DACF0E943E79A091E6
:10B13A002D07AD3038F50E942C79A09130050E9478
:10B14A002569A0912F050E943E6961F00E9431791C
:10B15A00A2E1B8E00E94217DE17011F4429801C099
:10B16A00429A0BC00E943179A0E1B8E00E94217D89
:10B17A00E17011F4429801C0429A0E9436790E9405
:10B18A00A168D5CFE0912F05E03019F4E1E0E09312
:10B19A002F05E0913005E03019F4E0E0E0932F0547
:10B1AA000E943E79A0912D07AA30A0F40E942C7922
:10B1BA00A0912D07E9E0EA1BA0E4B1E00E94217DFD
:10B1CA00E17011F4429801C0429A0E9436790E94B5
:10B1DA00A168E8CFE1E0E0933E07A0913E07A131E4
:10B1EA0030F5E1E0E0932D07A0912D07A930C8F4CE
:10B1FA000E942C79E0913E07F0E0E15CF84F008074
:10B20A00A0912D07E8E0EA1BA02D0E94107DE170B5
:10B21A0011F4429801C0429A0E9436790E94A168AC
:10B22A00E3CFE0913E07EF5FE0933E07D6CF429A25
:10B23A0084E08A95F1F7449A84E08A95F1F7A72D7C
:10B24A000E94C063A62D0E94B069A82D0E94B06911
:10B25A00AB2D0E94B0690E94BF680E94E77C0E2A4B
:10B26A00AFA5B8A9EBEFFFEF0E94A17D0E2A0E94BD
:10B27A00ED690E9488670E2A0E94F46BE02929F082
:10B28A00E0E0E093A307E093A407A92D0E945D657F
:10B29A00A0E0F099A1E00E943E6941F00E947A671D
:10B2AA00F09AE89427F8E0E0E0933005A0910305CE
:10B2BA00AE3128F4E0910305EF5FE0930305A09116
:10B2CA000305AE3169F5E0E0EFA7E8ABE0932605A8
:10B2DA00E093B408E093B508AC85A43029F00E9445
:10B2EA00BF66E093270516C00E94CD66E093270546
:10B2FA00E3E3F8E00E944779E0932805E7E3F8E002
:10B30A000E944779E0932905EBE3F8E00E94477928
:10B31A00E0932A05E0E0E0939C09E4E1E093030569
:10B32A00EC85E03009F058C0EDE4E093C400A09148
:10B33A008B09ECE30E94727D0E2EA0918C09E7E046
:10B34A000E94727D0E22A0919C09EBE00E94727D00
:10B35A00E021D1F10E944F79E1E0EE87AE85A93074
:10B36A0040F40E9455790E945B79EE85EF5FEE8783
:10B37A00F5CFE0919409E0932307A0912307E8E031
:10B38A000E94087DE0932307E0919509A091230785
:10B39A00EA0FE0932307A0919307B0919407F0E096
:10B3AA00EA17FB0779F4E0918D09E0932505E0910E
:10B3BA008E09E0932605A0918F09EAE0EA9FF00141
:10B3CA000E9467790E947B79A0919C09AC3020F099
:10B3DA000E9481790E948E79AC85A13009F065C0FE
:10B3EA00EDE4E093C400A0918B09E8E20E94727D2B
:10B3FA000E2EA0919C09E8E00E94727DE02109F4DA
:10B40A004CC00E944F79E0E0EE87AE85A73060F429
:10B41A000E945579A0919307B09194070E949A7956
:10B42A00EE85EF5FEE87F1CF0E94A279E091920953
:10B43A00F0E0EA17FB0789F5E1E0E09325050E94B1
:10B44A00ED69DD9710F0E1E001C0E0E0E093260548
:10B45A000E94A9790E948D77A0912605EA0FE093B0
:10B46A0026050E94A979E170A0912605EA0FE093CA
:10B47A002605E0918E09F0E0EFA7F8ABFFA5E0E022
:10B48A00EFA7F8ABE0918F09F0E0AFA5B8A9EA0FF2
:10B49A00FB1F0E9467790E947B79A0919C09A930C1
:10B4AA0020F00E9481790E948E79AC85A43009F03F
:10B4BA0039C2E0912407E03031F4E981F0E0E75144
:10B4CA00FA4FA0E0A083A0918B09EBE60E94727D5F
:10B4DA000E2EA0918C09EFE00E94727D0E22A0919F
:10B4EA009C09E0E10E94727DE02109F4C7C10E9433
:10B4FA004F79E1E0EE87AE85AF3040F40E9455798E
:10B50A000E945B79EE85EF5FEE87F5CF0E94A27904
:10B51A00E0919A09F0E0EA17FB0709F0AFC1E09160
:10B52A008F09E370E093D4050E94B1790E94B8793B
:10B53A00ED91FD913197FE93EE93503041F4A09135
:10B54A00D405B0E0A053BA4FE0918D09EC93A52F32
:10B55A00EDE50E94727D1E2E0E94226C0E2EA09195
:10B56A001C050E94E96CE12909F44EC00E94577734
:10B57A0041F0A091D405B0E0A25BBA4FE0918D09E9
:10B58A00EC930E94797741F0A091D405B0E0AB51D9
:10B59A00BA4FE0918D09EC930E94927769F0E0919D
:10B5AA00D405AFEAB7E0F0E00E946C6E0E94BE7963
:10B5BA00AFEAB7E00E94CA790E94FF770E94037837
:10B5CA0041F0A091D405B0E0A65EB84FE0918D0994
:10B5DA00EC930E940F78E4E30E94A26C0E94226C12
:10B5EA000E2EA0911C050E94E96CE12969F0E091F8
:10B5FA00D405A5EEB7E0F0E00E946C6E0E94BE7919
:10B60A00A5EEB7E00E94CA790E94DD790E94E4792A
:10B61A000E94DD790E94A57EE030A2E0FA0724F0BC
:10B62A000E94DD790E94EE79E091D405F0E0DE0116
:10B63A00DB960E94F579E09190090E94FF790E94B9
:10B64A00067A0E94E4790E94067A0E94A57EE0307A
:10B65A00A2E0FA0724F00E94067A0E94EE79E091AD
:10B66A00D405F0E0DE01D3960E94F579E0919109C4
:10B67A000E94FF79A091D405B0E0A45EBA4FE09190
:10B68A008F09E1700E940D7AA351BA4FE091920995
:10B69A00EC93E091D4050E946E6BE0919309FF2729
:10B6AA00662777270E94AF7EA091D405B0E0A95DF6
:10B6BA00BA4FE09194090E94127AE695E695E695CA
:10B6CA000E940D7AAB52BA4F0E94177AE6950E94F1
:10B6DA000D7AA752BA4F0E94177AE6950E940D7A00
:10B6EA00A352BA4F0E94177AE695EC93E091950916
:10B6FA00E170AE2FE091D4050E94087DE0932907FE
:10B70A00E091D405F0E0E352FA4F7E2F8F2F60814B
:10B71A00E0919509E170AE2FE0E0F799E1E0EA02E5
:10B72A00F001E62BA72FB82F0E94127AE6950E9405
:10B73A000D7AAF51BA4FE0919509E1700E941B7AD8
:10B74A000E946C6E0E94227AAEEBB8E0F0E00E9492
:10B75A006C6E0E942C7A0E941B7A0E94F579E09105
:10B76A0099090E94FF79E091D4050E94387A0E94D3
:10B77A00227A0E94387A0E942C7AEC93E091D405BE
:10B78A00A6EBB8E0F0E00E94F579E09198090E94F2
:10B79A00FF79E091D4050E943D7A0E94227A0E94A4
:10B7AA003D7A0E942C7AEC93E091D405AAE7B8E09E
:10B7BA00F0E00E94F579E09197090E94FF79E09103
:10B7CA00D405F0E0EA5EF84F0E94427AA6E9B9E0B1
:10B7DA00EC91E695EC93E091D405F0E0EE5EF84F3B
:10B7EA000E94427A0E947B79EDADFEADABADBCAD55
:10B7FA00EA0FFB1FDE01A15CBF4F0D90BC91A02D8B
:10B80A00EA0FFB1FDE01AF5BBF4F0D90BC91A02D6D
:10B81A00EA0FFB1FEFA7F8ABE0E0E0932605E09103
:10B82A00D505EE0FA091D905AE0FE091DD050E9476
:10B83A004B7AA091DA05E091D605EE0FAE0FE091B2
:10B84A00DE050E944B7AA091DB05E091D705EE0F49
:10B85A00AE0FE091DF050E944B7AA091DC05E091E2
:10B86A00D805EE0FAE0FE091E0050E944B7AE09109
:10B87A00D405F0E0E751FA4FA1E0A083A0919C091A
:10B88A00A03118F1E0E0E0938B09E0938C09E09392
:10B89A008D09E0938E09E0938F09E0939009E09374
:10B8AA009109E0939209E0939309E0939409E09354
:10B8BA009509E0939609E0939709E0939809E09334
:10B8CA009909E0939A09E0939C09E981F0E00E94C2
:10B8DA00717741F5E981F0E0E053FA4F0E94547A1A
:10B8EA00EB52FA4F0E94547AE752FA4F0E94547A66
:10B8FA00E352FA4F0E94547ADE01DB960E946C6E84
:10B90A00E0E0F0E0ED93FC93E9810E943D7A0E9429
:10B91A00597AE9810E94387A0E94597A0E94DD6A2E
:10B92A000E94597AEC85E03009F0C6C0ED85E03016
:10B93A0019F0E0E00E945E7AE8E9E093C100442051
:10B94A00D1F5A0912B07A43048F4E0912B07F0E041
:10B95A0034960E94DA69EA0FFB1F03C00E942E6A1E
:10B96A003F96A091EF07B091F007EA0FFB1FBF01C6
:10B97A00A989B0E0E7E00E94187DE60FF71FE0937F
:10B98A009307F0939407AEE30E944661A4E00E94F5
:10B99A004661A0912B07A43008F401C0ABE00E94D5
:10B9AA004661E989E795E0E0E7950E94647AA0910B
:10B9BA00EF070E946B7AE1E0E41509F07DC04424A8
:10B9CA00ACA5B0E00E94D56AEBA7EEA5E095E170C0
:10B9DA00EDA7EBA5F0E0BC96DF01EE27A40FBE1F92
:10B9EA00EDA5F0E0EA0FFB1F0F010E94F46DF0E0F5
:10B9FA00D001AE0FBF1FEAA5F0E0AE0FBF1FE09166
:10BA0A006607F0E0AE0FBF1FE0916707F0E0AE0FE8
:10BA1A00BF1FE0916807F0E0AE0FBF1FE9A5F0E095
:10BA2A00AE0FBF1FE0914005F0E0AE0FBF1F0E94AE
:10BA3A00706CE081F0E0AE0FBF1F0E942D75F0E040
:10BA4A00EA0FFB1FE0939307F0939407AEE30E947B
:10BA5A004661ACE20E944661A42F0E944661ADA5F0
:10BA6A000E9446610E94526F0E944661ABA50E94E5
:10BA7A004661AAA50E944661A09166070E94466196
:10BA8A00A09167070E944661A09168070E944661DB
:10BA9A00A9A50E944661A09140050E9446610E94A4
:10BAAA00706CA0810E944661E0912B07F0E0EA5B8E
:10BABA00FA4FA0810E946B7AAC85A13009F085C04B
:10BACA00AD85A13019F0E1E00E945E7AE8E9E093E1
:10BADA00C100E989EE0FEE0FE98BEF5FE98B0E9457
:10BAEA00ED69A93CE0E0BE0710F00E94406A0E949E
:10BAFA00ED69E5E00E94097E0E94CB690E94496ACD
:10BB0A00A3E3B3E383E890E40E94287CA0E0B0E0DA
:10BB1A0084E393E40E94D87B0E946C6AE989AFE2CD
:10BB2A00EA27AAA5AE27E1E0AE27E6E3AE27E09131
:10BB3A00F007F070EA270E94ED69EA27FB27BF01A8
:10BB4A000E94767AE627F7270E94DA69AE27BF278E
:10BB5A00E1E0F0E0AE27BF27E6E3F0E0EA27FB27C3
:10BB6A000F010E94F46DD001F0E0AE27BF27E091EB
:10BB7A002B070E949A79AFE20E944661A9890E9426
:10BB8A004661A0E00E944661AAA50E9446610E9401
:10BB9A007D7AE091F007AE2F0E944661A091EF07EF
:10BBAA000E9446610E94767A0E94647A0E947D7A97
:10BBBA00A0E00E9446610E94526F0E944661A091D5
:10BBCA002B070E9446610E94837AAC85A23019F441
:10BBDA00E0E8E093C100AC85A43009F04FC3E981E5
:10BBEA00A3E2B8E0F0E0EE0FFF1FEA0FFB1F0F0120
:10BBFA000E94B8790E94A57ED001ED93FC93E98159
:10BC0A00EF5FE983A09138050E94C063A0913805CF
:10BC1A000E94E66689F00E94877AA9810E94BD6C1B
:10BC2A001E2EFB01A0810E942569A981E1E00E94E4
:10BC3A00F37711F0E0E0E983A0913805A13099F497
:10BC4A000E94877AA981E1E00E94907DE0211E2E60
:10BC5A00FB01A0810E942569A981E3E00E94F37794
:10BC6A0011F0E0E0E983A09138050E94C063A09139
:10BC7A0038050E94E66661F0E0E0E093EC05E093A7
:10BC8A00EB050E940975E03019F4E0E0E093EA055B
:10BC9A00A09138050E945D650E94616F0E943E690D
:10BCAA0029F0E0E0E093EC05E093EB05AD85A430E4
:10BCBA0039F0E4E0ED87ECE0E093C4000E947A6793
:10BCCA00EFE0EA83442009F07EC10E94B8790E941D
:10BCDA00A57EE036AAEEFA0738F40E94B879ED910B
:10BCEA00FD913196FE93EE93E0E0E0932407A52FB1
:10BCFA000E94C063A0911B050E943E6919F0E0E012
:10BD0A00E0930B075D3521F50E94577719F0E8E0BB
:10BD1A00E0930B070E94797719F0E9E0E0930B07AB
:10BD2A000E94927719F0E6E0E0930B070E94FF77F2
:10BD3A000E94037819F0E5E0E0930B070E940F7860
:10BD4A00E4E30E948B7DE02119F0EAE0E0930B071F
:10BD5A00E091F605EF5FE093F605A091F605A230B3
:10BD6A0018F0E0E0E093F605E091F305E093F705BB
:10BD7A00E091F405E093F805EAE6E0935007EFE076
:10BD8A00E0935107EA81E0935207A2E5B7E00E94E7
:10BD9A00907AE2E5F7E00F01E081A981EA0FD0018C
:10BDAA00EC93E091FB06E03059F4E0914B05E09307
:10BDBA005307E0914C05E0935407E0914D0507C005
:10BDCA000E94406AE0E0E0935307E0935407E0934F
:10BDDA0055070E94957AA091FF06EA0FD001EC93CD
:10BDEA000E94957AA09100070E94A07AEE0FEE0FAA
:10BDFA00EC93A0912B07A43040F40E94A77AA0915B
:10BE0A002B07EA0FD001EC9305C0E0915307EF5FCF
:10BE1A00E0935307A0912C07E3E60E941675EDE51F
:10BE2A000E945A6E0E94E96C11F00E94136A0E94E5
:10BE3A00ED690E94D97EE0F4E0E0E0935607E091D4
:10BE4A003805E03031F40E94AC7A0E94B97A0E9437
:10BE5A00C87AA0913805A13051F40E94AC7AE093D7
:10BE6A0058070E94B97AE0935A07E09359072FC0FE
:10BE7A00E0EFE0935607E0913805E03031F4E091C5
:10BE8A006808E09357070E94C87AA0913805A13044
:10BE9A0051F4E0916808E0935A07E0935907E09358
:10BEAA005807E0935707A0913805A23081F4E09132
:10BEBA0079070E945C6C0E94587DE0935707E091D5
:10BECA007A070E945C6C0E94587D0E94C87AA091F1
:10BEDA002B07A43018F4E091560703C0E0915607E7
:10BEEA00E15FE0935607E091F505E0935B07ABE568
:10BEFA00B7E00E94907AEBE5F7E00F01E081A091AC
:10BF0A00F605EA0FD001EC93E0915B07F0E0E95007
:10BF1A00FA4FE081E0935C07E0910B07E0935D073D
:10BF2A00ADE5B7E0EC91EE0FEE0FEE0FEC93EDE519
:10BF3A00F7E00F01A081E0E0F6FCE1E0EA0FD001B2
:10BF4A00EC93ADE5B7E0EC91EE0FEC930E94706CC8
:10BF5A00BF01A0810E945D65FB01A081E3E00E9410
:10BF6A00727DE02951F0EDE5F7E00F01A081E0E0F4
:10BF7A0022FCE1E0EA0FD001EC93E0916708E0933C
:10BF8A005E070E944F79E1E0E0932D07A0912D070B
:10BF9A00AF3040F40E94D07AE0810E945B790E941F
:10BFAA00A168F4CF0E94D67AA0912D07AF3038F459
:10BFBA000E94D07AA08165D10E94A168F5CF0E9423
:10BFCA00837A0E94E17AE1E0E41509F057C1E0932F
:10BFDA002407E8E8E093C100ECE6E0935007EFE0BD
:10BFEA00E093510740935207E0911B05E0935307F2
:10BFFA00A3E5B7E0EC91EE0FEC93E0915307E093E1
:10C00A005307A3E5B7E00E94E97AA0913A05A13067
:10C01A0050F0E3E5F7E00F01A0810E94706CE08127
:10C02A00EA0FD001EC93A3E5B7E0EC910E94EE7A17
:10C03A00A09158050E94A07A0E94EE7AA091FD066E
:10C04A000E94A07A0E94EE7AA091FC060E94A07A31
:10C05A00EE0FEC93A0913A05A13048F0E3E5F7E042
:10C06A000F01A0810E942D75EA0FD001EC93E1E047
:10C07A000E94F17AAEA50E94FD7AE0915407EF5F23
:10C08A000E94F17AA9A50E94FD7AA0913F05A130EC
:10C09A0079F4E0E0E0933F05E0915407EF5F0E94F6
:10C0AA00067BE4E5F7E00F01E081A0913E050AC0B6
:10C0BA00E09154070E94067BE4E5F7E00F01E08176
:10C0CA00A0913B05EA0FD001EC93E0E0E09356071C
:10C0DA00E0935507A0913B050E948E740E940B7B4A
:10C0EA00E12989F00E947B6C0E94157BE091770719
:10C0FA000E94916B0E94287C0E94E168A5E5B7E046
:10C10A000E94657BEC93A0913B050E945D65A0911E
:10C11A0038050E943E690E941D7BE12989F00E9430
:10C12A007B6C0E94157BE09178070E94916B0E94BC
:10C13A00287C0E94E168A5E5B7E00E94657BEC9344
:10C14A00A0913B050E948E740E940B7BE12929F085
:10C15A000E94B070EC91E0935607A0913B050E94B3
:10C16A005D65A09138050E943E690E941D7BE12908
:10C17A0029F00E94B070EC91E0935607E091B7075E
:10C18A00E0935707AAE0EA9FF001A091F907EA1B9A
:10C19A00E0935807E091B707AAE0EA9FF001A0915F
:10C1AA00FD070E94D17EEA1BE0935907E091190529
:10C1BA00E0935A070E942D75E03021F4E091800740
:10C1CA00E0935B070E94A36F21F4E0917F07E0935D
:10C1DA005B07ABE5B7E00E94907AEBE5F7E00F0169
:10C1EA00A0810E942175EA0FD001EC93A0913A0533
:10C1FA00BB27EAA5F0E00E940F7EDF01E4E1F0E050
:10C20A000E942C7EE093ED07F093EE07E091ED0794
:10C21A00E0935C07E0E0E0935D07E0935E07E0915E
:10C22A003B05EF5FE0933B05A0913B05A43020F06E
:10C23A004424E0E0E0933B050E944F79E1E0E0937B
:10C24A002D07A0912D07AF3040F40E94D07AE081EB
:10C25A000E945B790E94A168F4CF0E94D67AA091CD
:10C26A002D07AF3038F40E94D07AA0810AD00E94FC
:10C27A00A168F5CF0E94837A0E94E17A0C94390A68
:10C28A00FFCFAA93E091C000E072E1F3E881E09366
:10C29A00C60021960895BA93AA931A93689435F81A
:10C2AA00E7E0E093A109E0E0E093AA09E093AB0993
:10C2BA00E093AC09E093AD09419A409AE093BC003F
:10C2CA00E091B900EC7FE093B900E981FA81A0E737
:10C2DA00B7E10E94197E1E2F183008F018501093EB
:10C2EA00B800E091BC00E078E564E093BC001881F6
:10C2FA0023960895AA93249735FE66C0EA85EE0F21
:10C30A00E093A209E885F985E093A309F093A409CB
:10C31A00E0E0E0939F09EF81E093A509ED81FE81BA
:10C32A00E093A609F093A709E0E0E093A009EC8165
:10C33A00E093A809E6E0E093A1097894EF81E03060
:10C34A0081F0E885F985309709F43EC0EC81E03048
:10C35A0021F0AD81BE81109709F001C035C0689403
:10C36A000DC0EC81E03051F1ED81FE81309761F131
:10C37A00E091A209E160E093A209E89434F8E89414
:10C38A0035F8E091BC00EF70E06AE093BC00E0E2AF
:10C39A00F1EA67E070E00E94B97E35FC0FC00E94A6
:10C3AA00B47E3197604070400E94B97E31F4E5E076
:10C3BA00E093A109689435F807C0EFCFA091A109CD
:10C3CA00E0E00E94727D01C0E0E02B9608950A9297
:10C3DA001A92FA926A937A938A939A93AA93BA933D
:10C3EA00EA93FA93EFB7EA930E94E87E1091A009C4
:10C3FA0000919F093091A5092091A109E12FA091EF
:10C40A00A609B091A709F0E0EA0FFB1FAF01E0917E
:10C41A00B900E87FE83011F420E002C0E03119F4F5
:10C42A00E091A20910C0E83111F0E83249F503178A
:10C43A0098F4E02F0F5FA091A309B091A409F0E04E
:10C44A00AE0FBF1FEC91E093BB00E091BC00EF7010
:10C45A00E068E093BC0013C0E091A8091E1770F4CD
:10C46A00E091A209E160E093A209E89434F8E0912E
:10C47A00BC00EF70E06AE093BC0013C138C011C180
:10C48A00E03531F4E091BB00DA01EC931F5F02C0A2
:10C49A00E03489F4E091A809E1501E1728F0E091F0
:10C4AA00BC00EF70E06804C0E091BC00EF70E06C83
:10C4BA00E093BC00F6C0E83531F4E091BB00DA0144
:10C4CA00EC931F5F02C0E03209F402C0E03309F4C2
:10C4DA0002C0E83469F4203051F434FE03C0031773
:10C4EA0028F005C0E091A8091E1708F424E0D1C07D
:10C4FA00E83331F422E0E091BC00EF70E068CDC08F
:10C50A00E83611F0E83711F422E005C0E03611F000
:10C51A00E037A9F420E010E0E89434F8E091A909A2
:10C52A00E03031F421E0E091BC00EF70E06804C033
:10C53A00E091BC00EF70E06CE093BC00B2C0E03860
:10C54A0011F0E03941F534FE02C021E0A2C0E091C9
:10C55A00BB00DA01EC931F5FE091A9091E17C0F432
:10C56A00E091AA09F091AB09309711F426E091C045
:10C57A00A0E0E091AA09F091AB090995E03039F001
:10C58A00E091BC00EF70E06CE093BC008AC002C08E
:10C59A00689434F802C0E83809F402C0E83939F47A
:10C5AA00E091BC00EF70E068E093BC007AC0E03A2A
:10C5BA00B9F4E091BC00EF70E06CE093BC006894C1
:10C5CA0035F8E091AA09F091AB09309739F0A1E06A
:10C5DA00E091AA09F091AB09099501C026E061C072
:10C5EA00E03B11F422E002C0E83AB9F4E091AC0968
:10C5FA00F091AD09309759F0A0E0E091AC09F091C3
:10C60A00AD0909953E2FE03011F020E002C026E086
:10C61A0040C000E0E89434F802C0E83B01F534FE7B
:10C62A0002C021E036C0E02F0F5FA091A309B091AC
:10C63A00A409F0E0AE0FBF1FEC91E093BB00031713
:10C64A0028F4E091BC00EF70E06C06C0689434F8FE
:10C65A00E091BC00EF70E068E093BC0022C0E03CCF
:10C66A0011F0E83C99F4E091BC00EF70E06CE093C3
:10C67A00BC00E091AC09F091AD09309731F0A1E02E
:10C68A00E091AC09F091AD09099509C0E03049F48F
:10C69A0023E0E091BC00EF70E06DE093BC00689489
:10C6AA0035F81093A00900939F092093A1093093AC
:10C6BA00A5090E94EF7E2696E991EFBFF991E991CB
:10C6CA00B991A9919991899179916991F990199062
:10C6DA0009901895AAE6B8E0F0E0EE0FFF1F08955A
:10C6EA00A091D107B091D2070895E0E0F0E00E944E
:10C6FA00B37D0E2E0895E0E0E7BDE8BD0895B0E0F1
:10C70A000E94287BE0E00895E0935D05E8E6EA935D
:10C71A00EDE5F5E0FA93EA93E1E0EA93EFE5F5E077
:10C72A00FA93EA930895E0E0E0935F05E0936005E9
:10C73A000895E8E6EA93EFE5F5E0FA93EA930895B7
:10C74A00E4E0EA93E0E0F0E0FA93EA93A0E00C94E4
:10C75A007F61E0E0E0935D05E0935E05E0E5EA9342
:10C76A00EDE5F5E0FA93EA93E2E0EA93EFE5F5E026
:10C77A00FA93EA930895E0E00E94727D0E2E0895DE
:10C78A00E0E00E94727D0E220895E0936705E0E0E2
:10C79A00E09368050895E0936A05E0E0E0936B058D
:10C7AA000895E0937505E0E0E09376050895E09337
:10C7BA007705E0E0E0937805E09379050895E09342
:10C7CA007E05E0E0E0937F050895E0938205E0E0CE
:10C7DA00E09383050895E0938405E0E0E0938505FE
:10C7EA00E09386050895E0938A05E0E0E0938B05DF
:10C7FA00E0938C050895E0E0E0938D05E0938E05C3
:10C80A00E0938F05E0939005E0939105E0939205FC
:10C81A000895E0939505E0E0E0939605E093970587
:10C82A00E0939805E0939905E0939A050895E093BB
:10C83A009B05E0E0E0939C05E0939D050895E09355
:10C84A009F05E0E5EA93EFE5F5E0FA93EA930895A8
:10C85A00E1E4EA93E0E0F0E0FA93EA93A0E00E94D0
:10C86A007F61AAE04CCFE0936105E0E0E0936205C6
:10C87A00E0936305E09364050895E0936505E0E0BD
:10C88A00E09366050895E0936905E0E084CFE0E06F
:10C89A00E0936C05E0936D050895E0937005E0E080
:10C8AA00E0937105E0937205E09373050895E093B0
:10C8BA007405E0E076CFE0E0E0938705E093880531
:10C8CA00E093890590CFE0E5EA93EFE5F5E0FA9386
:10C8DA00EA930895EA93E0E0F0E0FA93EA93A0E09D
:10C8EA000E947F61AAE00895B0E00E94287BE1E0FF
:10C8FA000895E0936005E0E0B6CFE0E0E0936E05CE
:10C90A00E0936F050895EBE0E0939009E8EBE0937C
:10C91A0091090895E093DC08F093DD080895E09307
:10C92A008408F093850808950E947F61E0915F056D
:10C93A000895E0939107F09392070895A0919107C3
:10C94A00B09192070895E0938107F09382070895C2
:10C95A00E0938307F09384070895E093F107F09337
:10C96A00F2070895E093F907F093FA070895A09162
:10C97A00F907B091FA070895E093F507F093F607DF
:10C98A000895A091F507B091F6070895E09301087C
:10C99A00F09302080895A0910108B0910208089541
:10C9AA00E0939507F09396070895A0919507B091A3
:10C9BA0096070895E0932B08F0932C0860932D08AE
:10C9CA0070932E080895A0912B08B0912C0880919D
:10C9DA002D0890912E0808950E94687D0E94ED7C92
:10C9EA000895E093A107F093A2070895A091A107E3
:10C9FA00B091A2070895E093A907F093AA070895B2
:10CA0A00A091A907B091AA070895E093B707F093F8
:10CA1A00B8070895A091B707B091B8070895E093B1
:10CA2A00FD07F093FE070895E0935E05E0E5EA93BB
:10CA3A00EDE5F5E0FA93EA93E2E0EA93EFE5F5E053
:10CA4A00FA93EA930895A091FD07B091FE0708951D
:10CA5A00E0935708F09358086093590870935A085E
:10CA6A000895A0915708B09158088091590890915B
:10CA7A005A080895E8E00E942A7DEACFF0E0F1DF43
:10CA8A00ABCFE6DFEEDFF6CFE093AB07F093AC0770
:10CA9A000895A091AB07B091AC070895E093890778
:10CAAA00F0938A070895A0918907B0918A0708959B
:10CABA00E1E00E94727D0E2E0895E0937D09F093C5
:10CACA007E090895A0917D09B0917E090895E093A9
:10CADA007F09F09380090895A0917F09B091800998
:10CAEA000895E093CE08F093CF080895A091CE0858
:10CAFA00B091CF080895E0938109F09382090895CF
:10CB0A00A0918109B09182090895E0938309F09375
:10CB1A0084090895A0918309B09184090895E09346
:10CB2A008509F09386090895A0918509B09186092F
:10CB3A000895E0938709F09388090895A0918709D9
:10CB4A00B09188090895E093DF07F093E00708950C
:10CB5A00E093FF07F09300080895A091FF07B091B2
:10CB6A0000080895E0934308F09344086093450849
:10CB7A00709346080895A0914308B09144088091A3
:10CB8A004508909146080895E093D907F093DA078B
:10CB9A000895E0934B08F0934C0860934D08709306
:10CBAA004E080895A0914B08B0914C0880914D0809
:10CBBA0090914E080895E8E00E942A7DEACFF0E0BD
:10CBCA00F1DF0ACFE6DFEEDFF6CFE093F208F0936B
:10CBDA00F3086093F4087093F5080895A091F20899
:10CBEA00B091F3088091F4089091F5080895E093C4
:10CBFA00F608F093F7086093F8087093F908089517
:10CC0A00A091F608B091F7088091F8089091F90878
:10CC1A000895E093AD07F093AE070895A091AD078C
:10CC2A00B091AE070895E093EA08F093EB08609399
:10CC3A00EC087093ED080895A091EA08B091EB080A
:10CC4A008091EC089091ED080895E093EE08F09336
:10CC5A00EF086093F0087093F1080895A091EE0828
:10CC6A00B091EF088091F0089091F1080895E0934F
:10CC7A004708F09348086093490870934A08089552
:10CC8A00A0914708B09148088091490890914A08B4
:10CC9A000895E0934F08F0935008609351087093F9
:10CCAA0052080895A0914F08B091500880915108F8
:10CCBA00909152080895F6DF8FCEA6E9B0E0A083DE
:10CCCA00B1830895A4E1B0E0A083B1830895E0910F
:10CCDA002B08F0912C0860912D0870912E08089568
:10CCEA00A4E6B0E080E090E00E94E97D08959BDF31
:10CCFA00E0E0E0935F05E3EBE09360059DDFE0E1B0
:10CD0A000E94367DE093610597DFE8E00E94367D58
:10CD1A00E0936205E091EA08E0936305D4CDB0E0C0
:10CD2A000E94287BE091B707F091B8074CDE66278E
:10CD3A0077270E94E97D89DFE0E0E0935F05E6EB73
:10CD4A00E09360058BDFE0E10E94367DE0936105A8
:10CD5A0085DFE8E00E94367DE0936205E091EE0807
:10CD6A00E0936305B0CDA0912B07E4E00E94727DA9
:10CD7A00E0290895EBE0F0E060E070E0E0932F082E
:10CD8A00F09330086093310870933208E8EB089505
:10CD9A00E0E0E0932F08E0933008E0933108E09355
:10CDAA0032080895A091F706BB27E091F806F0E053
:10CDBA00AE0FBF1F0895E1E06E2E9E2E8E2EBE2E60
:10CDCA000895E2E00E94727DE0290895A091FE088C
:10CDDA00B091FF0880910009909101090895A091EE
:10CDEA001209B091130980911409909115090895B7
:10CDFA00E0931209F09313096093140970931509CB
:10CE0A000895A0913209B091330980913409909123
:10CE1A0035090895E0E0F0E060E271E40895A09138
:10CE2A005E09B0915F098091600990916109089546
:10CE3A00E0935E09F0935F0960936009709361095A
:10CE4A000895EEEFFFEF6FE77FE30E94BB7C089542
:10CE5A00A0E0B0E080E89FE30E94D17B0895E091D2
:10CE6A005708F09158086091590870915A08089526
:10CE7A00EF5FFF4F6F4F7F4F0895E091D907F09111
:10CE8A00DA070895E0935F05EFE4E0936005E9DDD2
:10CE9A00E8E10E94427DE0936105E1DF0E945D7D49
:10CEAA00E0936205DEDDE8E00E94427DE0936305DF
:10CEBA00E0915708E093640506CDE0935F05ECE541
:10CECA00E0936005E0918A07E0936105E0918907A4
:10CEDA00E0936205F8CCE0935F05EEE5E093600528
:10CEEA00D0926105C0926205EECCAAE0B0E00C9443
:10CEFA00287BA0919707B09198070895A091A5075C
:10CF0A00B091A6070895E0E0F0E00E94B37D08958D
:10CF1A00E0911A09F0911B0960911C0970911D0991
:10CF2A000895E0913E09F0913F096091400970919E
:10CF3A00410908950E94657BED93FC930895E0E012
:10CF4A00F0E061EE75E40E94767C0895E09197071F
:10CF5A00F09198070895EDECFCEC6CEC7DE30E94EF
:10CF6A00287C0895A0911E09B0911F09809120097B
:10CF7A009091210908950E94677BED93FC9308958F
:10CF8A00E0932209F09323096093240970932509F9
:10CF9A000895E0912609F091270960912809709176
:10CFAA0029090895E0932609F0932709609328092F
:10CFBA00709329090895A0918808B0918908089565
:10CFCA00A0912E09B0912F098091300990913109D1
:10CFDA000895E0E0F0E060E972E40E94767C08954A
:10CFEA00A0913609B0913709809138099091390991
:10CFFA0008950E94D87BE0933609F093370960932D
:10D00A003809709339090895E0910609F0910709E2
:10D01A006091080970910909D3DF0E94287CDF0119
:10D02A00CB01E0E0F0EA6CE877E40E94767C0895B0
:10D03A00A0913A09B0913B0980913C0990913D0930
:10D04A0008950E94D87BE0933A09F0933B096093D4
:10D05A003C0970933D0908950E94D87BE0934209E8
:10D06A00F0934309609344097093450908950E9417
:10D07A00D87BE0934A09F0934B0960934C0970936B
:10D08A004D090895A0914609B09147098091480930
:10D09A00909149090895E0934609F09347096093EE
:10D0AA004809709349090895A0914E09B0914F0912
:10D0BA0080915009909151090895E0934E09F09397
:10D0CA004F0960935009709351090895E091360908
:10D0DA00F091370960913809709139090895E09102
:10D0EA00EA08F091EB086091EC087091ED08089558
:10D0FA00E150F040604070400895E0913A09F091A3
:10D10A003B0960913C0970913D090895E091EE0850
:10D11A00F091EF086091F0087091F1080895A0E08D
:10D12A00B0E080E89FE30895AF39E6E8BE07E1E0A2
:10D13A008E07E0E09E070895E0912D07EF5FE093E8
:10D14A002D0708950E94287CDF01CB010895A09144
:10D15A005209B09153098091540990915509089543
:10D16A00AAE0B0E080E090E00895E091A907F0918C
:10D17A00AA0708952BDEE0E0F0E060E070E0089591
:10D18A000E94E77C0E22A0916808B0916908E0E04D
:10D19A00F0E00895E091FE08F091FF08609100091F
:10D1AA00709101090895A0916209B0916309809173
:10D1BA006409909165090895AAE0B7ED83E29CE3BA
:10D1CA000E94287C0895AE8DECE30E948B7D089521
:10D1DA00E0914308F091440860914508709146082F
:10D1EA000895F4DD17DE0E94287C0895E09147082F
:10D1FA00F09148086091490870914A080895E091B1
:10D20A006308F09164086091650870916608089552
:10D21A00ACE3B0E080E090E00E94E97D0895AFA51C
:10D22A00B8A9E0E0F0E00E94A77D0895E4E6F0E006
:10D23A0060E070E00895662777270E94F77C0895DA
:10D24A00E0E00E94907D0E2E08950E22A0912C07F8
:10D25A00E3E608950E948B7D0E22A091FB06E0E092
:10D26A000E94727DE0210895A091A307B091A407BE
:10D27A000895E0E00E94727DE0210895E091A107FF
:10D28A00F091A2070895E091E307F091E407089569
:10D29A00E093E307F093E407E0E0E0935F05089585
:10D2AA00E093610510CBE09362050DCBA09168086D
:10D2BA00B0916908E0E0F0E00E94A77D0E2EA091EF
:10D2CA00EF07B091F0071FCEA0E022FCA1E0D1CF7A
:10D2DA00E1E04E2EE0E0E0933B050895E09170080E
:10D2EA00F09171080895E0919107F09192070895DD
:10D2FA00A0915308B091540880915508909156080E
:10D30A00662777270895A0E0B0E080E490E40E94C1
:10D31A00D87B0895E0915308F0915408609155081C
:10D32A007091560808950E949C7B0E94AF7E0895D2
:10D33A00E0910705A0910805AE170895E0E01A9953
:10D34A00E1E09E2EE0E01899E1E00895E0E0F0E0E7
:10D35A000E94A77D0895E0E00E94727D0E2A08953A
:10D36A00E0916A08F0916B0808950E94537DE0935A
:10D37A00EF07F093F0070895E0916C08F0916D08BB
:10D38A000895E0936808F09369080895E093EF0719
:10D39A00F093F0070895A0916A08B0916B08089578
:10D3AA00E0918107F09182070895A0916808B091F1
:10D3BA0069080895E0918307F09184070895F5DFDD
:10D3CA00EA17FB070895E091F107F091F207089533
:10D3DA00A091EF07B091F0070895E091F307F0915B
:10D3EA00F40708950E94AD7D0E2EA52DE1E00E945E
:10D3FA00907D0E2208950E94B37D0E2EA52DE1E0A8
:10D40A000E94907D0E220895E4E00E948B7DE02127
:10D41A000895E091EF07F091F0070895E0E0E093B6
:10D42A006808E09369080895E0E0E093EF07E09365
:10D43A00F0070895E4E00E94727D0E2E0895E5E05B
:10D44A000E94727DE0290895A0918107B091820718
:10D45A000895E0916808F09169080895EA1BFB0BAA
:10D46A00A8ECB0E00E94E17D0F010895A091F107B8
:10D47A00B091F2070895E8ECF0E088CFE0912B072D
:10D48A00F0E0ED5CFA4F0895E4DF0E94687D0E94A7
:10D49A009E7B0895E081F0E00E94687D0E949E7B59
:10D4AA000895ADECBCEC8CEC9DE30E94287C0895B9
:10D4BA000E94C87E0E94D17B089531DE0E94D87BEB
:10D4CA00089573DF0E946D7D0E94C57E0895A8E6C7
:10D4DA00B8E051CDEFA5F8A9AEE2B9E00E94687DA7
:10D4EA000E949E7B0E94AF7E08950E94687D0E94E2
:10D4FA009E7B0E94AF7E0895E0917208F0917308B6
:10D50A000895E091F507F091F607089566277727C1
:10D51A000E949E7B0895ED51F1400E94687D0E9411
:10D52A009E7BA1E7BDE38AEA9FE30E94287C0895D7
:10D53A000E940F7EDF01EEE5F1E00E942C7E089545
:10D54A000E94687D0E949E7BB3CFE981AAE7B8E07A
:10D55A00F0E0EE0FFF1FAE0FBF1F0E94A57E0895D9
:10D56A00A981E3E0EA9FF00108953196A2E9B8E0C3
:10D57A00EE0FFF1FEA0FFB1F0895E981A6EBB8E043
:10D58A00F0E0EE0FFF1FAE0FBF1F0E94A57E0895A9
:10D59A003296A2E9B8E0EE0FFF1FEA0FFB1F0895CB
:10D5AA00E2E0F0E00E942C7E08953196DF01F8CF88
:10D5BA00E981AEEBB8E0F0E0EE0FFF1FAE0FBF1F40
:10D5CA000895E0E0E0931007E093110708950E94A0
:10D5DA008B7D0E2EA52DE4E60E94907DE021089514
:10D5EA001A96E0915405F0E0EA17FB070895A09116
:10D5FA00D608B091D7080E94957D0E2E0895A09165
:10D60A00E905E1E00E94727DE0210895A091EA0512
:10D61A00E1E00E94727DE0210895A091EB05E1E02E
:10D62A000E94727DE0210895A091EC05E1E00E943C
:10D63A00727DE02108951A96E0915505F0E0EA1707
:10D64A00FB0708951A96E0915605F0E0EA17FB07E2
:10D65A000895A0E0B0E00E94957D0895E0912B071F
:10D66A00F0E0EE58F84FA081E0E00E94907D089526
:10D67A000E2EA0913805E1E00E94727D0E22EECFB7
:10D68A00ADE9BDEFA083B1830895E091AE08F091B2
:10D69A00AF08EA17FB070895E093AE08F093AF08C6
:10D6AA000895E091B008F091B108EA17FB070895D0
:10D6BA00E093B008F093B1080895E091B208F091B0
:10D6CA00B308EA17FB070895E093B208F093B3088A
:10D6DA000895AFE2B8E0F0E00E944E7DAE0FBF1FA2
:10D6EA000895A0910209B0910309809104099091CB
:10D6FA0005090895E0910209F0910309609104096E
:10D70A00709105090895E0930209F0930309609363
:10D71A000409709305090895F0E00E94687D0E944B
:10D72A009E7B0895E0919507F09196070895EEDEA5
:10D73A000E94AF7E0895E0E0F0E060EC70E40895A6
:10D74A00A0915A09B0915B0980915C0990915D0999
:10D75A0008950E94287CE093FE08F093FF086093E6
:10D76A000009709301090895DDDFD0CEA091D20897
:10D77A00B091D30808954EDB0E94287C089526DBD9
:10D78A00FF27662777270E949E7B08950E2EA09179
:10D79A002C07E3E60895A52FEAE50E94727D089515
:10D7AA00E091B907F091BA070895E093B907F093A9
:10D7BA00BA070895F5DFABEBB7E0EE0FFF1F089548
:10D7CA000E947563E5E2F0E00E94197E08950E94C6
:10D7DA007563E0E0F0E00E94957D0E2E0895E5DD88
:10D7EA00B5CDA091B907B091BA070895E0E0F0E08D
:10D7FA000E94957DE0210895A0E0B0E0A083B18366
:10D80A000895E4DAE0E0F0E060E87FE30E94E17C7A
:10D81A000E220895CADDEACFA0919008B09191082E
:10D82A000895E0919008F09191080895E091FF071A
:10D83A00F091000808954BDA53CAA0912C07E3E649
:10D84A000E948B7D0895C2DAE0E0F0E060E87FEBA9
:10D85A000E94E77C0895BCDDE0E0F0E00E94957D3F
:10D86A000E2EBDCF0E22A091FB0603CDE0912B0711
:10D87A00F0E0E659F84F0895FF27662777270E94B8
:10D88A009E7B0E94AF7E0895A0916A09B0916B09B0
:10D89A0080916C0990916D090895F6DF0E94287CA9
:10D8AA0000CEE0912B07F0E0EB59F84F0895F0E035
:10D8BA007CDD0E940F7E0895DF01E4E6F0E00E941D
:10D8CA002C7E0895E0916609F091670960916809D4
:10D8DA00709169090895E0912B07F0E0EF5BFA4F28
:10D8EA000895E081F0E0E558F84F0895E0912B079C
:10D8FA00A3E0B8E0F0E0EE0FFF1FAE0FBF1F0E94DB
:10D90A00A57E0895A0917209B09173098091740956
:10D91A00909175090895A0918909B0918A0908958D
:10D92A00E0E0E0938909E0938A0908958827992716
:10D93A000E94C57E0E94BB7C08950E948B7DE021D7
:10D94A001E2E0895E091DF07F091E0070895A09157
:10D95A00DF07B091E0070895E091230510CFE9E1D0
:10D96A00EA9FF001D8DF0E94B37DE6230E2E0895C8
:10D97A00E0E00E94907DE0210895E1E00E94727D3E
:10D98A00E0290895E0915609F091570960915809E4
:10D99A007091590908950E22A0915609B09157091C
:10D9AA0080915809909159090895E0E0F0E068E4FF
:10D9BA0073E40E94E17C08950E22A0E022FCA1E01B
:10D9CA00E1E00E94727D0895E1E00E94727DE0210B
:10D9DA000895E0935609F093570960935809709394
:10D9EA0059090895F5DC0C947A63E0E0F0E060E010
:10D9FA0070E00895A0E024FCA1E05AC8AC85E3E0F9
:10DA0A000E948B7DE0210895E0932405E89424F890
:10DA1A00E0E0EC8F0895AB89E2E00E94727D089500
:10DA2A00E091D808F091D90808950E94687D0E9473
:10DA3A009E7B0895E0916E09F0916F0960917009DB
:10DA4A0070917109A0915609B091570980915809AE
:10DA5A00909159090E94D87BDF01CB010895A091CA
:10DA6A00D808B091D9080E946D7D0E94C57E20CD4C
:10DA7A0049DF0E94287CA0916E09B0916F098091BC
:10DA8A00700990917109089590DCE0E0F0E00E943D
:10DA9A00957D08950E2E9CDCE0E0F0E00E94957DD5
:10DAAA000895A3DF0E94B97DE0210895A091560947
:10DABA00B0915709809158099091590908950E2EED
:10DACA00A0E021FCA1E00C94C563E0E0E093D80853
:10DADA00E093D908E0935609E0935709E09358096F
:10DAEA00E09359090895E0910505F0E035975DDC6A
:10DAFA000E94A17D0895E0936E09F0936F096093E7
:10DB0A007009709371090895E0916E09F0916F0997
:10DB1A0060917009709171090895E091F907F09187
:10DB2A00FA07E6CB0E94D17D0E2EA0915308B09140
:10DB3A0054088091550890915608EAE0F0E060E0B8
:10DB4A0070E00E94D97D0895E5DB0E94BC648827B5
:10DB5A0099270E94F77C0895A630E0E0BE07E0E02E
:10DB6A008E07E0E09E070895E091F907F091FA0721
:10DB7A000895A091DC08B091DD080895E091DC08D1
:10DB8A00F091DD080895F0DFA0915308B091540890
:10DB9A0080915508909156084ECB5BDCAAE0B0E024
:10DBAA000E940F7E0895AFA5B8A9AE1BBF0B0895BA
:10DBBA000E94E17DA0918408B09185080895E091C2
:10DBCA008408F09185080895DF01EFA5F8A9AE1B36
:10DBDA00BF0B0895EAE0F0E00E942C7E0895E091E0
:10DBEA002B07F0E0DE011396AE0FBF1FEC910895EC
:10DBFA0030DCA0917609B0917709809178099091EB
:10DC0A00790913CF26DCA6E7B9E06FCCA8ECB0E01F
:10DC1A00A083B1830895A0EFB0E0A083B1830895F3
:10DC2A00A0915405BB27E091AE08F091AF08AE1B56
:10DC3A00BF0B0895EAE0F0E00E94A17D0E2E089540
:10DC4A00E4E1F0E00E940F7E0895A0915505BB27FC
:10DC5A00E091B008F091B108AE1BBF0B0895A091F6
:10DC6A005605BB27E091B208F091B308AE1BBF0B73
:10DC7A000895E1E00E94727D0E220895A0912C077A
:10DC8A00E3E60E94777D0E2208950E22A1DBE0E0F2
:10DC9A00F0E00E94957D0E22B4CD0E94907D76CD53
:10DCAA00A52FEDE50E94727DD0CA0E94727D0E22D8
:10DCBA00A09164070895A0916407E8E30E948B7D10
:10DCCA00E0210895E0916407F0E0F4970895EE0FDB
:10DCDA00FF1FAE0FBF1F0895EA93E0E0F0E0FA934A
:10DCEA00EA93A0E00C947F61A0912005E3E00E94F2
:10DCFA00727D0E2E0895E0E0E093FF060895AA8D46
:10DD0A00E1E00E94907D0E2EE5E00E948B7D089551
:10DD1A00A0914005E3E00E948B7DE0210895E09107
:10DD2A00F205E0934C050895E1E0E98BE8CFE09134
:10DD3A002005F0E0DE019296AE0FBF1FEC91E7BD21
:10DD4A000895A0914B050C94C063A0914005E4E0AE
:10DD5A000E94727DE0210895A0914B0571CAEFEFF0
:10DD6A00E0934C05E0E0E093FF060895A09140059A
:10DD7A00E5E00E94727DE0210895EFEFE0934C0503
:10DD8A00E2E0E093FF060895A0914005E6E00E94D4
:10DD9A00727DE0210895A0914005E7E00E94727D1E
:10DDAA00E0210895E0913D05EF5FE0933D05E2E053
:10DDBA00E093FF060895A0914005E8E00E94727D75
:10DDCA00E0210895E0912005F0E0DE019296AE0F81
:10DDDA00BF1F0895A0917408B09175080895E4E1F1
:10DDEA000E948B7DE0210895E0910405E170AFEF78
:10DDFA00EA02F001E7BD0895E0910405E170AFEF92
:10DE0A00EA02F0010895A0917808B0917908E091AA
:10DE1A000108F09102080895EA1BEFA37DCCDE0108
:10DE2A0097960E94657BEC93A3EBB0E00A2EEC91E7
:10DE3A00AFA10895A0912C07E3E60E94727D0E2EF1
:10DE4A00A52FE3E60E94727DE0210895A0E0B0E0EC
:10DE5A0080E09FE30E94287C30CBA0911305BB276A
:10DE6A00E0910E07F0E0EA0FFB1FE75FFA4F089513
:10DE7A00A091CC05A9CDA0912C07E3E60E94727D62
:10DE8A00E0210895E0912C05EF5FE0932C05E091E5
:10DE9A002B05A0912C05EA170895E0912B07F0E0D5
:10DEAA00DE011396AE0FBF1FAC910895EF5FEC939E
:10DEBA00E0E0E09330050895E0912B07F0E0EE589A
:10DECA00F84FA0810895A0912B07B0E0AE58B84F43
:10DEDA00EC910895EC93E0E0E09330050895E09129
:10DEEA002B07F0E0EA5FF84FA0810895A0912B0775
:10DEFA00B0E0AA5FB84FEC910895A0912B07B0E06B
:10DF0A00AB59B84FEC910895E0912B07A3E0B8E024
:10DF1A00F0E0DDCEFE93EE93E0E0E0933005089565
:10DF2A00A0912B07B0E0A659B84FEC910895A091A3
:10DF3A002B07B0E0AF5BBA4FEC910895E0912B0745
:10DF4A00F0E0EA5BFA4FA081A1300895A0912B0777
:10DF5A00B0E0AA5BBA4FEC910895E091B707F0914F
:10DF6A00B80708950E940A65F8DFD0DAA2E5B8EB8F
:10DF7A008AE391E40E94287CADEFB7E00C949F6796
:10DF8A00ECDFC4CAA3E3B3E383E091E40E94287CF4
:10DF9A00A9EFB7E00C949F67E091FD07F091FE07A7
:10DFAA00089535970E94AD65E0E0E0933005089545
:10DFBA000E940F65EAE00E94097E0895A0918307F6
:10DFCA00B09184070895A0912B07B0E0AD5CBA4FD9
:10DFDA00EC910895E0939707F0939807E0E0E093B7
:10DFEA008D07E0938E07E0931E09E0931F09E093E3
:10DFFA002009E09321090E94AB67A6E1B9E097CB1B
:10E00A000E94C567E091A507F091A607AAE1B9E0C9
:10E01A008ECBA0911A09B0911B0980911C0990918D
:10E02A001D0989DB0E94767CE0931A09F0931B098B
:10E03A0060931C0970931D090E948D670E94D7671F
:10E04A00E0E0E09330050895E091A507F091A60776
:10E05A000895E093A507F093A607E0E0E0938D0703
:10E06A00E0938E07E0931E09E0931F09E0932009CD
:10E07A00E09321090E94AB67A6E1B9E058CBE09191
:10E08A000E07F0E0E75FFA4F0895DF01EC910ECF3B
:10E09A00E0910E07F0E0E65FFA4F0895E0910E076F
:10E0AA00F0E0E55FFA4F0895E0910E07F0E0E45FD3
:10E0BA00FA4F0895E0910E07F0E0E35FFA4F0895F2
:10E0CA00E1E00E948B7D0E2E08950E942D650E942C
:10E0DA003665EAE0F0E060E070E00E94317E40D808
:10E0EA000E94E97D0E942D65E0E0E09330050895E5
:10E0FA00ACE5BFE882E290E40E94287CA3ECB5EF8D
:10E10A0088E490E40E94287CA5E9B7E00C949F6714
:10E11A00DF01CB01ECE5FFE862E270E40E94767C65
:10E12A00DF01CB01E3ECF5EF68E470E40E94767C52
:10E13A00DE019C960E94657BCDCEA0910005B0E0E1
:10E14A0049CDA0910005BB27EAE0F0E00E945E7E7F
:10E15A000895F6DAA6CCE0912B07ADE0B8E0F0E03E
:10E16A00B6CDA52FEFE50E94727D0E2EA0E0F6FC3B
:10E17A00A1E00895E0910108F09102080895A52F01
:10E18A00E3E60E94727D0E2EA0E0F6FCA1E008955F
:10E19A00DF01EC91E1509ECEAA30E0E0BE07E0E05C
:10E1AA008E07E0E09E070895A0910105BB27EAE0EB
:10E1BA00F0E00E945E7E08950BD9EAE0F0E00E944A
:10E1CA00197E0895A0915308B0915408809155087A
:10E1DA00909156080895E093E307F093E4070895B1
:10E1EA00F0E00E94A77D0E2AE0917B090895A09194
:10E1FA00AE08B091AF0808950E94B37D4BCCA091B0
:10E20A00B008B091B1080895A091B208B091B308CE
:10E21A000895E093E608F093E7086093E80870939E
:10E22A00E9080895A091E608B091E7088091E80806
:10E23A009091E90808950E941B690E94567E0895EC
:10E24A00E1E00E94727D0E2A0895E170EE0FEE0F52
:10E25A00EE0F0895E0E00E94907DE0290895EAE03B
:10E26A00E0932F07E0933007E0933107E0933207FA
:10E27A00E0933307E0933407E0933507E0933607DA
:10E28A00E09337070895EAE0E0933807E093390707
:10E29A00E0933A070895EAE0E0933B07E0933C07EE
:10E2AA00E0933D070895EA2FE295E07FEE0FEE0F27
:10E2BA000E2E0895EA2FE295E07FEE0FE00DA09171
:10E2CA006207EA0FE093620708950E94287CD8014A
:10E2DA000E946D7D0E94C57E0E94BB7C089546DA2D
:10E2EA00E4E6F0E00E942C7EDF01EAE0F0E00E9422
:10E2FA005E7E08953BDA6ECCDF01EAE0F0E00E9430
:10E30A005E7EE093320708950E94FC7CDF0162CCB6
:10E31A00EAE0E09331070895A0918C08B0918D0846
:10E32A000895E0938E08F0938F080895A0918E08BF
:10E33A00B0918F080895FADF4DCCDF01EAE0F0E0F2
:10E34A000E945E7EE0932F070895F0DFEAE0F0E096
:10E35A000E945E7EE09330070895E0918C08F09168
:10E36A008D080895EF89ACEAB8E0F0E0B0CC0E94DD
:10E37A00A57EE73FAFEFFA0708950E94A57E0E94A7
:10E38A00FC7C0895E4E6F0E00E942C7EDF01EAE0DE
:10E39A00F0E00E945E7E0895DF01EAE0F0E00E946C
:10E3AA005E7E0895EAE0F0E00E945E7E0895A3ECA6
:10E3BA00B5EF80E091E40E94287C0895E0930A0971
:10E3CA00F0930B0960930C0970930D090895E0917D
:10E3DA000A09F0910B0960910C0970910D09A0E0EE
:10E3EA00B0E088EC92E40E94767C08950E94287C32
:10E3FA00E5CFE0933907EAE0E0933A070895E0931E
:10E40A003B07E0E0E0933C070895A0911C050C94BB
:10E41A00C563A0911D050C94C563A0911E050C94BB
:10E42A00C563A0911F050C943E69A0E0F799A1E08D
:10E43A00EA2FE295E07FA09162070895E8EEF3E003
:10E44A000E94197EDF01EAE0F0E00E945B7E0895F7
:10E45A000E945865E4E6F0E00E94197EDF01EAE0D6
:10E46A00F0E00E945B7E08950E945865EAE0F0E0C1
:10E47A000E94197EDF010895EAE0F0E00E945B7EC7
:10E48A0008950E94317EDF01CB01EAE0F0E060E00E
:10E49A0070E00E946C7E0895A031E7E2BE07E0E0DA
:10E4AA008E07E0E09E070895E0E1F7E260E070E0A1
:10E4BA000895A83EE3E0BE07E0E08E07E0E09E078D
:10E4CA000895E8EEF3E060E070E00895A436E0E035
:10E4DA00BE07E0E08E07E0E09E0708950E943665D9
:10E4EA00EAE0F0E060E070E008950E946C7EE0935C
:10E4FA003D070895E0933707E4E7E0933807089566
:10E50A00D3DF0E94567EDF01CB01EAE0F0E060E053
:10E51A0070E00E94707EE09339070895D2DF0E946E
:10E52A00567EDF01CB01EAE0F0E060E070E00E9495
:10E53A00707EE0933A070895DF01CB01EAE0F0E04C
:10E54A0060E070E00E94707E08950E942166EAE011
:10E55A00F0E060E070E008950E94567EEDCF0E94E0
:10E56A00707EE0933D070895E0916107E058E093DB
:10E57A006107A0912C0708950E943366EAE0F0E053
:10E58A0060E070E008954DD90E94FC7C0895E09106
:10E59A006107E058E09361070895E5E0E0933807E2
:10E5AA00E8E7E09339070895E8EEF3E00E942C7E4D
:10E5BA00F3CEE8ECF0E00E94197EDF015DCFE4E1E2
:10E5CA00F0E00E94197EDF0157CFE091FB07F0913E
:10E5DA00FC07F695E7950895A0919907B0919A07D7
:10E5EA000895EAE0F0E00E94197EDF0145CFE3E7F3
:10E5FA00E0933B07E8E3E0933C070895E09338078C
:10E60A00E8E3E09339070895E4E6F0E00E94197E12
:10E61A00DF0132CFA091D408B091D5080895E0E186
:10E62A00F7E20E942C7EB8CEE091D408F091D5088A
:10E63A000895FADF0E94FC7C0895E7E3E093370728
:10E64A00E8E7E0933807E0E5E09339070895ECE757
:10E65A00E0933707E7E7E09338070895E9E3E093A3
:10E66A003707E8E7E0933807E0E5E09339070895CC
:10E67A00A3E00E947F61E0916005E295EF70AAE055
:10E68A00EA02F001E0930005E0916005EF70A091C5
:10E69A000005EA0FE0930005E0916105E295E1705B
:10E6AA00AAE0EA02F001E0930105E0916105EF704A
:10E6BA00A0910105EA0FE09301050895B6D9A3ECEC
:10E6CA00B5EF88E09FE30E94287C0895E050F2406D
:10E6DA00ACD9A2E4B0E685E69BE30E94287C0895C3
:10E6EA00A0911708B09118080895EEE3E093370750
:10E6FA00ECE7E09338070895A0911908B0911A0839
:10E70A000895E0915A09F0915B0960915C09709152
:10E71A005D090895E0933707E3E7E0933807089522
:10E72A00A091D008B091D1080895A0918B07B0911B
:10E73A008C070895E9E7E0933707E0E5E0933807A7
:10E74A00EDE0E0933907A091D707B091D807A43636
:10E75A00E0E0BE070895A091D707B091D8070895C1
:10E76A00E0933C07F8DF88CE0E94ED680E94D765E7
:10E77A000E94317EE093D507F093D60708950E9450
:10E78A00727D0E2E0E94456630D90E94D97DE02105
:10E79A0008950E94FB680E94D7650E94317EE0932B
:10E7AA00D507F093D6070895E0933907A091D507C6
:10E7BA00B091D6070895A091D507B091D6070895CC
:10E7CA00E0933C07F8DF58CE0E94FB680E94576628
:10E7DA000E94317EE093E107F093E2070895E2E0B8
:10E7EA00E0933607ECE7E09337070895EDE0E0930E
:10E7FA003807A091E107B091E20706CFE0933B0703
:10E80A00E0913B07E0300895A091E107B091E2075B
:10E81A000895E0933C07F8DF2FCEA0916308B091EA
:10E82A0064088091650890916608EAE0F0E060E08B
:10E83A0070E00E946C7EE0933707A0913707AA30F8
:10E84A000895E4E7E0933807A0915F08B091600863
:10E85A008091610890916208EAE0F0E060E070E07F
:10E86A0010CEE0933907A0915F08B09160088091BB
:10E87A00610890916208EAE0F0E060E070E00E94CE
:10E88A006C7EE0933A07E4E5E0933B07A0915B08CE
:10E89A00B0915C0880915D0890915E08EAE0F0E032
:10E8AA0060E070E0EECDE0933C07A0915B08B09188
:10E8BA005C0880915D0890915E08EAE0F0E060E013
:10E8CA0070E013CEE0933A07E0913A07E0300895FA
:10E8DA00E0933B07A0913A07EAE00E94727D0E2E70
:10E8EA00A0913B070C943E69E0916107EF77E093B2
:10E8FA006107EAE0E09336070895E0933707E0E01E
:10E90A00E09338070895E0933A07E8E7E0933B0776
:10E91A000895E0E00E94727D1E2E0895E0933C0760
:10E92A00E7E7E0933D070895ECE7E0933807E0E571
:10E93A00E09339070895AF85E4E00E94727DAE2F17
:10E94A00E0E0F799E1E0EA230895AF85E5E00E9467
:10E95A00727DAE2FE0E0F799E1E0EA230895ECE753
:10E96A00E0933B07E0E5E0933C070895E7E7E0938F
:10E97A003B07E9E3E0933C0708950E94727DAE2FBE
:10E98A00E0E0F799E1E0EA230895A0911107E5E0B4
:10E99A000E948B7D0E22A0E0F799A1E00C94C5633A
:10E9AA00A0912807E4E10E94727DE0210895E09396
:10E9BA003A07EAE0E0933B070895E8E7E0933C076B
:10E9CA00EBE0E0933D070895E9E7E0933C07E0E5D3
:10E9DA00E0933D070895E2E0E0933005E0E0E0933C
:10E9EA001B050895E9E00E948B7D0E22A0E0F799AD
:10E9FA00A1E00C94C563E8E00E94907D0E2EA0E091
:10EA0A00F799A1E00C94C563E0912B07F0E0EE586A
:10EA1A00F84FE0810895E0912D07F0E0E25DF84FAC
:10EA2A0008950E94727D0E2EA52F0895F0E0E093BE
:10EA3A00F707F093F8070895E0912B07F0E0EA5FF3
:10EA4A00F84FE0810895E093F707F093F8070895E7
:10EA5A00E0912B07F0E0EA5BFA4FE0810895E4E0E9
:10EA6A000E94097EF0CFAE0FBF1F0E94A57E0895B7
:10EA7A000E94727D0E2AA52F0895A091F707B091E2
:10EA8A00F8070895E0211E2AA52FEEE50E94727D5F
:10EA9A000E2EA091520508950E94907D0E22A091FB
:10EAAA0052050895E0936107E0E0E0936207E0937E
:10EABA006307E093020508950E94867D0E2EA52F16
:10EACA000895E0E1F7E20E94197EDF01D5CCD5DF97
:10EADA00A436E0E0BE070895D0DF83CDCEDFCCCCEC
:10EAEA00E0933307E9E7E09334070895E751FA4FD3
:10EAFA00A0810C94C063EDE0E0933C07E0933D07EE
:10EB0A000895E0933507E091F707F091F8073097F9
:10EB1A000895E0E0E0933B07E1E7E0933C07E093E8
:10EB2A003D070895E0E0E0933C07E4E5E0933D0704
:10EB3A000895E0933307E3E7E09334070895E093F9
:10EB4A003307ECE7E0933407E8E3E09335070895E9
:10EB5A00E0933907EDE0E0933A070895A09178072A
:10EB6A00BB2720CCE0933307EEE3E0933407089504
:10EB7A00E0933407E0E5E09335070895E09333071F
:10EB8A00E8E7E09334070895E0933407E9E3E09374
:10EB9A0035070895E0933307EEE5E09334070895C7
:10EBAA00E0933B07EEE3E0933C07EEE5E0933D0795
:10EBBA000895E0933A07E0E0E0933B070895E7E71A
:10EBCA00E0933C07E8E7E0933D070895E7E7E09321
:10EBDA003307E9E3E09334070895E0933A07E7E758
:10EBEA00E0933B070895E0933C07E9E7E0933D078C
:10EBFA000895E0933807E0E5E09339070895E09334
:10EC0A003A07E9E7E0933B070895E0933C07E8E712
:10EC1A00E0933D070895E0933707E8E3E093380768
:10EC2A000895EEE3E0933C07E0E5E0933D0708959D
:10EC3A00E0933307E0E3E09334070895E0933A075B
:10EC4A00E4E5E0933B070895E0933307E7E7E093B1
:10EC5A0034070895B7DAEAE0F0E060E070E008957A
:10EC6A00E0933407E0E6E09363070895E0933707FB
:10EC7A00E0E5E09338070895E7E7E0933707E9E32B
:10EC8A00E09338070895E0933907A0916C08B09192
:10EC9A006D08A436E0E0BE070895A0916C08B09113
:10ECAA006D080895E8E3E0933A07E1E0E0933B0753
:10ECBA00E4E599CFE2DE0E94D97E0895E9E3E09384
:10ECCA003307E0E5E0933407EEE3E0933507089570
:10ECDA00E0933707E091F707F091F8073097089526
:10ECEA00E0933C07E8E5E0933D070895EEE5E093FD
:10ECFA003507EEE0E09337070895E9E3E093330739
:10ED0A00E0E5E09334070895A0919D07B0919E072E
:10ED1A000895E0933307E8E5E09334070895E8E7B8
:10ED2A00E0933A07E0E5E0933B07E1E0E0933C0734
:10ED3A00E3E7E0933D070895EEE3E0933807E4E75D
:10ED4A0058CBE0E0E0933B07E5E05FCFEEE3E093EA
:10ED5A003B07E4E7E0933C07E0E5E0933D070895CD
:10ED6A00E0933C07E0E5E0933D070895E093380718
:10ED7A00E8E7E0933907E0E5E0933A07E3E6E09352
:10ED8A003B07E9E3E0933C07EBE0E0933D07089596
:10ED9A00E8E7E0933A07E1E0E0933B07E4E523CFB5
:10EDAA00EEE3E0933B07ECE7E0933C070895E0933A
:10EDBA003C07E4E5E0933D070895E0933B07EAE06A
:10EDCA00E0933C070895E0933C07EDE0E0933D07AC
:10EDDA000895E0933907E9E7E0933A070895E09345
:10EDEA003C07E5E0E0933D070895E8E5E093330743
:10EDFA00E1E0E09334070895A0912707BB27D2CA20
:10EE0A00E0933307E0E5E09334077BCEE0E5E09357
:10EE1A003B07E9E7E4CFE0933407E8E7E0933507F7
:10EE2A000895E0933307E8E3E09334070895E7E7AA
:10EE3A00E0933707E0E4E0933807E8E7DACAE093BB
:10EE4A003B07E4E5E0933C070895E0933407EAE0E2
:10EE5A00E09335070895A091A707B091A8070895F0
:10EE6A00E9E3E0933907E4E54ECD0E94A57EDF0190
:10EE7A00B8CB0E94A57EDF01FFCAE1E0E093330729
:10EE8A00E4E5E09334070895A091D307B091D4073D
:10EE9A000895E0933507E09164070895E0916407C7
:10EEAA000C946F63A0916407E7E00E94907D0E2E98
:10EEBA00ECE00E948B7DE0210895E0916407F0E088
:10EECA003897E25BFA4FE0810895E170E0933D07DD
:10EEDA00E0916407F0E00895E751FA4FE081E030ED
:10EEEA000895E0933B0707CEA0916407EBE00E94E8
:10EEFA00907D0E2EE0E10E948B7DE0210895F0E0E6
:10EF0A003C97EB51FA4FE0810895E0916407F7CFFF
:10EF1A00E695E695E695E1700895A0916407EFE01D
:10EF2A000E94907D0E2E0C94F46EE0916107E068C9
:10EF3A00E09361070895E0933307E0916407089529
:10EF4A00E0916407F0E07097AFEAB7E00C946C6E5A
:10EF5A000E94A57EDF0158CBE0933D07E09164074C
:10EF6A00F0E008950E94907D0E2EA0916407089506
:10EF7A00E0916407F0E07497DE01DB960C946C6E06
:10EF8A000E94A57E0C94616C0E94A57EDF010C9400
:10EF9A00EF6D0E94A57EED39AFEFFA0708950E9442
:10EFAA00A57EB2C9F0E07897DE01D3960C946C6E18
:10EFBA00E0916407F7CFE0933C07A0913B07EAE0B2
:10EFCA000E94727D0E2EA0913C070C943E69E0913E
:10EFDA000A07A2E9B8E0F0E00C946C6E0E94907DFA
:10EFEA00E021E1290895F0E0B897E351FA4FA081B2
:10EFFA00B0E00895A0916407EBE2B4CFE0E30E9489
:10F00A008B7DE0210895F0E0BC97E65EF84FA08181
:10F01A00B0E00895A0916407EFE2A4CFF0E0F09782
:10F02A00A5EEB7E00C946C6EA3E2B8E00C946C6E9B
:10F03A00A091E008B091E1080895FADFA436E0E073
:10F04A00BE070895F5DFA83EE3E0BE070895E3E7AB
:10F05A00E0933707EBE0E09338070895A09139076A
:10F06A00EAE00E94727D0E2EA0913A070895E0937D
:10F07A003C07E3E6E0933D0708950E94F365EAE062
:10F08A00F0E060E070E008950E940566EAE0F0E0D2
:10F09A0060E070E00895E89431F8EAE0E0932F0721
:10F0AA00E093300735C9E0933207EAE0E09333078B
:10F0BA00CCCEE170E295E07FAE2F0895E295EF7035
:10F0CA00E695E170E295E07FEE0FEA2BAE2F089508
:10F0DA00E295EF70E695E695E170E295E07FEE0F36
:10F0EA00EE0FEA2BAE2F0895E295E170E795E0E086
:10F0FA00E795EA2BAE2F0895EA2BAE2FE09133075E
:10F10A000895E695E695E170EE0FEE0F0895E695FF
:10F11A00E695E6959AC8EA2BAE2FE0913507089551
:10F12A00EA2BAE2FE09134070895EA2BAE2FE09137
:10F13A0061070895E695E170E295E07FEE0FEA2B0C
:10F14A00AE2F0895E695E695E170E295E07FEE0F21
:10F15A00EE0FEA2BAE2F0895E795E0E0E795E5CFAD
:10F16A00EA2BAE2FE0913B070895E295EF70E69502
:10F17A00E170EE0F0895E295EF70E695E695E1707D
:10F18A00EE0FEE0F0895EA2BAE2FE0913C0708959B
:10F19A00E295EF70E6958DCFEA2BAE2FE091390715
:10F1AA000895E295EF70E695E6950895EA2BAE2F5D
:10F1BA00E0913D070895EA2BAE2FE09137070895B5
:10F1CA00E795E0E0E795EA2BAE2F0895EA2BAE2FFC
:10F1DA00E0912F070895E170E295E07FEE0F089520
:10F1EA00E695E170E295E07FEE0FEE0F0895EA2BC7
:10F1FA00AE2FE09162070895E695E695E170EE0F6D
:10F20A000895EA2BAE2FE09130070895E295EF704A
:10F21A00E695E170D5CFE695E170EE0FEE0F089511
:10F22A00EA2BAE2FE09163070895EA2BAE2FE09107
:10F23A0031070895EA2BAE2FE091320708954498DA
:10F24A0084E08A95F1F7E1E0E0932D070895439869
:10F25A0084E08A95F1F70895A0912D07ECE0EA1B66
:10F26A00089584E08A95F1F7439A84E08A95F1F744
:10F27A000895429A84E08A95F1F7449A84E08A953F
:10F28A00F1F7DDCFA0E0B0E080E090E00E94BE7E22
:10F29A00E0E00895E0E0E0939307E093940708958F
:10F2AA00EE85F0E0E557F64FE0810895F0E0A09191
:10F2BA009307B0919407EA0FFB1FE0939307F0932B
:10F2CA0094070895EFA7F8ABE0919009FF27662706
:10F2DA007727E0932F08F0933008609331087093F2
:10F2EA003208E0919109E09327050895E0E0E09360
:10F2FA009C09E09303050895E0E0E0938B09E0930D
:10F30A008C09E0938D09E0938E09E0938F090C94A0
:10F31A008864E0E0E0939209E0939309E09394090A
:10F32A00E0939509E0939C090895F0E0EA27FB270A
:10F33A00E0939307F09394070895E0919307F0916F
:10F34A009407F070DF010895E0912605EE0FE0932F
:10F35A002605E0918C090895AFE8B9E0EC91E695AD
:10F36A00E695EC930895E981ABE1B8E0F0E00C94FE
:10F37A006C6EE0918D09F0E0E370F070FE2FE0E032
:10F38A00ED93FC93E091D4050895F0E0EE0FFF1F92
:10F39A00EA0FFB1F0F01DF010E94A57EDF01E0914A
:10F3AA008E09F0E0EA0FFB1FD001ED93FC9308955C
:10F3BA00E091D405F0E0DE01DB960C946C6EE091EE
:10F3CA008F09F0E0E370F070FE2FE0E0ED93FC931C
:10F3DA00C3CFED91FD91E050F440FE93EE93089572
:10F3EA00EE0FFF1FEA0FFB1F0F01DF010E94A57E30
:10F3FA00DF010895F0E0EA0FFB1FD001ED93FC93C3
:10F40A000895E091D405F0E0DE01D3960C946C6E79
:10F41A00EC93A091D405B0E00895EC93A5E9B9E086
:10F42A00EC910895E0919509E170F7CFEC93E091A2
:10F43A00D405AEEBB8E0F0E00895E0919609F0E06B
:10F44A00E370F070ED93FC93E091D4050895ED918B
:10F45A00FD91FE2FE0E0FE93EE93A6E9B9E0EC9170
:10F46A00E695E6950895A6EBB8E0F0E00C946C6E8C
:10F47A00AAE7B8E0F0E00C946C6E0F01A081E0916D
:10F48A009609E170EA2BD001EC930895EE0FEE0F86
:10F49A00EA0FA0912605EA2BE09326050895A0E03D
:10F4AA00A083E981F0E00895E0E0F0E0ED93FC93B9
:10F4BA000895ED87EDE4E093C4000C947A67AE2FCB
:10F4CA000E944661A09168080C9446610E944661B8
:10F4DA00E0919407AE2F0E944661A09193070C9485
:10F4EA0046610E94DA69E0E0F1E00E942C7E08950C
:10F4FA00A1E00E944661A6E30C944661A09193079D
:10F50A000C944661E0912B07F0E0EE58F84FBF01EA
:10F51A00A0810C94C063EC91E295E07FEC9308958E
:10F52A00A3E5B7E0EC91EE0FEE0FEC93E3E5F7E01D
:10F53A000F01E0810895EA0FD001EC93A3E5B7E04B
:10F54A00EC910895E3E5F7E00F01E0810895E09179
:10F55A002607F0E00E94ED690E94E17DDF01E4E602
:10F56A00F0E00E94197E0895E0935707E09127077B
:10F57A00F0E00E94ED690E94E17DDF01E4E6F0E03F
:10F58A000E94197E0895E0935807E0E0E0935A0735
:10F59A00E09359070895E0912D07F0E0E05BF84FFA
:10F5AA000895E8E8E093C1008AE194E00197F1F751
:10F5BA00E0E0E0932D07089584E398E00197F1F7DE
:10F5CA00E0E9E093C1000895EC91EE0FEE0FEC93A1
:10F5DA000895EE0FEC93B6CFE0935407A4E5B7E095
:10F5EA00EC91EE0FEC93E4E5F7E00F01E08108956A
:10F5FA00EA0FD001EC93A4E5B7E0EC91EE0FEC939F
:10F60A000895E0935407A4E5B7E0DECFA0913B0547
:10F61A00E2E00E948B7D0E2EA09138050C94BD6C01
:10F62A000E948B6AADECBCEC8CEC9DE30C94A76851
:10F63A001E2EA0913B05E1E00E94907D0E2EA09126
:10F64A0038050C94BD6C109639F088EB9BE0019755
:10F65A00F1F7A8951197C9F708953097604070405F
:10F66A0009F070580895552342F4503811F4E0FF18
:10F67A0004C03196691F791F6BF050E8572711F4BF
:10F68A005F93CFC05F3F31F0660F000C57956795C7
:10F69A00752F08955F9300200AF0CFC0C8C050E8C4
:10F6AA00192E1522880F991F9527550F879550E80F
:10F6BA00072E0522660F771F7527550F6795089540
:10F6CA00689401C0E8945F93F2DF703818F07F3FC6
:10F6DA0008F4A7C056E1571BAAF4519558300EF406
:10F6EA00593030F0EFEFFFEF6FEF7FE777F91AC08D
:10F6FA0077275523B9F0EE0FFF1F661F771F5A951C
:10F70A00D1F710C07727583028F0EF2FF62F672F40
:10F71A005850F9CF552331F076956795F795E795C7
:10F72A005A95D1F700200AF466D15F91089568943A
:10F73A0001C0E894309760407040B1F0002426F090
:10F74A00772312F4009457D1172E7EE1112032F05C
:10F75A007A95EE0FFF1F661F111CF9CFEF2FF62FB8
:10F76A00612D5F938ADF5F9108954F93AF01FD0189
:10F77A00DA01AB01BC01CA01402D012C142E4F91B4
:10F78A000895EA0FFB1F681F0895E095F0956095AC
:10F79A00EF5FFF4F6F4F08955F9381DF903871F1EC
:10F7AA0050E8152604C05F937ADF903839F1703833
:10F7BA0021F1572F591B2BF112F4D7DFFACF583109
:10F7CA0018F0AA27BB278827583028F0AB2FB82F64
:10F7DA0088275850F9CF552329F08695B795A795CC
:10F7EA005A95D9F7502D512572F0CBDF38F4679529
:10F7FA00F795E795739513F420C0B7DF3EDF5F9165
:10F80A000895D8F7FBCFEA1BFB0B680B51F010F4F5
:10F81A000094BBDF662392F3EE0FFF1F661F7A95F3
:10F82A00CBF7EE27FF27662777275F910895EFEF3B
:10F83A00FFEF6FE77FEF5F910895EFEFFFEF6FE75D
:10F84A007FE75F9108955F932ADF703851F390380C
:10F85A0041F301240894791F23F41CF300203AF39E
:10F86A00ECCF0F921F932F933F934F931127222789
:10F87A009927689FA0018F9F302D410D591F6B9FBB
:10F88A00300D411D591F8E9F27D0BF9F25D06A9FDB
:10F89A0023D0BE9F1DD0AF9F1BD0AE9F110D291F35
:10F8AA00391F491F591FE32FF42F652F522F4F91EC
:10F8BA003F912F911F910F9066232AF0550FEE1F4B
:10F8CA00FF1F661F02C073954BF2CDDE5F9108954C
:10F8DA00100D211D391F02C0200D311D491F591F4E
:10F8EA0008955F93DCDE703821F411200AF49FCF6B
:10F8FA00A4CF903809F495CF01240894970B1BF4F0
:10F90A00D4F30020F3CF792F1F932F933F934F9374
:10F91A0011241127222733274427552790E2AE17AF
:10F92A00BF078607410730F0AE1BBF0B860B410BA2
:10F93A00089401C08894551F221F331F111CAA1F47
:10F94A00BB1F881F441F9A9551F7F901612D4F91EA
:10F95A003F912F911F91662332F0550FEE1FFF1F23
:10F96A00661F7A9543F27FDE5F91089599239AF094
:10F97A00772342F0971748F029F4AE17BF07860796
:10F98A0020F031F0989488940895989408940895F2
:10F99A001894889408957723C2F7971798F3A9F7CC
:10F9AA00EA17FB07680788F399F3ECCFDFDFE1E09A
:10F9BA0011F008F4EE270895D9DFE1E009F008F024
:10F9CA00EE270895D3DFE1E009F008F4EE27089561
:10F9DA00EA0FFB1F681F791F0895EA1BFB0B680BD0
:10F9EA00790B0895AE1BBF0B860B970B0895F19503
:10F9FA00E195F0400895F09560957095E195FF4F77
:10FA0A006F4F7F4F0895EE230E2EEA2F19F0EE0F57
:10FA1A000A94E9F70895EE230E2EEA2F19F0E695D7
:10FA2A000A94E9F70895EE230E2EFD0121F0EE0F58
:10FA3A00FF1F0A94E1F70895EE230E2EFD0121F02F
:10FA4A00F695E7950A94E1F70895EE230E2EFD0147
:10FA5A00BC0131F0EE0FFF1F661F771F0A94D1F722
:10FA6A000895EE230E2EFD01BC0131F075956795C0
:10FA7A00F795E7950A94D1F70895EE230E2EFD0126
:10FA8A00BC0131F076956795F795E7950A94D1F719
:10FA9A000895EE0FFF1FEE0FFF1F0895F595E795E6
:10FAAA00F595E7950895EF2FFF27E7FDFFEF0895F6
:10FABA00E62FF72F60E070E00895FE2FFF0FFF0B8F
:10FACA006F2F7F2F08956F2F660F660B762F08957D
:10FADA008B2F880F880B982F0895EA17E1E009F019
:10FAEA00EE270895EA17E1E009F4EE270895AE1724
:10FAFA00E1E00CF4EE270895AE17E1E00CF0EE27F2
:10FB0A000895EA17E1E00CF0EE270895AE17E1E058
:10FB1A0008F0EE270895EA17E1E008F0EE270895C5
:10FB2A00EA17FB07E1E009F0EE270895EA17FB0759
:10FB3A00E1E009F4EE270895AE17BF07E1E00CF003
:10FB4A00EE270895EA17FB07E1E00CF0EE27089587
:10FB5A00AE17BF07E1E008F0EE270895EA17FB07A2
:10FB6A00E1E008F0EE270895EA17FB07680779072E
:10FB7A00E1E009F0EE270895EA17FB07680779071D
:10FB8A00E1E008F4EE270895AE17BF078607970746
:10FB9A00E1E008F4EE270895AE17BF078607970736
:10FBAA00E1E008F0EE270895EA17FB0768077907EE
:10FBBA00E1E008F0EE270895FA9FF02DEB9FF00D93
:10FBCA00EA9FE02DF10D08957A9F702D6B9F700DBD
:10FBDA00F89F700DE99F700D6A9F602D710DFB9F54
:10FBEA00600D711DE89F600D711D8827FA9FF02D29
:10FBFA00610D781FEB9FF00D611D781FEA9FE02DC4
:10FC0A00F10D681F781F08956E2F6A9FF0016B9F90
:10FC1A00F00D089574D0D0DF0EF4E9DE08957DD09A
:10FC2A00D3DF0EF4E8DE08950024112490E1AA0F30
:10FC3A00BB1F001C111C0E1A1F0A18F40E0E1F1EE1
:10FC4A0001C0A1609A9599F7FD01D001089557D096
:10FC5A00EBDF0EF4CCDE08953F934F935F930024BD
:10FC6A0011244427552730E2AA0FBB1F881F991F6A
:10FC7A00001C111C441F551F0E1A1F0A460B570B56
:10FC8A0028F40E0E1F1E461F571F01C0A1603A9589
:10FC9A0059F7FD01BC01D001CA015F914F913F9113
:10FCAA0008953BD0D9DF0EF4A6DE0895BDDFFD012D
:10FCBA000895E894B7FF04C0A095B095119668948A
:10FCCA00F7FD95DEB1DFFD010EF491DE0895C4DF84
:10FCDA00FD01BC010895E89497FF09C0A095B0956D
:10FCEA0080959095AF5FBF4F8F4F9F4F689477FD78
:10FCFA0082DEB2DFFD01BC010EF47DDE0895E894D8
:10FD0A00F7FF02C074DE6894B7FF06C0A095B095ED
:10FD1A00119600F8039400FA0895E89477FF02C058
:10FD2A006ADE689497FF0BC00024A095B095809571
:10FD3A0090951196801D901D00F8039400FA08957D
:10FD4A00ED91FC9111970895ED91FD916D917C9142
:10FD5A0013970895ED93FD936D937C930895E8812D
:10FD6A00F9816A817B810895E883F9836A837B83B9
:10FD7A000895A083B183828393830895689401C010
:10FD8A00E89401D0D7DC182E862F612D192E972FD3
:10FD9A00712D1B2EBF2FF12D1A2EAE2FE12D089596
:10FDAA00309760407040089500240A160B060895A3
:10FDBA0000240A160B06080609060895EA17FB0727
:10FDCA006807790708955A934A933A932A931A939C
:10FDDA000A9308955D814C813B812A8119810881AA
:10FDEA000895AC0FBD1F05900D928A95E1F708950D
:00000001FF
